:020000040800F2
:1000000000000220ED1B00083D1700084117000802
:1000100045170008491700084D17000800000000A8
:10002000000000000000000000000000518B0008EC
:100030005117000800000000E18B0008458C000803
:100040003D1C00083D1C00083D1C00083D1C00082C
:100050003D1C00083D1C0008BD8D0108C58D010830
:10006000CD8D0108D58D0108DD8D01083D1C0008EE
:100070003D1C00083D1C00085517000861170008CA
:100080003D1C00083D1C00083D1C00083D1C0008EC
:100090003D1C00083D1C00083D1C0008E58D0108C2
:1000A0003D1C00083D1C00086D1700083D1C0008A1
:1000B0003D1C00083D1C00083D1C00083D1C0008BC
:1000C0003D1C00083D1C00083D1C00088917000865
:1000D000951700083D1C00083D1C00083D1C000849
:1000E0000D8E01083D1C00083D1C00083D1C000849
:1000F0003D1C00083D1C00083D1C00083D1C00087C
:100100003D1C00083D1C00083D1C00083D1C00086B
:100110003D1C00083D1C0008A1170008AD17000891
:10012000B91700083D1C0008C5170008D1170008C2
:100130003D1C0008DD1700083D1C00083D1C0008A0
:100140003D1C00083D1C00083D1C00083D1C00082B
:100150003D1C00083D1C00083D1C00083D1C00081B
:100160003D1C00083D1C00083D1C00083D1C00080B
:100170003D1C00083D1C00083D1C0008000000005C
:080180003D1C00083D1C0008B5
:1001900010B5054C237833B9044B13B10448AFF3C1
:1001A00000800123237010BD3002002000000000F9
:1001B0006CEE010808B5034B1BB103490348AFF3CC
:1001C000008008BD00000000340200206CEE010831
:1001D00001F0FF01102A2BDB10F0070F08D010F8F8
:1001E000013B013A8B422DD010F0070F42B3F6D1FC
:1001F000F0B441EA012141EA014122F007047FF015
:1002000000070023F0E80256083C85EA010586EA6B
:10021000010685FA47F5A3FA87F586FA47F6A5FAA7
:1002200087F68EB9EED1F0BC01F0FF0102F00702B3
:1002300032B110F8013B013A83EA010313B1F8D15E
:100240000020704701387047002D06BF354603383F
:10025000073815F0010F07D1013015F4807F02BF78
:10026000013015F4C03F0130F0BC0138704700BFC9
:10027000034613F8012B002AFBD1181A01387047E6
:1002800081F0004102E000BF83F0004330B54FEA47
:1002900041044FEA430594EA050F08BF90EA020FB4
:1002A0001FBF54EA000C55EA020C7FEA645C7FEA47
:1002B000655C00F0E2804FEA5454D4EB5555B8BF6A
:1002C0006D420CDD2C4480EA020281EA030382EADB
:1002D000000083EA010180EA020281EA0303362D6D
:1002E00088BF30BD11F0004F4FEA01314FF4801C40
:1002F0004CEA113102D0404261EB410113F0004F52
:100300004FEA03334CEA133302D0524263EB430308
:1003100094EA050F00F0A780A4F10104D5F1200EA6
:100320000DDB02FA0EFC22FA05F2801841F1000101
:1003300003FA0EF2801843FA05F359410EE0A5F1D5
:1003400020050EF1200E012A03FA0EFC28BF4CF006
:10035000020C43FA05F3C01851EBE37101F00045BC
:1003600007D54FF0000EDCF1000C7EEB00006EEBC9
:100370000101B1F5801F1BD3B1F5001F0CD3490853
:100380005FEA30004FEA3C0C04F101044FEA4452AA
:1003900012F5800F80F09A80BCF1004F08BF5FEA31
:1003A000500C50F1000041EB045141EA050130BD11
:1003B0005FEA4C0C404141EB0101013C28BFB1F523
:1003C000801FE9D291F0000F04BF01460020B1FA6E
:1003D00081F308BF2033A3F10B03B3F120020CDA41
:1003E0000C3208DD02F1140CC2F10C0201FA0CF01F
:1003F00021FA02F10CE002F11402D8BFC2F1200C84
:1004000001FA02F120FA0CFCDCBF41EA0C01904039
:10041000E41AA2BF01EB0451294330BD6FEA040482
:100420001F3C1CDA0C340EDC04F11404C4F120026D
:1004300020FA04F001FA02F340EA030021FA04F37F
:1004400045EA030130BDC4F10C04C4F1200220FAD6
:1004500002F001FA04F340EA0300294630BD21FA14
:1004600004F0294630BD94F0000F83F4801306BFDA
:1004700081F480110134013D4EE77FEA645C18BFCE
:100480007FEA655C29D094EA050F08BF90EA020F65
:1004900005D054EA000C04BF1946104630BD91EA5D
:1004A000030F1EBF0021002030BD5FEA545C05D160
:1004B0004000494128BF41F0004130BD14F580049F
:1004C0003CBF01F5801130BD01F0004545F0FE4113
:1004D00041F470014FF0000030BD7FEA645C1ABF48
:1004E000194610467FEA655C1CBF0B46024650EA7F
:1004F000013406BF52EA033591EA030F41F40021AB
:1005000030BD00BF90F0000F04BF0021704730B530
:100510004FF4806404F132044FF000054FF0000105
:1005200050E700BF90F0000F04BF0021704730B5C6
:100530004FF4806404F1320410F0004548BF40429B
:100540004FF000013EE700BF42004FEAE2014FEAF0
:1005500031014FEA02701FBF12F07F4393F07F4FCB
:1005600081F06051704732F07F4208BF704793F0CE
:100570007F4F04BF41F40021704730B54FF46074E1
:1005800001F0004521F000411CE700BF50EA0102E4
:1005900008BF704730B54FF000050AE050EA01028D
:1005A00008BF704730B511F0004502D5404261EBFD
:1005B00041014FF4806404F132045FEA915C3FF43E
:1005C000D8AE4FF003025FEADC0C18BF03325FEADB
:1005D000DC0C18BF033202EBDC02C2F1200300FA8C
:1005E00003FC20FA02F001FA03FE40EA0E0021FAB1
:1005F00002F11444BDE600BF70B54FF0FF0C4CF49F
:10060000E06C1CEA11541DBF1CEA135594EA0C0F50
:1006100095EA0C0F00F0DEF82C4481EA030621EA8B
:100620004C5123EA4C5350EA013518BF52EA0335C6
:1006300041F4801143F4801338D0A0FB02CE4FF078
:100640000005E1FB02E506F00042E0FB03E54FF0A8
:100650000006E1FB03569CF0000F18BF4EF0010EA0
:10066000A4F1FF04B6F5007F64F5407404D25FEA9C
:100670004E0E6D4146EB060642EAC62141EA55514F
:100680004FEAC52040EA5E504FEACE2EB4F1FD0C91
:1006900088BFBCF5E06F1ED8BEF1004F08BF5FEA0F
:1006A000500E50F1000041EB045170BD06F00046C1
:1006B00046EA010140EA020081EA0301B4EB5C046E
:1006C000C2BFD4EB0C0541EA045170BD41F4801166
:1006D0004FF0000E013C00F3AB8014F1360FDEBF8B
:1006E000002001F0004170BDC4F10004203C35DA67
:1006F0000C341BDC04F11404C4F1200500FA05F3EA
:1007000020FA04F001FA05F240EA020001F000428A
:1007100021F0004110EBD37021FA04F642EB060100
:100720005EEA430E08BF20EAD37070BDC4F10C042A
:10073000C4F1200500FA04F320FA05F001FA04F2EE
:1007400040EA020001F0004110EBD37041F10001DA
:100750005EEA430E08BF20EAD37070BDC4F12005E5
:1007600000FA05F24EEA020E20FA04F301FA05F24D
:1007700043EA020321FA04F001F0004121FA04F2F5
:1007800020EA020000EBD3705EEA430E08BF20EAC5
:10079000D37070BD94F0000F0FD101F000464000FF
:1007A00041EB010111F4801F08BF013CF7D041EA81
:1007B000060195F0000F18BF704703F00046520085
:1007C00043EB030313F4801F08BF013DF7D043EA56
:1007D0000603704794EA0C0F0CEA135518BF95EA0C
:1007E0000C0F0CD050EA410618BF52EA4306D1D193
:1007F00081EA030101F000414FF0000070BD50EAB2
:10080000410606BF1046194652EA430619D094EA3B
:100810000C0F02D150EA013613D195EA0C0F05D125
:1008200052EA03361CBF104619460AD181EA030179
:1008300001F0004141F0FE4141F470014FF0000031
:1008400070BD41F0FE4141F4780170BD70B54FF0CC
:10085000FF0C4CF4E06C1CEA11541DBF1CEA13554C
:1008600094EA0C0F95EA0C0F00F0A7F8A4EB05042E
:1008700081EA030E52EA03354FEA013100F0888025
:100880004FEA03334FF0805545EA131343EA1263EE
:100890004FEA022245EA111545EA10654FEA0026A3
:1008A0000EF000419D4208BF964244F1FD0404F55C
:1008B000407402D25B084FEA3202B61A65EB0305B8
:1008C0005B084FEA32024FF480104FF4002CB6EB75
:1008D000020E75EB030E22BFB61A754640EA0C00F5
:1008E0005B084FEA3202B6EB020E75EB030E22BF35
:1008F000B61A754640EA5C005B084FEA3202B6EB76
:10090000020E75EB030E22BFB61A754640EA9C0034
:100910005B084FEA3202B6EB020E75EB030E22BF04
:10092000B61A754640EADC0055EA060E18D04FEAC2
:10093000051545EA16754FEA06164FEAC30343EA62
:1009400052734FEAC2025FEA1C1CC0D111F4801F2F
:100950000BD141EA00014FF000004FF0004CB6E728
:1009600011F4801F04BF01430020B4F1FD0C88BFC7
:10097000BCF5E06F3FF6AFAEB5EB030C04BFB6EBD2
:10098000020C5FEA500C50F1000041EB045170BDC5
:100990000EF0004E4EEA113114EB5C04C2BFD4EBF2
:1009A0000C0541EA045170BD41F480114FF0000E76
:1009B000013C90E645EA060E8DE60CEA135594EAF2
:1009C0000C0F08BF95EA0C0F3FF43BAF94EA0C0FF5
:1009D0000AD150EA01347FF434AF95EA0C0F7FF46A
:1009E00025AF104619462CE795EA0C0F06D152EABE
:1009F00003353FF4FDAE1046194622E750EA4106A2
:100A000018BF52EA43067FF4C5AE50EA41047FF4B2
:100A10000DAF52EA43057FF4EBAE12E74FF0FF3C17
:100A200006E000BF4FF0010C02E000BF4FF0010CE8
:100A30004DF804CD4FEA410C7FEA6C5C4FEA430C61
:100A400018BF7FEA6C5C1BD001B050EA410C0CBFB0
:100A500052EA430C91EA030F02BF90EA020F002012
:100A6000704710F1000F91EA030F58BF994208BF79
:100A700090422CBFD8176FEAE37040F00100704736
:100A80004FEA410C7FEA6C5C02D150EA013C07D18D
:100A90004FEA430C7FEA6C5CD6D152EA033CD3D0D8
:100AA0005DF8040B704700BF8446104662468C46D2
:100AB0001946634600E000BF01B5FFF7B7FF002805
:100AC00048BF10F1000F01BD4DF808EDFFF7F4FF2E
:100AD0000CBF012000205DF808FB00BF4DF808EDB9
:100AE000FFF7EAFF34BF012000205DF808FB00BFDC
:100AF0004DF808EDFFF7E0FF94BF012000205DF8FE
:100B000008FB00BF4DF808EDFFF7CEFF94BF0120B2
:100B100000205DF808FB00BF4DF808EDFFF7C4FFAB
:100B200034BF012000205DF808FB00BF4FEA410CF4
:100B30007FEA6C5C02D150EA013C0AD14FEA430CD7
:100B40007FEA6C5C02D152EA033C02D14FF0000014
:100B500070474FF0010070474FEA410212F5001252
:100B600015D211D56FF47873B3EB625212D94FEAF4
:100B7000C12343F0004343EA505311F0004F23FADE
:100B800002F018BF404270474FF00000704750EA33
:100B9000013005D111F0004008BF6FF000407047F0
:100BA0004FF00000704700BF4A0011D212F500124A
:100BB00011D20DD56FF47873B3EB62520ED44FEAB5
:100BC000C12343F0004343EA505323FA02F0704735
:100BD0004FF00000704750EA013002D14FF0FF3073
:100BE00070474FF0000070474FEA4102B2F1E04316
:100BF00024BFB3F5001CDCF1FE5C0DD901F0004C04
:100C00004FEAC0024CEA5070B2F1004F40EB830053
:100C100008BF20F00100704711F0804F21D113F17F
:100C20003872BCBF01F00040704741F480114FEAB8
:100C30005252C2F11802C2F1200C10FA0CF320FA41
:100C400002F018BF40F001004FEAC1234FEAD3235E
:100C500003FA0CFC40EA0C0023FA02F34FEA4303C8
:100C6000CCE77FEA625307D150EA01331EBF4FF051
:100C7000FE4040F44000704701F0004040F0FE406C
:100C800040F40000704700BF53B94AB9002908BFBB
:100C900000281CBF4FF0FF314FF0FF3000F0A6B925
:100CA000ADF1080C6DE904CE00F03CF8DDF804E08D
:100CB000DDE9022304B0704738B500220023044662
:100CC0000D46FFF70BFF28B920462946BDE83840FE
:100CD00000F00AB8204605F1004100F005F8404256
:100CE00061EB410138BD00BFD0B50C4B0022064678
:100CF0000F46FFF781FCFFF757FF0446FFF702FCA2
:100D0000074B0022FFF778FC02460B463046394677
:100D1000FFF7BAFAFFF748FF2146D0BD0000F03DCB
:100D20000000F0412DE9F047089E0D4604460F46AD
:100D3000002B4AD18A42944665D9B2FA82F343B174
:100D400002FA03FCC3F120029F4020FA02F217438B
:100D50009C404FEA1C4E1FFA8CF5B7FBFEF1220CAB
:100D60000EFB117742EA074201FB05F090420AD9D7
:100D70001CEB020201F1FF3780F01C81904240F22F
:100D8000198102396244121AA4B2B2FBFEF00EFBC2
:100D9000102244EA024400FB05F5A5420AD91CEBE7
:100DA000040400F1FF3280F00781A54240F2048183
:100DB0006444023840EA0140641B00211EB1DC405B
:100DC0000023C6E90043BDE8F0878B4208D9002E16
:100DD00000F0ED800021C6E900050846BDE8F08777
:100DE000B3FA83F1002949D1AB4202D3824200F227
:100DF000F880841A65EB030201201746002EE2D02A
:100E0000C6E90047DFE702B9FFDEB2FA82F3002B42
:100E100040F090808A1A4FEA1C471FFA8CFE01218D
:100E2000B2FBF7F507FB1520220C42EA00420EFB4D
:100E300005F0904208D91CEB020205F1FF3802D2FE
:100E4000904200F2CB804546121AA4B2B2FBF7F0F2
:100E500007FB102244EA02440EFB00FEA64508D917
:100E60001CEB040400F1FF3202D2A64500F2BB8065
:100E70001046A4EB0E0440EA05409FE7C1F12007AD
:100E80008B4022FA07FC4CEA030C05FA01F420FA25
:100E900007F3FD404FEA1C492343B5FBF9F81FFA5D
:100EA0008CFE09FB18551C0C44EA054408FB0EF5A2
:100EB000A54202FA01F200FA01F00BD91CEB04047E
:100EC00008F1FF3A80F08880A54240F28580A8F1C1
:100ED00002086444641B9DB2B4FBF9F309FB13449C
:100EE00045EA044403FB0EFEA64508D91CEB0404A6
:100EF00003F1FF356CD2A6456AD9023B644443EA4C
:100F00000843A3FB0295A4EB0E04AC42C846AE46D0
:100F100056D353D056B1B0EB080264EB0E0404FA7A
:100F200007F7CA40CC401743C6E9007418460021B1
:100F3000BDE8F087C3F1200102FA03FC20FA01F2B8
:100F400025FA01F19D402A434FEA1C471FFA8CFE07
:100F5000B1FBF7F007FB1015110C41EA054100FB4E
:100F60000EF58D4204FA03F408D91CEB010100F1DF
:100F7000FF382FD28D422DD902386144491B92B2DD
:100F8000B1FBF7F507FB151142EA014205FB0EF133
:100F9000914208D91CEB020205F1FF3816D29142AA
:100FA00014D9023D6244521A45EA004138E73146FD
:100FB000304608E73946E6E61046FBE64845A9D242
:100FC000B9EB020865EB0C0E013BA3E74546EAE7E7
:100FD0002B4694E74046D1E7D0467BE7023D62448A
:100FE00032E708460AE76444023842E7704700BF28
:100FF000054808B5054B036000F0C0FF00B908BD07
:10100000BDE8084000F09AB94C02002000300240D0
:101010000B4B02689A4200D0704782B000220192C6
:10102000D3F8302842F48052C3F8302803F5006327
:101030001B6B03F480530193019B02B0704700BF08
:101040000030024000B583B01F4B00220092186BA5
:1010500040F480001863186B00F480000090009842
:101060000192186B40F4001018631B6B03F400131B
:10107000052101930E20019B00F010FF0E2000F0CF
:1010800057FF002205210F2000F008FF0F2000F07D
:101090004FFF00220521382000F000FF382000F02B
:1010A00047FF002205213A2000F0F8FE3A2000F028
:1010B0003FFF00223B20052100F0F0FE3B2003B063
:1010C0005DF804EB00F034BF00380240044B0360CD
:1010D00010B48023034C0C605DF8044B1360704720
:1010E000580400205802002010B5094C0FCC88B0DD
:1010F0000DF1040CACE80F0094E807008CE8070041
:10110000002101A805F09CF9024B186008B010BD41
:1011100088EE01085402002030B500248DB0CDE9DE
:101120000644CDE90844414B00940A941A6B404DA3
:1011300042F010021A631A6B02F010020092009A39
:1011400001941A6B42F004021A631A6B02F0040253
:101150000192019A02941A6B42F080021A631A6B90
:1011600002F080020292029A03941A6B42F001028A
:101170001A631A6B02F001020392039A04941A6B29
:1011800042F002021A631A6B02F002020492049AFD
:1011900005941A6B42F008021A631B6B03F00803F4
:1011A0000593224628460821059B02F0BDFB4FF619
:1011B000FF72032306A91F480894CDE9062302F015
:1011C00015FA4FF6C172032306A91B480894CDE90E
:1011D000062302F00BFA49F60912032306A9174861
:1011E0000894CDE9062302F001FA4CF2DF32032322
:1011F00006A913480894CDE9062302F0F7F94FF643
:10120000F772032306A92846CDE90623089402F0C5
:10121000EDF90822012306A92846CDE90623CDE9E8
:10122000084402F0E3F90DB030BD00BF00380240C1
:10123000000C024000100240000802400000024082
:101240000004024030B5002395B0CDE90A33CDE962
:101250000C33CDE90333CDE90533214901930793DD
:10126000086C204A40F080500864096C01F08051FD
:10127000019101990293136843F48043136013684A
:1012800003F4804301204FF4803102934FF4800235
:10129000902302240425CDE90801CDE90E42CDE9D1
:1012A00010530222062308A8CDE91223029902F066
:1012B00061FB08B172B6FEE703460F22CDE9044395
:1012C00003924FF480534FF4A052294603A8CDE96E
:1012D000062302F0FDFD08B172B6FEE715B030BD81
:1012E000003802400070004008B500F07BFDFFF7B9
:1012F000A9FFFFF711FFFFF7A5FE00F005FC00F0C6
:101300000BFBFFF775FE00F01DF800F069FB00F025
:101310003DFB00F0C5FA00F03DF800F061F8FFF782
:10132000E3FE05F07FF8FEE7034B02689A4200D027
:10133000704700F071BD00BF0048014072B6FEE783
:10134000704700BF054808B5054B036002F018FF61
:1013500000B908BDBDE80840FFF7F0BFFC0400205D
:1013600000080650094B02689A4200D0704782B0CC
:10137000074B002201925A6B42F040025A635B6BAA
:1013800003F040030193019B02B070470008065030
:101390000038024010B51048104C4FF48272C0E97A
:1013A000004202210122C0E904124FF480243022BD
:1013B0000023C0E9064280210A22C0E90233C0E9C5
:1013C0000813C0E90A3202F0D3FF00B910BDBDE82E
:1013D0001040FFF7B3BF00BF8C0600200030014073
:1013E00010B51048104C4FF48272C0E9004202213F
:1013F0000122C0E904124FF4007428220023C0E93E
:10140000064280210A22C0E90233C0E90813C0E97C
:101410000A3202F0ADFF00B910BDBDE81040FFF781
:101420008DBF00BFE4060020003800402DE9F041E8
:1014300003687E4A8CB000249342CDE90644CDE98E
:10144000084405460A9405D0794A934276D00CB0F8
:10145000BDE8F081774B00945A6C7748774E42F4A0
:1014600080525A645A6C02F480520092009A01949D
:101470001A6B42F001021A631A6B02F00102019228
:10148000019A02941A6B42F002021A631B6B03F07A
:1014900002030293702202234FF00308052706A9D6
:1014A000CDE90623CDE90987029B02F09FF82022AF
:1014B00002236348CDF8248006A9CDE906230894C9
:1014C0000A9702F093F85F4A4FF0C063C6E9002321
:1014D00030464FF48063C6E90244C6E90434C6E9E5
:1014E0000644C6E9084400F06BFD002840F09580F2
:1014F000554C5649EE644FF0C0620023C4E9001217
:10150000204640214FF48062C4E90213C4E9053348
:10151000C4E90733B5632261636200F051FD00281E
:1015200078D100220521AC642320A56300F0B6FC2D
:10153000232000F0FDFC0CB0BDE8F0813D4B03948E
:101540001A6C4348434E42F480421A641A6C02F407
:1015500080420392039A04941A6B42F004021A63C5
:101560001A6B02F004020492049A05941A6B42F07A
:1015700002021A631B6B03F0020305930C2205277A
:1015800002234FF0030806A9CDE90623CDE9098718
:10159000059B02F02BF8022329480A9706A94FF46D
:1015A0008067CDE90673CDF82480089402F01EF818
:1015B000294B336030464023C6E90143C6E903475F
:1015C000C6E90544C6E90744746200F0F9FC38BB7B
:1015D000224C2349AE6400234FF480622046C4E9C4
:1015E0000013C4E90233C4E90533C4E90733B56322
:1015F0002261636200F0E4FCA8B9002205212420E6
:10160000EC64A56300F04AFC242000F091FC0CB0CF
:10161000BDE8F081FFF792FE83E7FFF78FFE67E7F3
:10162000FFF78CFED4E7FFF789FEE6E700300140C4
:101630000038004000380240000002400C05002045
:1016400000040240106402406C050020586402400F
:10165000000802402C06002070600240CC050020EB
:101660005860024082B00E4B00220092596C41F447
:1016700080415964586C00F48040009000980192B9
:10168000186C40F0805018641B6C03F08053019379
:10169000019B0F216FF0010002B000F0FFBB00BF03
:1016A0000038024070B588B000251F4B02955A6C77
:1016B0001E4C42F480225A645B6C03F4802301A91F
:1016C0000293064603A8029B02F038FD02F026FDB5
:1016D000174A226040F2E732E260164A2561430071
:1016E000A2FB03239B0C013B2046C4E90135A56105
:1016F00003F052FC054610B1284608B070BD2046E4
:1017000003F048FD05460028F6D11A2000F010FC31
:101710000F2E01D90125EFE72A4631461A2000F0A5
:10172000BDFB054B1E60E7E7003802403C07002088
:101730000048014083DE1B4308000020FEE700BF95
:10174000FEE700BFFEE700BFFEE700BFFEE700BF09
:10175000704700BF014800F0FFBD00BFCC0500206E
:10176000014800F0F9BD00BF2C06002008B5044870
:1017700004F03AF8BDE80840024804F035B800BF6C
:10178000880700203C070020014803F077BB00BF1A
:101790008C060020014803F071BB00BFE406002066
:1017A000014804F021B800BF18080020014804F0E7
:1017B0001BB800BF60080020014800F0CDBD00BF8D
:1017C0000C050020014800F0C7BD00BFA80800209C
:1017D000014800F0C1BD00BF6C050020014801F0C8
:1017E000AFBA00BF140B002001207047024B162235
:1017F0001A604FF0FF307047E81E0120014B16229F
:101800001A60FEE7E81E012070B5161E07DD0C46C3
:101810008D19AFF3008004F8010BA542F9D13046D1
:1018200070BD00BF4FF0FF30704700BF4FF4005352
:101830004B600020704700BF0120704700207047B8
:101840000D490E4A0B6810B40D4C121B83B118449D
:10185000904204D808605DF8044B18467047094B65
:101860005DF8044B0C221A604FF0FF3318467047A6
:10187000054B0B60EBE700BF84070020000002204F
:1018800000100000E81E0120F01E0120034AD2F8DB
:10189000883043F47003C2F88830704700ED00E0F0
:1018A00000B51B481B4A02608F22002387B04260AC
:1018B00042F20F72CDE90233CDE90433CDE90033B2
:1018C000C0E90232C0E90433836103F065FB98B9D3
:1018D0004FF480530E48029302A903F0D7FC98B945
:1018E000002200230A486946CDE9002304F026F8C7
:1018F00028B907B05DF804FBFFF720FDE8E7FFF724
:101900001DFD07B05DF804FBFFF718FDE8E700BF19
:10191000880700200000014000B51A481A4A0260FA
:101920004722002387B0426042F20F72CDE90233B2
:10193000CDE90433CDE90033C0E9023203618361AC
:1019400003F02AFB98B94FF480530E48029302A982
:1019500003F09CFC98B9002200230A486946CDE9AF
:10196000002303F0EBFF28B907B05DF804FBFFF795
:10197000E5FCE8E7FFF7E2FC07B05DF804FBFFF7E2
:10198000DDFCE8E7D00700200004004000B5124865
:1019900012494722002383B0C0E900124FF6FF72BC
:1019A000CDE90033C0E90232836103F0F5FA58B99A
:1019B0000022002308486946CDE9002303F0BEFF5A
:1019C00028B903B05DF804FBFFF7B8FCF0E7FFF7B8
:1019D000B5FC03B05DF804FB1808002000100040BF
:1019E00000B5124812495122002383B0C0E9001209
:1019F0004FF6FF72CDE90033C0E90232836103F094
:101A0000CBFA58B90022002308486946CDE90023E3
:101A100003F094FF28B903B05DF804FBFFF78EFCD8
:101A2000F0E7FFF78BFC03B05DF804FB60080020D3
:101A30000014004000B52F4A0368934285B030D0AF
:101A40002D4A934208D02D4A934214D02C4A9342F7
:101A50003DD005B05DF804FB2A4B002201921A6CC0
:101A600042F002021A641B6C03F002030193019B13
:101A700005B05DF804FB234B00220292196C41F083
:101A8000100119641B6C03F010033620029305212A
:101A9000029B00F003FA362005B05DF804EB00F07D
:101AA00047BA184B00220092596C41F00101596469
:101AB0005B6C03F0010300931A200F21009B00F0E0
:101AC000EDF91A2005B05DF804EB00F031BA0D4BCA
:101AD00000220392196C41F0200119641B6C03F081
:101AE0002003372003930521039B00F0D7F937200B
:101AF000D2E700BF00000140000400400010004099
:101B0000001400400038024010B50B480B4C002375
:101B10004FF461210C22C0E90041C0E90233C0E961
:101B20000432C0E9063304F03BF800B910BDBDE84B
:101B30001040FFF703BC00BF08090020001001405F
:101B400070B5264B026888B000249A42CDE9024461
:101B5000CDE90444069401D008B070BD03F5943378
:101B600000945A6C1E4E42F010025A645A6C02F0F5
:101B700010020092009A01941A6B42F001021A635B
:101B80001B6B03F0010301934FF4C0620223CDE904
:101B90000223032305930546019B1248072302A94C
:101BA000069301F023FD104A4FF00063C6E90023BD
:101BB00030464FF48063C6E90244C6E90434C6E9FE
:101BC0000644C6E9084400F0FBF918B9AE63B563F2
:101BD00008B070BDFFF7B2FBF8E700BF001001408E
:101BE000A80800200000024040640240DFF834D022
:101BF0000D480E490E4A002302E0D458C450043365
:101C0000C4188C42F9D30B4A0B4C002301E013603B
:101C10000432A242FBD3FFF739FE19F0BDFEFFF7F5
:101C200063FB704700000220000000202C0200200F
:101C30006C30020830020020F01E0120FEE7000098
:101C400080B1CB6873B18A6862B130B40C6964B199
:101C5000D1E90051C0E90423C0E9025184610020A8
:101C600030BC70474FF0FF3070474FF0FF30F7E760
:101C700070B5446882B0002305460193002C47D11B
:101C8000836803B1984720232B60002607E0019B5F
:101C900003F01F03A34216D00134202C0BD06B6934
:101CA000204601AA122198470028F0DA0134202C9E
:101CB0006FF00406F3D12C681F2C38D96FF00206A0
:101CC000304602B070BD2C602B694FF400422046B4
:101CD0000021984700282DDB6B69286801AA0021A4
:101CE000984700282CDBAB69984704460DE0AB69A8
:101CF0009847001BB0F5FA7F01AA4FF000011CD8ED
:101D00006B692868984700281ADB019B1B04EED4F6
:101D1000AB6998470446AB699847031BB3F5FA6F64
:101D2000F9D901236B600026304602B070BD002E49
:101D3000FAD1C9E76FF00306F6E76FF00106F3E7A3
:101D40006FF00406F0E700BF30B583B000254369AB
:101D50000195044601AA006801219847A8423DDB8D
:101D60006369206801AA01219847002836DB019B9E
:101D70005B072AD56369206801AA2946984700288D
:101D80002CDB019BDD0414D56369206801AA1F21A7
:101D90009847002822DB019BDA041DD503F01C03C1
:101DA000182B17D0082B13D0142B0BD1042003B001
:101DB00030BD03F40452B2F5045F0BD0980407D48D
:101DC000D905F3D4052003B030BD012003B030BDE8
:101DD0000320F8E70220F6E70620F4E76FF004009E
:101DE000F1E700BF08B50B4B1A6842F400721A60A5
:101DF0001A6842F480621A601A6842F480721A60AB
:101E0000032000F02DF80F20FFF74CFCFFF72AFC11
:101E1000002008BD003C0240034A044B11681B78B7
:101E20000B441360704700BF4C09002004000020E1
:101E3000014B1868704700BF4C09002038B50446B4
:101E4000FFF7F6FF631C054602D0044B1B781C44C9
:101E5000FFF7EEFF431BA342FAD338BD0400002076
:101E6000C31E042B10B504460ED80A49CA682302C3
:101E70004FF6FF0003F4E0630240134343F0BF63F7
:101E800043F40033CB6010BD03489021FFF758FAAC
:101E9000EBE700BF00ED00E018F001080F2A70B575
:101EA000164605460C4637D80F2C30D81D4BDB683C
:101EB000C3F30223C3F10701042903F1040228BF7D
:101EC0000421062A18D9033B4FF0FF329A4026EA34
:101ED00002064FF0FF328A4024EA02049C40002DA3
:101EE00044EA06020BDB05F16045120105F5614588
:101EF000D2B285F8002370BD00263346E9E70A4BCD
:101F000005F00F0512012B44D2B21A7670BD0748B6
:101F1000A921FFF715FAC9E70448A821FFF710FA2D
:101F2000C2E700BF00ED00E0FCEC00E018F00108A3
:101F3000002808DB4109064A00F01F000123834006
:101F400042F8213070470348BC21FFF7F9B900BFC0
:101F500000E100E018F00108BFF34F8F0549064B80
:101F6000CA6802F4E0621343CB60BFF34F8F00BF37
:101F7000FDE700BF00ED00E00400FA05C8B10E4B1C
:101F800002689A4210B5044603D00C486821FFF756
:101F9000D7F9637903F0FF021BB1012363710020BD
:101FA00010BD20462271FFF733F801236371002032
:101FB00010BD0120704700BF0030024054F00108FE
:101FC00038B50446FFF734FF002C00F01281236877
:101FD000A74A9342054631D0183293422ED0183288
:101FE00093422BD01832934228D01832934225D0F6
:101FF0001832934222D0183293421FD018329342A3
:102000001CD002F55672934218D01832934215D064
:102010001832934212D0183293420FD018329342A2
:102020000CD01832934209D01832934206D018329D
:10203000934203D08F48B721FFF782F9636833F0EA
:10204000C06306D0B3F1006F03D08A48B821FFF710
:1020500077F9A36833F0400240F09680E36833F4E8
:10206000007340F09D80236933F4806340F0A180C9
:10207000636933F4006203D0B3F5805F40F0A5805C
:10208000A36933F4005203D0B3F5804F40F0A7802A
:10209000E36933F0200206D0B3F5807F03D07548A2
:1020A000BE21FFF74DF9236A33F4403303D0714862
:1020B000BF21FFF745F9636ADBB1042B05D06D48FA
:1020C000C021FFF73DF9636A9BB1A36A032B00F2BD
:1020D000B180E36A33F0C07303D06648C621FFF7CE
:1020E0002FF9236B33F4C00303D06248C721FFF7F5
:1020F00027F923680022022184F8351084F834205F
:102100001A6822F001021A6005E0FFF791FE401BF9
:10211000052853D823681A68D107F6D4D4E90120DA
:10212000E16802430A43D4E90451A0692A430A43FF
:10213000E1691D6802430A434F492940256A2A4341
:102140000A43616A042956D01A605A6922F00702CC
:102150001143D8B2494A59611038A2FB0052120902
:10216000474923F47F73895CE16523F003035F280B
:1021700088BF04333F228A40A36500209A60012370
:10218000606584F8353038BD802B3FF467AF39483F
:10219000B921FFF7D5F8E36833F400733FF463AF78
:1021A0003448BA21FFF7CCF8236933F480633FF455
:1021B0005FAF3048BB21FFF7C3F859E70323202264
:1021C000626584F83530184638BD2A48BC21FFF7CF
:1021D000B7F8A36933F400523FF45AAF54E72548E7
:1021E000BD21FFF7ADF8E36933F020023FF45BAFA8
:1021F00052E7012038BDD4E90B512943114319603E
:102200005969A26A21F00701114341F00401002D30
:102210009FD0A0B1B0F5005F1BD0022A03D9032ADA
:1022200097D1EA0195D501234022626584F83530C3
:10223000184638BD0F48C521FFF782F849E7012A43
:1022400003D032F0020284D1EBE7B5F1C07F80D138
:10225000E9E7032A3FF67DAF01A050F822F000BF66
:102260002722000823220008272200084B2200080A
:10227000106002408CF001083F8010F0ABAAAAAABF
:10228000C4F001082DE9F843D0F8588004461E46F2
:10229000581E4FF6FE739842894617463CD894F86C
:1022A0003430012B41D094F835300122934284F828
:1022B000342005D0002384F834300220BDE8F883B0
:1022C000022384F835302568E26D002363652B68AE
:1022D00023F480232B60A3686E60402B4FF03F03F4
:1022E00003FA02F30BBFAF60C5F80890C5F80C9075
:1022F000EF60C8F808302B68226C43F016032B609F
:102300001AB12B6843F008032B602B6843F00103DC
:1023100000202B60BDE8F883054840F2CB11FFF7A1
:102320000FF894F83430012BBDD10220BDE8F883BA
:102330008CF0010890F83530022B03D080234365E0
:10234000012070470268052380F83530136823F0B8
:102350000103002013607047F0B583B0674A876DB2
:10236000166800230193C36D3D6808229A402A42F3
:10237000044603D001680868400778D401229A40D7
:102380002A4203D02168496908066AD404229A4087
:102390002A4203D02168096889075CD410229A4038
:1023A0002A4203D021680868000741D420229A40BD
:1023B0002A4214D021680868C00610D5BA6094F883
:1023C0003520052A63D00B6813F4802F0B687ED06C
:1023D000190340F18980E36B0BB120469847636D88
:1023E00023B3636DDA071AD522684549052384F8BB
:1023F00035301368A1FB061623F00103B60A1360FB
:1024000002E01368DB0704D5019B0133B34201935B
:10241000F7D90122002384F8352084F83430E36CA6
:1024200023B1204603B0BDE8F040184703B0F0BD2B
:10243000BA600A6812F4802F0A6822D1D20503D448
:102440000A6822F008020A60226C002AAED02046F8
:102450009047E36DAAE7BA60626D42F004026265DC
:102460009CE7BA60626D42F0020262658EE708681E
:1024700020F004000860BA60626D42F001026265FB
:102480007CE71103E0D5A26C002AE0D18EE70A6850
:1024900022F016020A604A6922F080024A61226C28
:1024A0003AB30A6822F008020A603F2202FA03F3F4
:1024B000216DBB600122002384F8352084F834307C
:1024C0000029B3D0204603B0BDE8F040084713F41C
:1024D000807380D10A6822F010020A60012284F819
:1024E000352084F8343076E7636C002B7FF475AFC9
:1024F00075E7A26C002AD4D1D7E700BF0000002006
:10250000B5814E1B2DE9F041866A8F6800EB860C81
:10251000DCF818301C68002CC0F28B80DCF82C40F2
:10252000002C40F086803C689C605C687D6824F4E8
:10253000FF5424F01F042C430D685C60EC0706D5A3
:102540001C6824F4400E4C694EEA04041C60AC067E
:1025500005D50C69196821F04061214319606907AC
:1025600003D5196841F080011960196841F0805164
:102570001960BFF35F8F1C68B96844F000441C60A9
:10258000002900F08C80DFF854813446002A6AD19B
:10259000012217E0DEF82C507DBB0D689D605D6860
:1025A0004F6805EA08053D435D60BFF35F8F1D6816
:1025B000896845F0004502F1010E1D60002900F018
:1025C000878072461D6804F1010E25F000551D60DC
:1025D000BEF1030F1D68A4F1030498BF744600EB1D
:1025E000840E25F080451D60DEF818301D6825F04A
:1025F00080551D601D68002DCCDADCF818400025E0
:10260000BAB1BFF35F8F2168731C21F00041032B27
:1026100000EB8307216008D9F31E00EB830101352D
:10262000AA428C6905D01E46EBE70135AA42BC6977
:10263000F9D10220BDE8F081DEF82C50002DDCD16C
:102640000D689D605D684F6805EA08053D435D6063
:10265000BFF35F8F1D68896845F0004502F1010EE8
:102660001D60F9B172461D6804F1010E25F0005598
:102670001D60BEF1030F1D68A4F1030498BF7446EA
:1026800000EB840E45F080451D60DEF818301D68B3
:1026900025F080551D601D68002DCDDAADE734466C
:1026A000B2B10A46196841F080411960196841F0D9
:1026B0000051196000EB8403C16BD962846272B669
:1026C000036C01331344036462B60020BDE8F0815B
:1026D000196821F080411960E8E700BF00E0FFFFC2
:1026E0002DE9F043D0E91A5683B005F11203002218
:1026F00050F8234001923EB3DFF8809007464FF434
:102700008C48236A5BB3BB6D002B33D1C4F80490B3
:10271000BFF35F8F23686A1C43F00043032A05F16F
:102720001301236013D9033D05F11203013E57F84D
:102730002340E6D1FB6EB34206D03B6803F58053DD
:1027400000229A60C7E91A5603B0BDE8F083013E43
:1027500057F821401546EDD0236A002BD3D101A8AC
:1027600003F01EFE019B002BE4D0A3602362BB6D2F
:10277000002BCBD0C4F80480CAE700BF004600801D
:10278000002800F01981F0B5D0F8843083B00546F8
:10279000002B00F00B81894AA86800230193516C3B
:1027A000874B41F480415164526C02F480420192A3
:1027B000019A5A6822F400025A6059682A68014353
:1027C00002F5805259605B68136843F0010313609F
:1027D000FFF72EFB064606E0FFF72AFB831BB3F547
:1027E000FA7F00F2DA802B6803F58052146814F047
:1027F0000104F1D11968734A0A4042F49C421A60FC
:1028000001201E68FFF71AFB2A68166093694FF6CD
:1028100041710B4043F08003936101209669FFF7FB
:102820000DFB2B6803F580529E619169664B0B404E
:1028300043F0087343F00403936101209669FFF7A6
:10284000FDFA2B68614A03F5805301209E611A60EE
:102850001E68FFF7F3FA2968EA6801F5805113460C
:102860000E60146054609460D4601068AA6140F4F3
:10287000801043F8280BD360106840F440001060CB
:102880009462D46214635463EB61936A02F1500062
:1028900043F4801393625063936A43F4400393625A
:1028A000146554659465D465136D286243F48013F0
:1028B00002F178001365D065136D43F4400313658E
:1028C0009467D467C2F88040C2F88440936F68620E
:1028D00043F480139367C2F88420936F43F440035A
:1028E00093672B69AC624FF000400A614FF48C4251
:1028F0001C605C609C60DC6018605A605E6803F17C
:10290000280726F000465E60C3E90844AB64DF6038
:10291000C3E912449C62DC621C635C639862DA6205
:10292000DE6A26F00046DE62EF6403F150075F6363
:102930001C655C659C65DC6518655A655E6D26F0F6
:1029400000465E6503F17806C3E91C442F65DE6529
:102950009C67DC67C3F88040C3F884409867DA67F7
:10296000DA6F22F00042DA67C3E926446E65C3F8E5
:102970008430C5E91744C5E91A44AC656A68CB6080
:10298000134B918819641168596410222046C5F8C8
:102990008840C5F8842003B0F0BD0422E023012064
:1029A000C5F88820C5F8843003B0F0BD2323C0F8F3
:1029B000843003F00BFCEEE6012070470038024043
:1029C000003801400F8120FF233FDEF88020C10244
:1029D00000800240D0F88430102B01D001207047D5
:1029E000F0B503682326C0F88460DA6B012542F451
:1029F00002728565DA63D3F80C2142F4003242F0AA
:102A00006002C3F80C21D3F8102142F403120446EB
:102A1000C3F81021042383B0C366FFF761FE236867
:102A20001A6842F008021A6028461F68FFF706FA83
:102A300023681F601A6842F004021A6028461F6863
:102A4000FFF7FCF9236828461F60002503F5805333
:102A500001959A6942F480129A619B690193FFF78C
:102A6000EDF92368019A03F5805328469A619A6923
:102A700042F400529A619A6942F002029A61DA695C
:102A800042F4D03242F0C102DA61C4F8846003B08B
:102A9000F0BD00BFD0F88430232B01D00120704757
:102AA000016870B5C0F8843001F580530446DA69D6
:102AB00022F4D03222F0C102DA619A6922F4005283
:102AC0009A619A6922F002029A610B6823F004036A
:102AD00082B00B6001200E68FFF7B0F92368002573
:102AE0001E6003F5805301959A6942F480129A6141
:102AF0009B6901930120FFF7A1F92368019903F570
:102B00008052012091611A6822F008021A601E6842
:102B1000FFF794F92368A16C1E604B68E26C43F0E8
:102B200000434B605368216D43F0004353604B6892
:102B3000626D43F000434B605368102143F0004343
:102B400028465360A565C4F8841002B070BD00BF6C
:102B500010B5044651B3D0F88420232A01D00120B7
:102B600010BD4B6BC3630122FFF7CCFCB0B9BFF3C0
:102B70004F8FA36A5A1C032A84BF033BA3622368B6
:102B800098BFA26203F58053586910F00400E7D0A3
:102B900000220421596110465A6010BDD4F88830D3
:102BA00043F002030120C4F8883010BDD0F888300B
:102BB00001200343C4F8883010BD00BF2DE9F04F59
:102BC00085B00546039100296AD0D0F88430232BC4
:102BD0005ED1D0F85C8008F1120350F82340C36E38
:102BE0002268002AC3F1040B73DBBBF1000F72D023
:102BF0004FF0000900F18001CA467C3003E0CB456C
:102C00003FD0002E55D12368DE0503D5A369AB67FD
:102C1000E3696B6723689A0501D4EE6F0EB32368EE
:102C200026686F699B0548BFC5E918AA16F4807627
:102C300006D0276823682B67C7F30D47043F01269A
:102C4000A2682262BBB2CDE9010103F0CDFB2B6E7D
:102C500001332B666B6EDDE901013B446B66C4F802
:102C600020A008F10103032B8CBFA8F103089846AC
:102C700008F1120309F1010955F823402368002BDC
:102C8000BDDAEB6E4B44EB6633B9C5F85C80CEB968
:102C9000012005B0BDE8F08F2846FFF721FDF4E7DD
:102CA000D0F8883001200343C5F8883005B0BDE86E
:102CB000F08FEB6E4B44EB6613B12846FFF710FD27
:102CC000C5F85C800399EA6F0A6000231846EB6739
:102CD000DFE7002BDCD0FFF703FDC5F85C80D7E70A
:102CE0002DE9F041D0E9105475B10646002706EBF6
:102CF0008408A300D8F82C002344013D38B1F268C1
:102D000052F83330002B0ADA0020BDE8F08101349C
:102D100004F00304002DEAD10020BDE8F081013465
:102D200004F0030403F07CFBC8F82C70C6E91054CF
:102D3000002DDCD1F0E700BF704700BF704700BF37
:102D4000026802F5805310B559694906044602D558
:102D5000D969490648D45969C90702D5D969C8074C
:102D600038D45969090402D5D96908040ED4936B83
:102D7000190723D4264B5A69120300D410BD4FF40F
:102D800000225A612046FFF7D9FF10BDD4F88820F1
:102D900042F00802C4F888205A6912F4005F5A69A8
:102DA0002AD148F280610A40C4F88C20596120463B
:102DB00003F014F92268936B1907DBD5D36A03F08B
:102DC0006003C4F894302046FFF7B6FF0023C4F830
:102DD0009430CFE74FF001125A61204603F0F8F823
:102DE000226802F58053BCE70A4A5A6103F0EAF808
:102DF000226802F58053AEE707480240C4F88C20F1
:102E0000DA69E02122F4C032DA61C4F88410CEE736
:102E1000003C01404000010000207E0070B50446E7
:102E200000681D460369920103F01C0302F4F86276
:102E3000C9021A4389B2114341F001010161FEF751
:102E4000F7FF064604E021680A6912F0010207D084
:102E5000FEF7EEFF821BB2F5803FF4D3012070BD78
:102E60004B699BB210462B6070BD00BF38B504465D
:102E7000006805699BB29201436102F4F86205F0B3
:102E80001C03C9021A4389B2114341F003010161D5
:102E9000FEF7CEFF054604E023681B6913F001032B
:102EA00007D0FEF7C5FF431BB3F5803FF4D30120E5
:102EB00038BD184638BD00BF002960D003681A68C5
:102EC000C2F3001281F8282010B41C681A6882F43A
:102ED0000072C2F3402281F820201A68C2F3004237
:102EE000CA771A6882F40052C2F340328A771A68AD
:102EF000C2F300320A7704F060044C621C681A685E
:102F000004F4006402F48042C1E905241A6882F4E2
:102F10008002C2F380524A741A6882F40002C2F33B
:102F2000C0520A741A68C2F3C012CA731C681A68C5
:102F3000C2F380220A719A69C2F3400281F85420D8
:102F40009A6982F08002C2F3C01204F4602481F80E
:102F50004C208C609A6902F030020A659A699C697B
:102F6000C4F3800C81F856C09B695DF8044B120CC9
:102F7000C3F3C00300208A6481F8553070470120F4
:102F8000704700BF39B1F8B5D0F88430102B044633
:102F900003D00120F8BD012070470268374B10684C
:102FA0000340886803434869034388690343486AC8
:102FB0000343C87F43EA0043087F43EA00330879AC
:102FC00043EA8023C87B43EAC01391F8280043EA10
:102FD0000013087CB0FA80F0400943EAC053487CF3
:102FE000B0FA80F0400943EA8053887FB0FA80F05D
:102FF000400943EA403391F82000B0FA80F04009DC
:1030000043EA4023136001200F461668FEF716FFBF
:1030100025682E60AB6997F856004FF64172134051
:103020003A6D1343BA6C43EA024397F84C20B2FA64
:1030300082F2520943EAC21397F85520A2F1010225
:10304000B2FA82F2520943EAC20397F85420A0F17F
:103050000101B1FA81F1A2F101024909B2FA82F249
:1030600043EA8103520943EA4203AB610120AD699F
:10307000FEF7E4FE236800209D61F8BD0F8120FF6C
:1030800038B5036805461C6901F032F8134B144A41
:103090000344934224F01C0404D244F008042B6837
:1030A0001C6138BD0F4B104A0344934204D82B686F
:1030B00044F00C041C6138BD0C4B0D4A0344934290
:1030C000EDD30C4B0C4A034493422B6894BF44F05D
:1030D000040444F010041C6138BD00BF00D3CEFED0
:1030E000C0E1E40040F1E9FD3F787D0100796CFC2E
:1030F000005A6202001F0AFA7FF0FA02D0F88C0030
:10310000704700BF1B4BDA68D10605D51A49CA695A
:1031100010200243CA61D860164BDA68920606D5C1
:103120001549CA69202042F00802CA61D860114BD3
:10313000DA68500606D51049CA69402042F00402F8
:10314000CA61D8600B4BDA68110606D50A49CA690C
:10315000802042F00202CA61D860064BDA6892070A
:1031600006D50549CA69022042F02002CA61D8602A
:10317000704700BF003C0240500900202DE9F84F85
:10318000784F9B463B7E012B00F0B880012303283B
:103190008046894692463B766AD80023FB61FEF75B
:1031A00047FE714D04464CF2503604E0FEF740FEF7
:1031B000001BB04257D8EB68D803F7D4EB68D907A7
:1031C00044BF0123EB60684BDB6813F0F20F54D16E
:1031D000B8F1000F76D0B8F1010F09F1784300F093
:1031E0009080B8F1020F4CD0B3F5801F07D309F1DE
:1031F000604303F50843B3F5047F80F0AD805A4B7C
:103200001A6922F440721A611A6942F440721A6112
:103210001A6942F001021A61C9F800A0BFF36F8F6A
:10322000C9F804B00023FB61FEF702FE4E4D0446D0
:103230004CF2503604E0FEF7FBFD001BB0423FD8D5
:10324000EB68DA03F7D4EB68DB0744BF0123EB60DC
:10325000454BD86810F0F20074D1434A136923F04B
:103260000103136100E0032000233B76BDE8F88FE3
:103270003E48A221FEF764F88FE7FFF743FF0120E5
:10328000F2E7B3F5801F0BD309F1604303F5084360
:10329000B3F5047F04D3354840F28721FEF750F898
:1032A000314B1A6922F440721A611A6942F40072B1
:1032B0001A611A6942F001021A61C9F800A0B1E767
:1032C0000320CAE709F17843B3F5801F5FFA8AFA51
:1032D00006D309F1604303F50843B3F5047F35D203
:1032E000214B1A6922F440721A611A691A611A692B
:1032F00042F001021A6189F800A093E70220BDE8BC
:10330000F88FB3F5801F1FFA8AFA0BD309F16043D7
:1033100003F50843B3F5047F04D314484FF4287130
:10332000FEF70EF8104B1A6922F440721A611A69FE
:1033300042F480721A611A6942F001021A61A9F816
:1033400000A06FE7FFF7DEFE012086E7074840F2A6
:10335000B921FDF7F5FFC3E7044840F26521FDF709
:10336000EFFF4CE750090020003C0240CCF0010880
:10337000064B1A69002A01DB002070470449054A00
:1033800059605A601869C00F704700BF003C024086
:1033900023016745AB89EFCD034A136943F000432E
:1033A00000201361704700BF003C0240144B70B511
:1033B00000220446DA61FEF73BFD124E0546631C0F
:1033C0000FD1104AD368D803FCD40E4BDA68D20769
:1033D00044BF0122DA600B4BD86810F0F2000BD129
:1033E00070BDF368D903F0D524B1FEF721FD401B71
:1033F000A042E4D9032070BDFFF784FE012070BD18
:1034000050090020003C0240144B1A6891050FD56A
:103410001A6822F400721A601A6842F400621A6094
:103420001A6822F400621A601A6842F400721A6084
:103430000A4B1A6852050FD51A6822F480621A6086
:103440001A6842F480521A601A6822F480521A6094
:103450001A6842F480621A60704700BF003C024064
:103460002DE9F84F5E4E337E012B7DD0012333765C
:103470000368012B82460F4603D95A48A921FDF75C
:103480005FFF4CF25030FFF791FF0546002858D1FE
:103490004FF0FF333B60DAF80030012B70D0DAE9EF
:1034A00002934B445A1E0B2A62D8994547D2DFF843
:1034B00034814D4C2BE0BBF1030F35D8BBF1000F2D
:1034C00044D1236923F440732361236943EA0B0346
:1034D0002361236923F0F8032361236943EAC903C5
:1034E00043F002032361236943F4803323614CF2E8
:1034F0005030FFF75BFF236923F0FA032361D8B94B
:10350000DAE9022309F1010913444B4517D9B9F14E
:103510000B0F9AF810B0CED940F2D9314046FDF7E2
:103520000FFFBBF1030FC9D940F2DA314046FDF776
:1035300007FF4FF4407BC4E7C7F800900546FFF74C
:1035400063FF002333762846BDE8F88FBBF1010FF7
:1035500002D14FF4807BB4E7BBF1020F0CBF4FF4F4
:10356000007B4FF4407BACE702252846BDE8F88F8E
:103570001C48C121FDF7E4FEDAE902934B4494E7CD
:10358000DAF81040DAF80450E3B2032B21D8012D09
:1035900019D1154F3A6922F440723A613A6942F002
:1035A00004023A613A6923029BB2134343F4803325
:1035B0003B614CF25030FFF7F9FE3B6923F0040306
:1035C00005463B61BBE7074840F2BB31FDF7B8FE5B
:1035D000DFE7044840F2BA31FDF7B2FED7E700BF9B
:1035E0005009002008F10108003C02402DE9F04F8D
:1035F000B74B984283B00746884623D003F58063D3
:1036000098421FD003F5806398421BD003F5806376
:10361000984217D003F58063984213D003F5806376
:1036200098420FD003F5806398420BD003F5806376
:10363000984207D003F58063984203D0A548AC2197
:10364000FDF77EFED8F800309AB2002A00F0D18053
:103650001B0C1B04002B40F0CC80D8F80430012B4D
:103660000DD9B3F5041F0AD000F2E280B3F5881F2C
:1036700005D040F2D180B3F5901F40F0D4800026F1
:10368000DFF874A2354605E00135102D06F102067B
:1036900000F0AC80D8F800300124AC4004EA030903
:1036A00034EA0303F0D1D8F8042002F00303591ED2
:1036B000012940F2CC804FF0030B0BFA06FB6FEAB6
:1036C0000B0B032B23D0D8F80810022900F2D88066
:1036D000F868B14000EA0B000143022BF96016D1F3
:1036E000D8F8100010B10D2800F28880EC0807EB24
:1036F000840405F00701D4F820C089004FF00F0EB4
:1037000088400EFA01F12CEA010108432062396871
:10371000B34001EA0B010B4312F4403F3B60B3D0CE
:103720006D4B00210191596C41F4804159645B6CEF
:1037300003F48043019325F0030303F1804303F571
:103740009C3305F0030401999968A4000F20A04060
:1037500021EA00015E4887421DD0574500F0A48051
:103760005E48874200F0A4805D48874200F0A48054
:103770005C48874200F0A4805B48874200F0A48048
:103780005A48874200F0BA80594887420CBF072048
:103790000820A04001439960564B9B68D0026FEA15
:1037A0000901544854BF0B4049EA03038360C368CE
:1037B0005048940254BF0B4049EA0303C360436876
:1037C00090034C4854BF0B4049EA0303436003682D
:1037D000D20305F10105474A54BF0B4049EA0303F0
:1037E000102D136006F102067FF454AF03B0BDE85C
:1037F000F08F3848AD21FDF7A3FD2EE70F283FF4E9
:1038000075AF3448DE21FDF79BFDD8F80420D8F8C9
:10381000100002F0030369E7032B7FF630AF113B82
:10382000012B7FF62CAF2B48AE21FDF789FD26E753
:10383000B3F5441F3FF423AF23F48013B3F5081FFF
:103840003FF41DAF2348AE21FDF77AFD17E7D8F806
:103850000C1003291DD8B8684FF0030B0BFA06FBB8
:1038600020EA0B00B1400143B9607868C2F300114F
:1038700020EA0400A94001436FEA0B0B796020E7BE
:10388000D1211448FDF75CFDD8E9012102F00303C2
:103890001EE7C0210F48FDF753FDD8F80420D8F8E3
:1038A0000C1002F00303D6E70120A040014372E7A9
:1038B0000220A04001436EE70320A04001436AE7D5
:1038C0000420A040014366E70520A040014362E7D1
:1038D0000000024048F101080038024000080240A0
:1038E000000C024000100240001402400018024088
:1038F000001C0240003C0140000402400620A040A1
:10390000014348E738B505460C4629B12B691C42EE
:1039100014BF0120002038BD02484FF4BE71FDF7EE
:103920000FFDF3E748F1010870B5064615460C4651
:1039300061B1012D03D805B92404B46170BD0648F6
:103940004FF4CF71FDF7FCFCB46170BD024840F24A
:103950009D11FDF7F5FCECE748F10108044A5169B7
:10396000014200D1704708B5506115F0B5FE08BDA1
:10397000003C0140002800F065822DE9F041036819
:103980000F2B82B0044600F23D81DD0737D5636816
:1039900033F4803203D0B3F5A02F40F0A781A44ABE
:1039A000936803F00C03042B00F08381936803F009
:1039B0000C03082B00F079816368B3F5803F00F0B9
:1039C0008281B3F5A02F00F00A82994D2A6822F473
:1039D00080322A602A6822F480222A60002B40F07C
:1039E0007781FEF725FA064605E0FEF721FA801BEF
:1039F000642800F29D812B689B03F6D423689F07FF
:103A000030D5E368012B00F21B8123691F2B00F2E4
:103A10002081874B9A6812F00C0F00F0FD809A68A5
:103A200002F00C02082A00F0F380E368002B00F09B
:103A30009B81804B7E4E01221A60FEF7F9F9054604
:103A400005E0FEF7F5F9401B022800F271813368AA
:103A50009807F6D53368226923F0F80343EAC203D6
:103A6000336023681A0700F1B4805D0744D5A3686A
:103A7000012B06D9052B04D06F484FF4C571FDF713
:103A80005FFC6B4A136C13F0805340F0028101938A
:103A9000136C43F080531364136C03F08053019351
:103AA000019B0125654E3368D80540F13181A3683B
:103AB000012B00F04181052B00F0C6815C4E326F76
:103AC00022F001023267326F22F004023267002BCB
:103AD00040F03781FEF7ACF941F28838074605E03F
:103AE000FEF7A6F9C01B404500F22281336F9B0709
:103AF000F6D4002D40F07D81A069022800F2CB8031
:103B0000002862D04A4DAB6803F00C03082B00F08C
:103B10003C81022840F08581E36933F4800304D0BE
:103B200045484FF4EB71FDF70BFC236A3F2B00F285
:103B30007281636A323BB3F5BF7F00F26681A36A8C
:103B4000022B0CD0082B05D84FF4A87222FA03F3ED
:103B5000D80704D4384840F2D911FDF7F1FBE36AE5
:103B6000023B0D2B00F24B81324B314E00221A6684
:103B7000FEF75EF9054605E0FEF75AF9401B0228FC
:103B800000F2D68033689901F6D4D4E90731626A2D
:103B9000274D0B4343EA8213D4E90A21520843EA32
:103BA0000163013A234943EA0243012273600A6632
:103BB000FEF73EF9044605E0FEF73AF9001B02283D
:103BC00000F2B6802B689A01F6D5002002B0BDE85D
:103BD000F0816369012B53D8002B40D0154B144E54
:103BE0000122C3F8802EFEF723F9054605E0FEF713
:103BF0001FF9401B022800F29B80736F9B07F6D5CC
:103C0000236832E70C48E621FDF79AFB2368BCE6FF
:103C10005B685E023FF509AF054B1B689D076AD5DF
:103C2000E368012B67D0012002B0BDE8F08100BF3E
:103C3000003802400000474284F101080070004053
:103C4000864840F21D11FDF77BFB23691F2B7FF691
:103C5000E0AE82484FF48F71FDF772FBD9E6804ADF
:103C6000804EC2F8803EFEF7E3F8054604E0FEF71A
:103C7000DFF8401B02285BD8736F9F07F7D4BFE7BC
:103C800076484FF4AF71FDF75BFB6369002BE6D01C
:103C9000A4E7002506E7714840F2CD11FDF750FB7F
:103CA000A06900287FF42EAF8FE7536858027FF594
:103CB00083AE6C4B1B6899037FF5A0AE6368002B45
:103CC0007FF49CAEAFE7674A136843F48033136018
:103CD000FEF7AEF8634E054604E0FEF7A9F8401B78
:103CE000642825D833689A03F7D587E65B48EB212B
:103CF000FDF726FB53E65B4A2169136823F0F803BE
:103D000043EAC103136023681A077FF5AEAE60E78C
:103D1000336843F480733360FEF78AF807463368EC
:103D2000D9053FF5C4AEFEF783F8C01B0228F6D9CB
:103D3000032002B0BDE8F0814A4A136F43F001034B
:103D40001367FEF775F8474F064641F2883804E0DE
:103D5000FEF76EF8801B4045EAD83B6F9A07F7D50F
:103D6000002D3FF4C9AE44E03D4A3E4E1360FEF7DD
:103D70005FF8054604E0FEF75BF8401B0228D7D841
:103D800033689907F7D423686CE601283FF41EAF27
:103D90006B68E26903F4800191427FF444AF226AC8
:103DA00003F03F0191427FF43EAF616A47F6C07273
:103DB0001A40B2EB811F7FF436AFA26A520803F4B7
:103DC0004031013AB1EB024F7FF42DAFE26A03F0CC
:103DD0007063B3EB026F14BF01200020F6E6214BA5
:103DE0001A6842F480221A601A6842F480321A601B
:103DF0006EE71C4A136C23F0805313647CE617486B
:103E00004FF4ED71FDF79CFAAEE614484FF4EC71F7
:103E1000FDF796FA93E6114840F2D711FDF790FAB4
:103E200087E60F4B00221A66FEF702F8044605E00B
:103E3000FDF7FEFF001B02283FF67AAF2B689B01BF
:103E4000F6D4C2E601207047064B1A6F42F0040216
:103E50001A671A6F42F001021A6772E784F10108CB
:103E60000000474200380240164908B58B6803F04D
:103E70000C03042B1BD0082B17D14A684B684968E8
:103E800013F4800302F03F0213D10F48C1F38811ED
:103E9000A1FB0001FCF7F8FE0A4B5B68C3F301438A
:103EA00001335B00B0FBF3F008BD074808BD0748CD
:103EB00008BD0648C1F388110023A1FB0001FCF7EF
:103EC000E3FEE9E7003802400024F40000127A0023
:103ED000002800F0FE800368013B0E2B2DE9F04125
:103EE0000D46044600F2CF80072D00F2C1807A4AC9
:103EF000136803F00703AB4265D32368980728D5FE
:103F0000590704D575498A6842F4E0528A601A0755
:103F100004D572498A6842F460428A60A26892B10C
:103F2000C02A10D000F2BD80A02A0CD000F2B580CB
:103F300022F01001802906D0694840F27E21FDF769
:103F4000FFF9A26823686548816821F0F0010A43FF
:103F50008260DF0727D56368032B00F2B180012B55
:103F600000F0A8809A1E012A5C4A126840F29180F3
:103F7000910725D5594EB26822F003021343B3606E
:103F8000FDF756FF41F28838074605E0FDF750FF80
:103F9000C01B404500F29B80B368626803F00C03CD
:103FA000B3EB820FF2D14C4A136803F00703AB4224
:103FB00014D9EBB21370136803F00703AB420DD0B2
:103FC0000120BDE8F081EBB21370136803F0070322
:103FD000AB42F5D12368980792D4BAE723685A0711
:103FE00018D5E16831F480520ED021F40062B2F5A8
:103FF000A05F09D0B1F5C05F06D040F2C3213848B8
:10400000FDF79EF9E16823683448826822F4E052A3
:104010000A4382601B0718D5226932F480530DD001
:1040200022F40063B3F5A05F08D0B2F5C05F05D0FD
:104030002B4840F2CA21FDF783F9226927498B6892
:1040400023F4604343EAC2038B60FFF70DFF234A6A
:10405000244C92682449C2F303120346A25C23480D
:10406000D34000680B60FDF71DFB0020BDE8F08128
:104070001B4840F25B21FDF763F9174BEDB21A685C
:104080001D701B689CE7164840F25A21FDF758F94D
:104090002AE790013FF56EAF92E7B02A3FF453AFA5
:1040A0004AE7E02A3FF44FAF22F02001D0297FF405
:1040B00043AF48E7094A126896033FF55BAF7FE7D5
:1040C000074840F28521FDF73BF9636847E7032085
:1040D00077E70120704700BF003C024000380240F3
:1040E00084F1010800F00108000000200800002011
:1040F000014B1868704700BF00000020044B0549C1
:104100009B68054A0868C3F38223D35CD840704794
:10411000003802400000002010F00108044B05495F
:104120009B68054A0868C3F34233D35CD8407047A4
:10413000003802400000002010F001080E4B0F2252
:1041400002609A6802F0030242609A6802F0F0028C
:1041500082609A6802F4E052C2609B68DB0810B487
:1041600003F4E053054C036123685DF8044B03F04E
:1041700007030B60704700BF00380240003C02405C
:10418000F8B1114B02689A4210B5044603D00F48AB
:10419000A321FDF7D5F8637903F0FF0263B121682D
:1041A000022363710B68012043F0040300220B60BB
:1041B00060711046A26010BD22712046FDF7D2F852
:1041C000EDE70120704700BF00080650BCF1010870
:1041D000F8B50379012B27D0437901229342044695
:1041E0000271DEB206D004238360164600232371D9
:1041F0003046F8BD022343710D46FDF719FE2368D2
:1042000007465A68D20712D4FDF712FEC01B0228D7
:104210002368F6D95A6812F00102F2D10121022373
:1042200061712271A360E3E702263046F8BD9B6806
:10423000E36001222B6000266271D7E72DE9F0418F
:1042400082B01D4616460C460746FDF7F1FD354483
:104250002D1AFDF7EDFD274B1B68C3F3CB3305FB90
:1042600003F380460193731C396807D18B6834EAE5
:104270000303FBD0002002B0BDE8F0818B6834EA74
:104280000303F7D1FDF7D4FDA0EB0800A84208D244
:10429000019B002B019B03F1FF3308BF0025019315
:1042A000E1E7D7E900315A68B1F5827F22F0E002F8
:1042B0005A6013D0BA6AB2F5005F07D11A6822F4C7
:1042C00000521A601A6842F400521A600122002358
:1042D00087F8512087F850300320CCE7BA68B2F550
:1042E000004F02D0B2F5806FE4D11A6822F040028C
:1042F0001A60DFE70000002038B513464268B2F5C7
:10430000827F044606D00A460121FFF797FF78B95D
:10431000002038BD8268B2F5004F1CD0B2F5806F26
:104320000CD00A4620468021FFF788FF0028EFD0F6
:10433000636D43F020030320636538BD05680A46BA
:10434000296821F0400129600121FFF777FF00284B
:10435000EED10020DDE70068026822F04002026032
:104360000A4620468021FFF769FF0028D0D0DFE70A
:10437000002800F00A8138B5944A03689342044645
:104380000CD0A2F57842934208D002F580629342A5
:1043900004D08F484FF4A071FCF7D2FF63683BB1A3
:1043A000B3F5827F04D08A4840F24111FCF7C8FF80
:1043B000A36833F4806240F0AA80E36833F40063BA
:1043C00040F0B380A36933F4007203D0B3F5802FBB
:1043D00040F0D180E36983B1182B40F2B980203BD3
:1043E000182B05D84FF0013222FA03F3DB0704D46F
:1043F000774840F24511FCF7A3FF236A33F08003AE
:1044000004D073484FF4A371FCF79AFF636A002B42
:104410005DD1236933F0020304D06D484FF4A571D8
:10442000FCF78EFF6369012B04D9694840F24B11F8
:10443000FCF786FF6368B3F5827F00F0A880002355
:10444000E36194F851300021A16203F0FF02002BD8
:1044500000F08880D4E90130E268256800F4044067
:1044600003F48273034302F4006003432069A269EA
:1044700000F002000343022084F85100606900F05C
:1044800001000343E06902F4007E00F0380C206A6A
:1044900043EA0E0300F0800043EA0C0303430B439E
:1044A000616A120C01F0100102F004020A4329684B
:1044B00021F0400129602B606A60EB6923F40063FE
:1044C000EB6100200123606584F8513038BD102B6A
:1044D00007D03F4840F24711FCF732FF636A002BD8
:1044E00097D0E3697BB1182B25D9203B182B05D831
:1044F0004FF0013222FA03F3DA0704D4344840F2D1
:104500005911FCF71DFF0023C4E9043399E7B3F503
:10451000004F3FF452AF2E484FF4A171FCF710FF4B
:10452000E36833F400633FF44DAF294840F2431190
:10453000FCF706FF46E7072BE0D9264A22FA03F3E9
:10454000DB07E0D4224840F25911FCF7F9FEDAE724
:10455000072B7FF64DAF1F4A22FA03F3DD077FF5E5
:1045600047AF4AE784F850202046FCF75FFFA16A76
:1045700001F400516EE716484FF4A271FCF7E0FE1B
:10458000E369002B3FF439AF26E701207047E36968
:10459000002B3FF456AF182B0FD9203B182B06D811
:1045A0004FF0013222FA03F3D8073FF54AAF08482B
:1045B00040F24F11FCF7C4FE43E7072BF7D9054A39
:1045C00022FA03F3D907F2D53BE700BF00300140E0
:1045D000F4F10108000101012DE9F0410446806871
:1045E00082B00F4690461E46002840F0AE8094F8F8
:1045F0005000012800F0B380012384F85030FDF70B
:1046000017FC054694F8510063680128C2B211D026
:10461000B3F5827F09D002200122002384F85120C3
:1046200084F8503002B0BDE8F081A1680029F2D1D1
:10463000042AF0D1002F00F09680B8F1000F00F0AE
:104640009280002E00F08F8094F85120C4F83880BA
:10465000042A1CBF052284F8512000226265C4E9A7
:1046600010222268E687E6861168A6874906276336
:10467000A68603D4116841F040011160E168B1F5EC
:10468000006F00F0A880002B00F09B80012E00F04E
:104690009880089B01334FF0010628D065E021681F
:1046A0008B6898070FD5E38E9BB263B15EB1236B25
:1046B0001B780B73E38E226B2168013B01329BB2A6
:1046C0000026E38622638A6812F001020DD0E38F90
:1046D0009BB253B1A36BC9681970E38FA16B013B07
:1046E00001319BB2A163E3871646FDF7A1FBE28E81
:1046F00092B2002AD3D1E38F9BB2002BCFD17E4B55
:104700007E4A1B68A2FB032362684FF47A715B0D3B
:1047100001FB03F3B2F5827F019307D1DCE0019B3B
:104720002268013B019393681B0602D5019B002B75
:10473000F5D1A068002840F08C8023680090DA68EA
:1047400000929B680093009B66E76D4840F27C41B5
:10475000FCF7F6FD94F8500001287FF44DAF0220DD
:1047600002B0BDE8F081012056E7E38E9BB21BB991
:10477000E38F9BB2002BC2D02268936899070FD5B4
:10478000E38E9BB263B15EB1236B1B781373E38E30
:10479000226B013B01329BB222632268E386002632
:1047A000936813F0010304D0E18F89B2002940F02F
:1047B0008780FDF73DFB089B401B9842D5D3032023
:1047C0002AE73B781373E38E226B013B01329BB2E5
:1047D0002263E3865DE7002B3DD137F8023BD360CF
:1047E000E38E2763013B9BB2E386089B01334FF0C6
:1047F000010625D032E023689A6892070DD5E28E33
:1048000092B252B14EB1216B31F8022BDA60E28ED6
:104810002163013A92B20026E2869A6812F0010200
:104820000CD0E18F89B249B1A16BDB6821F8023B62
:10483000E38FA163013B9BB21646E387FDF7F8FACD
:10484000E38E9BB2002BD6D1E38F9BB2002BD2D14B
:1048500055E70020E0E6012EC7D1BEE7E38E9BB20C
:1048600023B9E38F9BB2002B3FF449AF22689368D2
:104870009F070DD5E38E9BB253B14EB1216B31F83A
:10488000023BD360E38E2163013B9BB2E3860026AB
:10489000936813F001030CD0E18F89B249B1D1685C
:1048A000A26B22F8021B1E46E38FA263013B9BB260
:1048B000E387FDF7BDFA089B401B9842CED37EE705
:1048C000A16BD2680A70E28FA16B013A013192B2FA
:1048D000A163E2871E466CE7089A2B46802120469A
:1048E000FFF7ACFC00283FF424AF636D2022134394
:1048F0006365012062658FE600000020819F5E16DF
:10490000F4F101082DE9F0414668B6F5827F82B0E6
:10491000044690461D460F466ED094F85030012B49
:1049200076D0012384F85030FDF782FA94F851C014
:10493000BCF1010F06465FFA8CF009D0022001227B
:10494000002384F8512084F8503002B0BDE8F08193
:10495000002FF4D0B8F1000FF1D0A268A763B2F530
:10496000004F2268A4F83C804FF000034FF0040190
:1049700084F85110C4E9103363652363A386A4F857
:104980003E80E386134607D1116821F04001116093
:10499000116821F4804111601168480603D4116840
:1049A00041F040011160E168002954D0E18F89B2E3
:1049B000A9B1691C3ED19368DB0744D5A36BD168CC
:1049C00023F8021BB4F83EC0A3630CF1FF3C1FFAAE
:1049D0008CFCA4F83EC0E38F9BB2002BEBD1324697
:1049E00029462046FFF788FC08B120236365606DE7
:1049F000003818BF0120A2E78368002B8DD10095F5
:104A00000425134680F851500A46FFF7E5FD9CE760
:104A1000022002B0BDE8F081A26BDB6822F8023B05
:104A2000E38FA263013B9BB2E387E38F9BB2002B32
:104A3000D5D023689A68D207EED4FDF7F9F9801B28
:104A4000A84243D2F1E7FDF7F3F9E38F9BB2002BC5
:104A5000C5D02268AFE7E28F92B2002ABFD06F1CA8
:104A600013D02BE0A26B1B7B1370B4F83EC0A26B7B
:104A70000CF1FF3C1FFA8CFCA4F83EC0E38F01321E
:104A80009BB2A263002BAAD023689A68D007E9D40E
:104A9000FDF7CEF9E38F9BB2002BF5D19FE7A26B18
:104AA0001B7B1370E38FA26B013B01329BB2A263AD
:104AB000E387E38F9BB2002B91D023689A68D107DC
:104AC000EDD4FDF7B5F9801BA842F2D3032036E7F9
:104AD000F8B50446C06C0F4616461D46002800F087
:104AE0008580A06C00287BD0A06800286DD194F848
:104AF0005000012872D094F851000123012884F855
:104B00005030C2B263680CD0B3F5827F04D002206B
:104B1000002384F85030F8BDA368002BF7D1042A95
:104B2000F5D1002F4FD0002E4DD0002D4BD094F852
:104B30005130E06CA586042B1CBF052384F851304E
:104B400000236365E586E58794F85120A587042A4C
:104B5000C4E9103307BF2D4A2D4B2E4A2E4B216836
:104B60002763A663C0E90F32E38F2C4AC264002595
:104B70009BB232460C310565FDF784FB00283BD122
:104B80002268A16C536843F001035360E38E0C323A
:104B9000C1E90F00C1E913009BB20846216BFDF784
:104BA00071FB48BB23681A68520603D41A6842F0A6
:104BB00040021A605A6842F020025A605A6842F075
:104BC00002025A60A4E70120A2E7154840F24271B0
:104BD000FCF7B6FB94F8500001288CD10220F8BDF8
:104BE0000F4840F23F71FCF7ABFB7DE70C4840F209
:104BF0003E71FCF7A5FB74E7636D012243F01003DF
:104C00006365104684F8512082E700BF314C0008EC
:104C1000754C0008414C0008D54D0008514C000867
:104C2000F4F10108704700BF704700BF704700BF34
:104C300008B5806BFFF7FAFF08BD00BF704700BFE3
:104C400008B5806BFFF7FAFF08BD00BF704700BFD3
:104C5000806B026808B5536823F003035360436D0B
:104C6000012143F01003436580F85110FFF7EEFF78
:104C700008BD00BF70B5064682B0856BFDF7D8F859
:104C800032681268D1055BD42A68AB68516821F09C
:104C9000200104465160002B57D068685168B0F578
:104CA000827F21F0010151605DD0FDF7C1F86434CD
:104CB000241AFDF7BDF8464B2A681B68C3F3CB33B3
:104CC00004FB03F301939368DB0706460BD430E043
:104CD000019A019B2968013B01938B68002A08BF58
:104CE0000024DA0725D5FDF7A3F8801B8442EFD80E
:104CF000D5E900315A68B1F5827F22F0E0025A60AE
:104D000049D0AA6AB2F5005F07D11A6822F40052AE
:104D10001A601A6842F400521A60012385F8513073
:104D20006B6D002243F0200385F850206B65202333
:104D30006B6501230022EA8785F851306B6D6BB9F2
:104D40002846FFF76FFF02B070BD6B68B3F5827F36
:104D500053681CD023F001035360A6E72846FFF7F1
:104D600075FF02B070BDB3F5004F20D1136823F07A
:104D7000400313602346642280212846FFF75EFA31
:104D80000028D6D06B6D43F020036B65CFE723F08E
:104D900003035360EEE7AA68B2F5004F02D0B2F504
:104DA000806FAED11A6822F040021A60A9E7B3F50D
:104DB000806FDFD1116821F0400111602346642229
:104DC00001212846FFF73AFA0028B2D0DAE700BFFF
:104DD0000000002030B5054683B0846BFDF728F84D
:104DE0002A681268D20527D4224B22681968224B00
:104DF0005568A3FB0131490D4FF47A7303FB01F1B0
:104E0000636825F02005B3F5827F556001911ED1BE
:104E10000346642280212046FFF710FA00BB226877
:104E20005368002123F0030301205360E186E187EA
:104E300084F85100636D73B92046FFF7F5FE03B0A7
:104E400030BD019B013B019393681B06E8D5019B94
:104E5000002BF6D1E4E72046FFF7F8FE03B030BDA3
:104E6000636D226843F020036365636D43F02003A4
:104E70006365D5E700000020819F5E16026810B5CB
:104E80005168936803F0410CBCF1010F84B00446F3
:104E90005AD0980701D508065ED413F4B07F51D0DC
:104EA00088064FD558060ED594F8510003285DD0DA
:104EB000606D40F00400606500200090D0680090B4
:104EC00090680090009898060CD5606D40F0010045
:104ED00060650020029090680290106820F0400009
:104EE00010600298D80508D5636D002043F00803D0
:104EF0006365039093680393039B636D13B35368D7
:104F000023F0E003536001208B0784F8510029D07F
:104F10005368E06C23F00303536040B1174B036503
:104F2000FDF708FA18B1636D43F040036365A06CA8
:104F300040B1124B0365FDF7FDF918B1636D43F005
:104F40004003636504B010BD11F0400FA1D0036CA5
:104F500004B0BDE810401847636C204604B0BDE8BB
:104F6000104018472046FFF771FEEBE7002301933E
:104F7000D368019393680193019BE3E7814F000895
:104F800008B5806B0023C387C386FFF75FFE08BDAB
:104F900090F85100704700BF002800F0F5800368CA
:104FA0007A4A934210B5044637D0B3F1804F34D0DB
:104FB000A2F57C42934230D002F5806293422CD01D
:104FC00002F58062934228D002F58062934224D099
:104FD00002F58062934220D002F5704293421CD0C9
:104FE00002F57052934218D002F58062934214D0B9
:104FF00002F58062934210D0A2F5983293420CD011
:1050000002F58062934208D002F58062934204D098
:105010005F4840F21311FCF793F9A36833F01002D4
:105020000AD023F04002202A06D0402B04D0584852
:105030004FF48A71FCF784F9236933F4807203D04A
:10504000B3F5007F40F09580A36933F0800342D12F
:1050500094F83D3003F0FF02002B47D022684B4903
:10506000022384F83D308A4213686ED0B2F1804F3B
:1050700042D0A1F57C418A423ED001F580618A424E
:105080003AD001F580618A4236D001F578418A42F2
:105090005BD001F570518A4232D001F580618A42BD
:1050A0002ED001F580618A422AD0A1F598318A423A
:1050B00026D001F580618A4222D001F580618A42C2
:1050C0001ED0A069E16823F0800303431360636886
:1050D000D162936221E02E484FF48B71FCF730F9D6
:1050E00094F83D3003F0FF02002BB7D184F83C2048
:1050F0002046FCF79FFCB1E7A16823F070030B4347
:105100002069A16923F44073034323F08003E0681E
:105110000B4361681360D06291620123536184F88C
:10512000463084F83E3084F83F3084F8403084F8CC
:10513000413084F8423084F8433084F8443084F8B5
:10514000453084F83D30002010BDA068216923F06F
:105150007003034323F440730B43A16923F08003DE
:105160000B431360E368D3626368936263691363FC
:10517000D3E7074840F21511FCF7E2F8A36933F0D2
:1051800080033FF465AFA6E70120704700000140AF
:105190002CF201083A4A0368934210B5044637D00E
:1051A000B3F1804F34D0A2F57C42934230D002F567
:1051B000806293422CD002F58062934228D002F59F
:1051C0008062934224D002F58062934220D002F59F
:1051D000704293421CD002F57052934218D002F5EF
:1051E0008062934214D002F58062934210D0A2F5FF
:1051F000983293420CD002F58062934208D002F5B7
:105200008062934204D01F4840F2CF11FCF798F817
:1052100094F83D30012B2FD123681949022284F8DC
:105220003D20DA688B4242F00102DA6019D0B3F116
:10523000804F16D0144A934213D002F580629342F5
:105240000FD002F5806293420BD002F57842934270
:1052500007D002F57052934203D0A2F594329342E4
:1052600004D19A6802F00702062A07D01A6842F0B1
:10527000010200201A6010BD012010BD002010BDE9
:10528000000001402CF201080004004090F83C307E
:10529000012B00F023820223012270B580F83C200C
:1052A00080F83D300B68B3F5805F04460D4600F092
:1052B000FB80602B00F0618264D823F01002402A4A
:1052C00003D033F0300240F045812268916821F428
:1052D0007F4121F077019160402B00F0018240F284
:1052E000B080502B40F0A580984B9A421FD0B2F16D
:1052F000804F1CD0A3F57C439A4218D003F58063FD
:105300009A4214D003F580639A4210D003F5784393
:105310009A420CD003F570539A4208D0A3F5943307
:105320009A4204D08A4841F2F641FCF709F86B68CA
:10533000B3F5004F09D033F0020206D00A2B04D097
:10534000834841F2F941FBF7FBFFEE680F2E00F2B4
:105350001C82236869681A6A22F00A0211431A6AD9
:1053600022F001021A629A6922F0F00242EA061261
:105370009A6119629A6822F0700242F05702002086
:105380009A6057E0702B00F04481B3F5005F98D12C
:105390000268936823F47F4323F0770393606B4B99
:1053A0009A4217D0B2F1804F14D0A3F57C439A42B1
:1053B00010D003F580639A420CD003F580639A42C3
:1053C00008D003F578439A4204D0614841F2E241A3
:1053D000FBF7B6FFAB6833F4405304D05C4841F2AE
:1053E000E541FBF7ADFF6B68B3F5004F09D033F033
:1053F000020206D00A2B04D0554841F2E641FBF7E1
:105400009FFFE8680F2800F2CE812268D5E901539A
:1054100091682B4321F47F410B4343EA00239360BF
:10542000936843F480430020936003E033F010015D
:105430000CD001200122002384F83D2084F83C3068
:1054400070BD202B02D0F1D9302BF2D13F498A42D6
:1054500021D0B2F1804F1ED0A1F57C418A421AD0F2
:1054600001F580618A4216D001F580618A4212D02E
:1054700001F578418A420ED001F570518A420AD076
:10548000A1F594318A4206D0314841F22951FBF707
:1054900057FF22682B68916821F070010B4343F09D
:1054A000070300209360C5E70268936823F47F43F5
:1054B00023F077039360254B9A4200F00081B2F10C
:1054C000804F00F0FC80A3F57C439A4200F0F78007
:1054D00003F580639A4200F0F28003F580639A42FC
:1054E00000F0ED8003F580639A4200F0E88003F558
:1054F00080639A4200F0E38003F570439A4200F023
:10550000DE8003F570539A4200F0D98003F5806382
:105510009A4200F0D48003F580639A4200F0CF8075
:10552000A3F598339A4200F0CA8003F580639A424B
:1055300000F0C58003F580639A4200F0C080044803
:1055400041F2C341FBF7FCFE002073E7000001407D
:105550002CF2010841F2B7419D48FBF7F1FE2268A9
:105560002B68916821F47F4121F07701602B9160D5
:1055700040F0A780974B9A421FD0B2F1804F1CD0C9
:10558000A3F57C439A4218D003F580639A4214D065
:1055900003F580639A4210D003F578439A420CD009
:1055A00003F570539A4208D0A3F594339A4204D07D
:1055B000874841F20651FBF7C3FE6B68B3F5004F15
:1055C00009D033F0020206D00A2B04D0804841F201
:1055D0000951FBF7B5FEE8680F2800F2EB8023685D
:1055E0006D681A6A22F010021A6299691A6A21F427
:1055F000704122F0A00241EA003142EA05129961AD
:105600001A629A6822F0700242F0670200209A60E3
:1056100010E70268936823F47F4323F077039360D5
:105620006C4B9A421FD0B2F1804F1CD0A3F57C4343
:105630009A4218D003F580639A4214D003F5806330
:105640009A4210D003F578439A420CD003F5705378
:105650009A4208D0A3F594339A4204D05C4841F2B0
:10566000CA41FBF76DFEAB6833F4405304D0584891
:1056700041F2CD41FBF764FE6B68B3F5004F09D0F2
:1056800033F0020206D00A2B04D0514841F2CE4139
:10569000FBF756FEE8680F2800F293802268D5E9F0
:1056A000015391682B4321F47F410B4343EA0023CC
:1056B0009360936843F0770300209360BAE600207C
:1056C000B8E67FF609AEB3F5805F3FF4F4AEB3F50C
:1056D000005F3FF464AE702BA2D0AAE602207047B0
:1056E0003C4B9A421FD0B2F1804F1CD0A3F57C43B3
:1056F0009A4218D003F580639A4214D003F5806370
:105700009A4210D003F578439A420CD003F57053B7
:105710009A4208D0A3F594339A4204D02C4841F21F
:105720001651FBF70DFE6B68B3F5004F09D033F04F
:10573000020206D00A2B04D0254841F21951FBF78A
:10574000FFFDEE680F2E27D8236869681A6A22F0D9
:105750000A0211431A6A22F001021A629A6922F0BF
:10576000F00242EA06129A6119629A6822F0700207
:1057700042F0470200209A605CE60268936823F4D6
:105780007F4323F077039360F4E6114841F2FA4136
:10579000FBF7D6FDEE68DCE50D4841F21A51FBF748
:1057A000CFFDEE68D0E70A4841F2E741FBF7C8FDBC
:1057B000E8682AE6064841F20A51FBF7C1FDE868AD
:1057C0000DE7034841F2CF41FBF7BAFDE86865E712
:1057D0002CF2010800000140704700BF704700BF75
:1057E000704700BF704700BF03681A69910710B582
:1057F000044602D5DA6892075FD41A69500702D5C9
:10580000DA68510746D41A69120702D5DA68100718
:105810002ED41A69D20602D5DA68D00618D41A69CD
:10582000D10702D5DA68D2075DD41A69100602D50D
:10583000DA6811065FD41A69520602D5DA68500692
:1058400061D41A69910602D5DA68920643D410BD74
:105850006FF01001082219612277DB6913F4407F91
:10586000204664D0FFF7BAFF002223682277D6E7EC
:105870006FF00801042219612277DB69990720463D
:1058800052D1FFF7A9FF2046FFF7AAFF00222368A5
:105890002277BEE76FF004010222196122779B692B
:1058A00013F4407F20463CD1FFF796FF2046FFF7D8
:1058B00097FF002223682277A5E76FF002010122FB
:1058C000196102779B699B0725D0FFF787FF0022AC
:1058D0002368227791E76FF0200220461A61BDE825
:1058E000104000F0B9B86FF001021A612046FBF7D2
:1058F0001BFD236899E76FF080021A61204600F0D3
:10590000ADF8236897E76FF040021A612046FFF771
:1059100069FF236895E7FFF75FFF2046FFF760FF09
:10592000D5E7FFF75BFFC4E7FFF758FFAEE7FFF7E8
:1059300053FF2046FFF754FF96E700BF38B5444AAF
:105940000368934204460D461FD0B3F1804F1CD02C
:10595000A2F57C42934218D002F58062934214D0A3
:1059600002F58062934210D002F5806293420CD01F
:1059700002F58062934208D002F57042934204D04F
:10598000344840F2B171FBF7DBFC2B6833F0400286
:105990000CD0402B47D9602B08D023F02003502B8C
:1059A00004D02C4840F2B271FBF7CAFC6B6833F0AC
:1059B000800342D194F83C30012B47D02368022267
:1059C00084F83D205A682868996822F070020243E2
:1059D0005A601F4A93421AD0B3F1804F17D0A2F5F4
:1059E0007C42934213D002F5806293420FD002F5BD
:1059F000806293420BD002F57842934207D002F5C1
:105A00007052934203D0A2F59432934204D16A6853
:105A100021F08001114399600020012384F83D307A
:105A200084F83C0038BD202BC0D023F02003102B7D
:105A3000B7D16B6833F08003BCD0064840F2B37135
:105A4000FBF77EFC94F83C30012BB7D1022038BD27
:105A50000000014064F20108704700BF704700BFBA
:105A600038B54268494B9A42044600F28380E368A5
:105A700033F4005304D0464840F66261FBF760FC03
:105A8000236933F4806202D0B3F5C06F78D16069C6
:105A90004FF6F373184266D1002864D02268E1689B
:105AA0001369256923F440530B431361A368D1683C
:105AB0002B43E56921F4164121F00C012B430B43E4
:105AC0000343D3605369A069324923F4407303430D
:105AD0008A42536128D0304B9A4225D0FEF70EFB04
:105AE000E369B3F5004F25D16268192192184FF090
:105AF00000035B41A0FB0101FBF7C6F8274A2468BD
:105B0000A2FB00314909642303FB1103DB0032339C
:105B1000A2FB0323C3F342121B0902EB011203F49D
:105B2000F8731344A36038BDFEF7F8FAE369B3F5E0
:105B3000004FD9D0636819219A00A0FB01019B0F87
:105B4000FBF7A2F8154AA2FB00135B092168642445
:105B500004FB130000013230A2FB00201B0103EB09
:105B600050138B6038BD0A4840F66461FBF7E8FBD0
:105B7000606993E7064840F66161FBF7E1FB76E771
:105B8000034840F66361FBF7DBFB80E7A037A0002A
:105B9000A0F2010800100140001401401F85EB51E4
:105BA000002800F0888038B583690446002B50D067
:105BB000026842498A426AD0A1F54C418A4266D0C5
:105BC00001F580618A4262D001F54C418A425ED083
:105BD0003B4840F27311FBF7B3FBA369002B56D18E
:105BE000A36833F4805304D035484FF4BD71FBF7FC
:105BF000A7FBE36933F4004304D0314840F27B1142
:105C0000FBF79EFB94F83D3003F0FF02002B4CD0D5
:105C10002268242384F83D30D36823F400532046BF
:105C2000D360FFF71DFF23681A6922F490421A61BE
:105C30005A6922F02A025A61DA680025202142F4CA
:105C40000052DA60256484F83D1084F83E1028463E
:105C500038BD0368194A9342C2D0A2F54C42934220
:105C6000BED002F580629342BAD002F580629342C0
:105C7000B6D002F580629342B2D002F5444293421C
:105C8000AED00F484FF4BC71FBF75AFBA8E723F4E2
:105C90000072B2F5807FA3D0B3F5007FA0D0084892
:105CA0004FF4BA71FBF74CFB9AE784F83C2020468E
:105CB000FBF746FFACE70120704700BF0010014032
:105CC000A0F201082DE9F843054690F83D00202890
:105CD00077D18946002940D01446002A3DD01E467F
:105CE00095F83C30012B6CD0012385F83C304FF007
:105CF00000082123C5F8408085F83D30FCF798F86E
:105D0000AB68AC84B3F5805FEC8407465CD0EB8C69
:105D100000229BB285F83C20002B7ED02C68721CA0
:105D20001ED122681306FCD5B9F1000F44D019F832
:105D3000013B6360EB8C013B9BB2EB84EB8C9BB231
:105D4000002BECD1711C45D123685A06FCD52023C9
:105D500085F83D300020BDE8F8830120BDE8F883D8
:105D600023681806E0D42EB1FCF762F8C01B864207
:105D70002C68D4D204F10C0353E8003F23F4D07311
:105D800004F10C0141E80032002AF3D104F11403BC
:105D900053E8003F23F0010304F1140141E800320D
:105DA000002AF3D1202385F83D3085F83C2085F882
:105DB0003E300320BDE8F88338F8023BC3F3080304
:105DC000B7E70220BDE8F8832B69002B9FD1C846B6
:105DD00099469CE723685B06B9D42EB1FCF728F8F6
:105DE000C01B86422C68ADD204F10C0353E8003F7F
:105DF00023F4D07304F10C0141E80032002AF3D1FE
:105E000004F1140353E8003F23F0010304F11401EB
:105E100041E80032002AF3D1C4E72C6892E700BFC2
:105E2000002070472DE9F043144CDFF85480DFF870
:105E3000549083B00646002720684FF0FF3100F0F1
:105E40000FFC0028F8D198F800300197002BF3D10F
:105E500001A94846FCF7B2FE019D31462846002DB7
:105E6000EAD0336998470028EDD0284606F006FEB0
:105E700098F800300197002BDED1E9E7D40A002022
:105E8000D00A0020140B0020FBF7D2BF08B502484F
:105E9000FDF7F6F8002008BD140B0020844608B575
:105EA000054813460A466146FCF7B8FF003818BF9C
:105EB0000120404208BD00BF140B0020844608B5F5
:105EC000054813460A466146FCF7D0FF003818BF64
:105ED0000120404208BD00BF140B002030B58DB03A
:105EE0000C4630220021684615F086FC5CB3D4E9EC
:105EF00000316289CDE90012EBB1D3E90020598964
:105F0000049103AB03900293A2B1D2E9003051890E
:105F1000079106AA06900592002B32D0D3E9002003
:105F200059890A9109AB0990089342B36FF00B00AD
:105F30000DB030BD01230CAA03EB430302EB830336
:105F4000002243F8282C104D23896B602046C5F8A9
:105F500008D06C6306F040FF29460C480C4DFCF756
:105F6000F7FD28684FF0FF3100F07AFB0446002867
:105F7000F7D10648FCF7B4FE20460DB030BD032330
:105F8000D9E70223D7E700BFD80A0020140B00206E
:105F9000100B002008B50146074806F06BF9074BC7
:105FA0001A78012A00D008BD054900221A70BDE800
:105FB0000840086800F080BB78F30108D00A002090
:105FC000D40A0020014B186800F076BBD40A0020E8
:105FD000014B186800F070BB100B002008B5FDF7EE
:105FE0008DF8030600D408BD024B1868BDE80840D0
:105FF00000F062BBD40A0020F0B50446A3B000282C
:1060000000F0B2805C4B5D485D4A5E4D206347F214
:106010007341E187626100216422A36109A815F040
:10602000EBFB594A2A604FF40002AA60574AEA6023
:10603000574A2A61574BC5F804D04FF4C0626A61D1
:106040001A6800921A795B798DF8053028468DF828
:106050000420FCF795FB504F342200210646381DE2
:1060600015F0CAFB21234D483B604FF440037B6190
:1060700006F052F86B684A4D062284F83C201A78E4
:1060800084F836205A7884F837209A7884F83820B3
:10609000DA7884F839201A7984F83A2094F83D2087
:1060A000597984F83B1042F00A0340F2DC52A28690
:1060B00084F83D3003220021012000F0B9FC394B67
:1060C000032218600021012000F0B2FC364B18605A
:1060D0000FCD0DF1080CACE80F0095E807008CE837
:1060E0000700214602A800F0ABF930493048FBF721
:1060F000A7FD2F48FBF7BCFD1EBB2D48FBF724FE78
:10610000012828DD0338022820D82A4A2A4B52F8D1
:10611000206053F820501B4809A9FCF7CDFE09A9BF
:106120001848CDE90E56FCF72DFF1648FCF752FC37
:10613000204606F063FA204606F0E0FA002023B07D
:10614000F0BDFBF7FBF8002023B0F0BD4FF4804515
:106150004FF40066DFE7204606F018FB204606F005
:106160008DFA002023B0F0BD144B1549154840F2BC
:10617000E71215F097FA45E7DD5E000830F30108F5
:10618000D96D0108140B002000800240100A002085
:1061900070090020F0190120D80A002078F30108C6
:1061A000A4EE0108D40A0020100B00200C000020EF
:1061B000B00A002040F301084CF30108DCF20108AA
:1061C000F8F2010808F30108FBF732BEF0B5424BC4
:1061D00002688DB000249A42CDE90644CDE9084416
:1061E0000A9401D00DB0F0BDA3F5904300941A6B52
:1061F0003A4842F000721A631A6B02F00072009281
:10620000009A01941A6B42F080621A631A6B02F0D2
:1062100080620192019A02941A6B42F000621A6342
:106220001A6B02F000620292029A03941A6B42F017
:1062300004021A631A6B02F004020392039A049494
:106240001A6B42F001021A631A6B02F00102049207
:10625000049A05941A6B42F002021A631B6B03F056
:1062600002033222059303260B2506A90223CDE95A
:1062700006230227059BCDE90965FDF7B7F98623BB
:1062800006A917480A95CDE90637CDE90846FDF776
:10629000ADF94FF4605306A912480693CDE90846BC
:1062A00007970A95FDF7A2F9224605213D20FBF745
:1062B000F5FD3D20FBF73CFE224608210A48FDF78C
:1062C00033FB3220FBF7BAFD074801220821FDF716
:1062D0002BFB0DB0F0BD00BF008002400008024063
:1062E0000000024000040240000C02402DE9F04F83
:1062F00004469BB06422002101A815F07DFA002716
:10630000236ADFF894B0DFF894A0214D214E204697
:106310009847B946B84604E001280DDC642000F037
:10632000C1F82846FBF710FD94F83D305A07F3D525
:1063300001281EDD5B07F1D40238032823D85BF85F
:1063400020905AF8207001A93046FCF7B5FD01A94C
:106350003046CDE90697FCF715FE3046FCF73AFBD0
:10636000204606F04BF9204606F0C8F94FF0010828
:10637000D4E73046FCF78EFB204606F07FF9204636
:1063800006F004FACAE7B8F1000FC7D0DBE700BF98
:10639000B00A0020140B002058F3010868F301082C
:1063A00010B5044682B00D4805F0FEFE034678B1F4
:1063B00000F120020A4922604FF4C06019610021F7
:1063C000CDE900204122084606F088FA02B010BD4F
:1063D000044A20600121117002B010BD78F3010859
:1063E000955F0008D00A002030B4002542F8205CF8
:1063F000A2F1200422F8163C22F8185C026862B16F
:106400000A6814600C6002682AB11189194411816C
:106410001268002AF9D130BC70470460F2E700BF6F
:1064200006F02CBB08B501F0ADFE002008BD00BF92
:10643000EFF305830BB101F059BF01F051BF00BF6D
:1064400070B5446986B084460B46ACB186699EB18E
:10645000BCF908E0DCF80010DCF810204068BEF160
:10646000840F14BF0EF103050025CDE90146009508
:1064700001F0FAFC06B070BDBCF90840BCF8102071
:10648000842C14BF03340024DCE90010009405AC14
:10649000019401F09FFD01280CBF0598002006B073
:1064A00070BD00BF08B5012838BF012001F03AFED9
:1064B000002008BD00B5002385B0CDE90233EFF31D
:1064C0000583BBB102AB0093012203AB02F054FA87
:1064D000012815D1029B4BB14FF0E0234FF08052C1
:1064E000C3F8042DBFF34F8FBFF36F8F039805B030
:1064F0005DF804FB03AB012202F0BEF90128F5D0E0
:106500004FF00040F3E700BF30B585B000230446EC
:106510000293EFF3058048B18223019304AB13E9A2
:10652000070084E80700204605B030BD1346154635
:1065300002AA02F051F9012804D02B1E18BF012332
:106540009B01EAE7029B002BACBF08238623E4E70C
:106550004168012009B100F0CBBC00F037BD00BF9D
:1065600010B582B00024019410B3EFF3058333B962
:1065700000F09EFF012818D1002002B010BD01AA32
:10658000214601F03FF901280FD1019B002BF3D0E8
:106590004FF0E0234FF08052C3F8042DBFF34F8F2C
:1065A000BFF36F8F204602B010BDFF2002B010BDB8
:1065B000802002B010BD00BF10B582B0002401944D
:1065C000EFF305839BB101A900F09CFD012814D1D4
:1065D000019BABB14FF0E0234FF08052C3F8042D84
:1065E000BFF34F8FBFF36F8F204602B010BD1A4626
:1065F000194600F0FFFA012802D0FF2002B010BDBA
:10660000002002B010BD00BF30B5446883B008461A
:1066100094B1012905D0224603B0BDE8304000F016
:1066200047BA0022032300931146234600F094F951
:106630000546284603B030BD012904D003B0BDE8AB
:10664000304000F093BA0322214600F0F1F90546EC
:106650000028EED023462246214600F0CBFAE8E798
:1066600010B582B00024019410B3EFF3058333B961
:1066700000F01EFF012818D1002002B010BD01AAB1
:10668000214601F0BFF801280FD1019B002BF3D068
:106690004FF0E0234FF08052C3F8042DBFF34F8F2B
:1066A000BFF36F8F204602B010BDFF2002B010BDB7
:1066B000802002B010BD00BF10B582B0002401944C
:1066C000EFF305839BB101A900F01CFD012814D153
:1066D000019BABB14FF0E0234FF08052C3F8042D83
:1066E000BFF34F8FBFF36F8F204602B010BD1A4625
:1066F000194600F07FFA012802D0FF2002B010BD39
:10670000002002B010BD00BF10B5EFF305841CB926
:1067100001F0FAF8204610BD8224204610BD00BFCB
:1067200082685AB1C3684BB110B582B00024D0E979
:106730000001009400F010F902B010BDD0E9000192
:10674000002200F075B900BF10B584B0002401919B
:106750000394EFF305835BB1234603AA01A900F07C
:106760006BFC01280CD1039B6BB9002004B010BD59
:10677000012A38BF012201A900F03CFA0128F4D017
:10678000FF2004B010BD4FF0E0234FF08052C3F85B
:10679000042DBFF34F8FBFF36F8F204604B010BDA1
:1067A00030B50B4685B00021CDE9021304468BB30A
:1067B0000091EFF3058199B902A91846154600F03A
:1067C000F9FC012829D02A1E18BF0122920101924A
:1067D00004AB13E9070084E80700204605B030BD8C
:1067E00018466A4602A901F00DF8A0F10100B0FABE
:1067F00080F04009009B00010190002BE8D04FF091
:10680000E0234FF08052C3F8042DBFF34F8FBFF346
:106810006F8FDDE780230193DAE710230193D7E739
:10682000EFF305830BB101F061B801F049B800BF87
:1068300010B5EFF305841CB901F066F8204610BDD1
:106840008224204610BD00BF00F108034FF0FF3145
:106850000022C0E90131C0E903330260704700BF84
:1068600000230361704700BF43689A688A6002682A
:1068700010B49C684B600132616099605DF8044B14
:1068800008610260704700BF30B40D686B1C10D007
:1068900000F108031C465B681A68AA42FAD902682C
:1068A0004B60013299608C606160086130BC0260AD
:1068B000704704696368F2E7036910B4D0E9011214
:1068C0005C688A608442516008BF5A601A685DF84B
:1068D000044B0021013A01611A601868704700BF3B
:1068E00070B50446006CA66B20B925684DB301361F
:1068F000A66370BD154602467DB9606815F072F852
:106900006368226C1344A2686360934224BF2368C7
:10691000636001362846A66370BDE06815F062F832
:10692000226CE36851429B1A2268E360934202D2D0
:10693000A3680B44E360022D08D001360020A66353
:1069400070BDA06801F080FEA560D0E7012E38BFC1
:1069500001260020CCE700BF40B94FF0500383F37D
:106960001188BFF36F8FBFF34F8FFEE710B51C4642
:1069700082B07BB102B3B1B148230193019B482B94
:1069800023D04FF0500383F31188BFF36F8FBFF311
:106990004F8FFEE74FF0500383F31188BFF36F8FE3
:1069A000BFF34F8FFEE74FF0500383F31188BFF31F
:1069B0006F8FBFF34F8FFEE781BB48220192019A90
:1069C000482ADED1019A224600E0019B22604FF066
:1069D000010C84F846C0C4E90F0102F0CBF8D4E9F9
:1069E0000F122368636002FB01F18A1A19441A44EA
:1069F000A1600020FF21A063E26084F8441004F14C
:106A0000100084F84510FFF71FFF04F12400FFF782
:106A10001BFF02F0D1F8204602B010BD4FF050032A
:106A200083F31188BFF36F8FBFF34F8FFEE700BF73
:106A300040B94FF0500383F31188BFF36F8FBFF35A
:106A40004F8FFEE770B5054601FB00F048300E465B
:106A500002F0F2F9044630B3002380F8463026B342
:106A600000F148032360C4E90F5602F083F8D4E92B
:106A70000F232168616003FB02F2D31A0A440B441E
:106A8000A2600020FF22A063E36084F8442004F1A8
:106A9000100084F84520FFF7D7FE04F12400FFF72B
:106AA000D3FE02F089F8204670BD0346DAE700BF46
:106AB00040B94FF0500383F31188BFF36F8FBFF3DA
:106AC0004F8FFEE7884208D24FF0500383F31188BE
:106AD000BFF36F8FBFF34F8FFEE730B5154685B01C
:106AE000002A39D048230393039B482B08D04FF04A
:106AF000500383F31188BFF36F8FBFF34F8FFEE70F
:106B00000024012382F846302A60C2E90F04019173
:106B1000039B02F02FF8D5E90F032A68AC6303FB4F
:106B200000F0C31A4FF0FF0E1044134485F844E000
:106B30006A60EB6085F845E0A86005F11000FFF79A
:106B400083FE05F12400FFF77FFE02F035F801997E
:106B5000A963284605B030BD4FF0500383F3118878
:106B6000BFF36F8FBFF34F8FFEE700BFF8B540B99B
:106B70004FF0500383F31188BFF36F8FBFF34F8F34
:106B8000FEE788420E46044608D24FF0500383F3D6
:106B90001188BFF36F8FBFF34F8FFEE7482002F0DD
:106BA0004BF9054618B30027C0E90F4780F8467037
:106BB000006001F0DFFFD5E90F232968AF6303FB15
:106BC00002F2D31A0A440B44AA60FF2285F844203B
:106BD0006960EB6085F8452005F11000FFF734FE91
:106BE00005F12400FFF730FE01F0E6FFAE63284612
:106BF000F8BD00BF2DE9F04385B00192002800F0F8
:106C0000A48088461F460446002900F09180022F88
:106C10000BD1E36B012B08D04FF0500383F31188A5
:106C2000BFF36F8FBFF34F8FFEE701F0ADFC05465A
:106C3000002800F09380002504F1240601F09AFF5B
:106C4000A26BE36B9A42C0F0EF80022F00F0EC8061
:106C50000198002800F00181002D00F0E18001F092
:106C6000ABFF01F025FB01F085FF94F84430FF2BCA
:106C700004BF002384F8443094F84530FF2B04BF50
:106C8000002384F8453001F097FF01A902A801F024
:106C900027FC002840F0E68001F06CFFA26BE36B5C
:106CA0009A4268D001F088FF01F064FF94F8452013
:106CB00055B2002D04DC11E06A1ED3B255B26BB19F
:106CC000636A304653B101F0B7FB0028F4D001F0FD
:106CD0004FFC6A1ED3B255B2002BF1D1FF2384F8CA
:106CE000453001F069FF01F045FF94F8442055B2AA
:106CF000002D14DD04F1100903E06A1ED3B255B271
:106D00006BB12369484653B101F096FB0028F4D0DB
:106D100001F02EFC6A1ED3B255B2002BF1D1FF2335
:106D200084F8443001F048FF01F0CAFA012585E7F4
:106D3000036C002B3FF46BAF4FF0500383F31188CB
:106D4000BFF36F8FBFF34F8FFEE74FF0500383F316
:106D50001188BFF36F8FBFF34F8FFEE7019B002BAE
:106D60003FF46AAF4FF0500383F31188BFF36F8F86
:106D7000BFF34F8FFEE704F1100901F01DFF0199E9
:106D8000484601F009FB01F0F5FE94F845305DB28C
:106D9000002D04DC11E06B1EDAB25DB26AB1636AE9
:106DA000304653B101F048FB0028F4D001F0E0FB7D
:106DB0006B1EDAB25DB2002AF1D1FF2384F84530B0
:106DC00001F0FAFE01F0D6FE94F844305DB2002DD9
:106DD00004DC11E06B1EDAB25DB26AB12369484689
:106DE00053B101F029FB0028F4D001F0C1FB6B1E68
:106DF000DAB25DB2002AF1D1FF2384F8443001F009
:106E0000DBFE01F05DFA002890D14FF0E0234FF057
:106E10008052C3F8042DBFF34F8FBFF36F8F85E708
:106E200002A801F051FB1AE73A4641462046FFF717
:106E300057FD636A002B53D148B14FF0E0234FF068
:106E40008052C3F8042DBFF34F8FBFF36F8F01F053
:106E5000B3FE012005B0BDE8F083009001F0ACFE68
:106E60000098F7E701F086FE94F845305DB2002DFA
:106E700010DD04F1240603E06B1EDAB25DB24AB104
:106E8000636A304633B101F0D7FA0028F4D001F03C
:106E90006FFBF1E7FF2384F8453001F08DFE01F030
:106EA00069FE94F844305DB2002D10DD04F1100647
:106EB00003E06B1EDAB25DB24AB12369304633B1EA
:106EC00001F0BAFA0028F4D001F052FBF1E7FF23F9
:106ED00084F8443001F070FE01F0F2F90020B9E7C7
:106EE00004F1240001F0A8FA0028B0D0A5E700BF03
:106EF000002941D030B583B048230193019B482B32
:106F000008D04FF0500383F31188BFF36F8FBFF3A6
:106F10004F8FFEE7002501230C46C1E90F3581F8AC
:106F200046300960019B01F025FED4E90F2321685A
:106F3000616003FB02F2D31A0A440B44A260FF22F1
:106F4000E360A56304F1100084F8442084F8452030
:106F5000FFF77AFC04F12400FFF776FC01F02CFE29
:106F6000A5602560E5602B462A4629462046FFF7A6
:106F700041FE204603B030BD4FF0500383F311882B
:106F8000BFF36F8FBFF34F8FFEE700BF38B538B147
:106F90008568044601F0F2FA85420AD0002038BD27
:106FA0004FF0500383F31188BFF36F8FBFF34F8F00
:106FB000FEE7E368013BE3600BB1012038BD1A46F0
:106FC00019462046FFF716FE012038BD38B5482087
:106FD00001F032FF044660B30025012380F84650DB
:106FE0002060C0E90F3501F0C5FDD4E90F23216809
:106FF000616003FB02F2D31A0A440B44A260FF2231
:10700000E360A56304F1100084F8442084F845206F
:10701000FFF71AFC04F12400FFF716FC01F0CCFD89
:10702000A5602560E5602B462A4629462046FFF7E5
:10703000E1FD204638BD00BF00284BD02DE9F041CE
:107040000E4617461D46044621B3022D0BD1E36BB5
:10705000012B08D04FF0500383F31188BFF36F8FDB
:10706000BFF34F8FFEE701F0B9FEEFF311884FF049
:10707000500383F31188BFF36F8FBFF34F8FA26B61
:10708000E36B9A4212D3022D10D0002088F31188AE
:10709000BDE8F081036C002BD7D04FF0500383F391
:1070A0001188BFF36F8FBFF34F8FFEE72A4694F826
:1070B0004550A36B31466DB22046FFF711FC6B1CA7
:1070C00011D06B1C5BB284F84530012088F3118825
:1070D000BDE8F0814FF0500383F31188BFF36F8F49
:1070E000BFF34F8FFEE7636A002BEED004F124005C
:1070F00001F0A2F90028E8D0002FE6D00120386086
:10710000C4E700BF70B3036C70B5064643B14FF0DF
:10711000500383F31188BFF36F8FBFF34F8FFEE7E8
:1071200003680C463BB301F059FEEFF311854FF0B5
:10713000500383F31188BFF36F8FBFF34F8FB36B8F
:10714000F26B9A4223D996F845200133FF2AB363A4
:1071500053B220D001335BB286F84530012085F36D
:10716000118870BD4FF0500383F31188BFF36F8F08
:10717000BFF34F8FFEE78368002BD4D04FF050034E
:1071800083F31188BFF36F8FBFF34F8FFEE70020AB
:1071900085F3118870BD736A002BDFD006F12400DF
:1071A00001F04AF90028D9D0002CD7D00120206066
:1071B000EEE700BF2DE9F04385B00192002800F012
:1071C0005C810F460446002979D001F0DDF90028E2
:1071D00000F0818001F0CEFCA56B002D40F03881DD
:1071E000019B002B00F0D58002A801F06DF9A846A4
:1071F00004F1240601F0E0FC01F05AF801F0BAFCB9
:1072000094F84430FF2B08BF84F8448094F845304C
:10721000FF2B08BF84F8458001F0CEFC01A902A82D
:1072200001F05EF9002863D101F0A4FCA36B002BF0
:1072300000F0B58001F0C0FC01F09CFC94F84530F2
:107240005DB2002D04DC11E06B1EDAB25DB26AB1F2
:10725000636A304653B101F0EFF80028F4D001F032
:1072600087F96B1EDAB25DB2002AF1D1FF2384F8F0
:10727000453001F0A1FC01F07DFC94F844305DB292
:10728000002D14DD04F1100903E06B1EDAB25DB2CB
:107290006AB12369484653B101F0CEF80028F4D012
:1072A00001F066F96B1EDAB25DB2002AF1D1FF235C
:1072B00084F8443001F080FC01F002F860E0036CD7
:1072C000002B82D04FF0500383F31188BFF36F8FF0
:1072D000BFF34F8FFEE7019B002B3FF47BAF4FF0D6
:1072E000500383F31188BFF36F8FBFF34F8FFEE717
:1072F00001F040FC94F845305DB2002D04DC11E053
:107300006B1EDAB25DB26AB1636A304653B101F006
:1073100093F80028F4D001F02BF96B1EDAB25DB2BD
:10732000002AF1D1FF2384F8453001F045FC01F03B
:1073300021FC94F844305DB2002D14DD04F11009F5
:1073400003E06B1EDAB25DB26AB12369484653B1FD
:1073500001F072F80028F4D001F00AF96B1EDAB2DD
:107360005DB2002AF1D1FF2384F8443001F024FCFF
:1073700000F0A6FF01F0FEFBA36B53B101F01CFC73
:1073800001F0F8FBA56B002D62D1019B002B7FF46F
:1073900031AF01F011FC002005B0BDE8F08301F031
:1073A0000BFC0199304600F0F7FF01F0E3FB94F885
:1073B00045305DB2002D04DC11E06B1EDAB25DB227
:1073C0006AB1636A304653B101F036F80028F4D050
:1073D00001F0CEF86B1EDAB25DB2002AF1D1FF23C4
:1073E00084F8453001F0E8FB01F0C4FB94F8443028
:1073F0005DB2002D14DD04F1100903E06B1EDAB25A
:107400005DB26AB12369484653B101F015F800280E
:10741000F4D001F0ADF86B1EDAB25DB2002AF1D102
:10742000FF2384F8443001F0C7FB00F049FF002837
:10743000A6D14FF0E0234FF08052C3F8042DBFF3E4
:107440004F8FBFF36F8F01F095FBA56B002D9CD084
:10745000226C52B1E168A36811449942E16024BFF3
:107460002168E160384614F0BDFA013DA563236947
:1074700063B901F0A1FB01208EE74FF0500383F3C5
:107480001188BFF36F8FBFF34F8FFEE704F1100039
:1074900000F0D2FF0028ECD04FF0E0234FF08052F4
:1074A000C3F8042DBFF34F8FBFF36F8FE1E700BF29
:1074B0002DE9F04184B0019100285CD0076C0446AE
:1074C00047B14FF0500383F31188BFF36F8FBFF3C1
:1074D0004F8FFEE701F058F80546002854D03D468E
:1074E00004F1240601F046FBA36B002B40F0488119
:1074F000019B002B00F03A81002D00F09D8001F0EF
:107500005BFB00F0D5FE01F035FB94F84430FF2B17
:1075100004BF002384F8443094F84530FF2B04BFA7
:10752000002384F8453001F047FB01A902A800F0D0
:10753000D7FF002835D101F01DFBA36B002B00F015
:10754000A48001F039FB01F015FB94F845305DB2E1
:10755000002D05DC74E06B1EDAB25DB2002A6FD03C
:10756000636A3046002B6BD000F066FF0028F2D033
:1075700000F0FEFFEFE74FF0500383F31188BFF3F5
:107580006F8FBFF34F8FFEE7019B002B00F0D4807D
:107590004FF0500383F31188BFF36F8FBFF34F8F0A
:1075A000FEE701F0E7FA94F845305DB2002D04DC07
:1075B00011E06B1EDAB25DB26AB1636A304653B154
:1075C00000F03AFF0028F4D000F0D2FF6B1EDAB2D0
:1075D0005DB2002AF1D1FF2384F8453001F0ECFAC6
:1075E00001F0C8FA94F844305DB2002D14DD04F1C6
:1075F000100803E06B1EDAB25DB26AB1236940463F
:1076000053B100F019FF0028F4D000F0B1FF6B1E59
:10761000DAB25DB2002AF1D1FF2384F8443001F0E0
:10762000CBFA00F04DFE01F0A5FAA36B002B7CD045
:1076300001F0C2FA012555E702A800F045FF5EE718
:10764000FF2384F8453001F0B7FA01F093FA94F87B
:1076500044305DB2002D10DD04F1100803E06B1E14
:10766000DAB25DB24AB12369404633B100F0E4FEBC
:107670000028F4D000F07CFFF1E7FF2384F84430C9
:1076800001F09AFA00F01CFED4E701F095FA2368A5
:10769000002B62D00199304600F07EFE01F06AFABC
:1076A00094F845305DB2002D04DC0DE06B1EDAB2BB
:1076B0005DB24AB1636A304633B100F0BDFE0028C6
:1076C000F4D000F055FFF1E7FF2384F8453001F0D6
:1076D00073FA01F04FFA94F844305DB2002D10DDDA
:1076E00004F1100803E06B1EDAB25DB24AB12369FF
:1076F000404633B100F0A0FE0028F4D000F038FF7F
:10770000F1E7FF2384F8443001F056FA00F0D8FD89
:1077100000288FD14FF0E0234FF08052C3F8042DA2
:10772000BFF34F8FBFF36F8F84E701F045FA2FB996
:10773000384604B0BDE8F0810746D1E601F01AFAF8
:10774000616A19B1236B1968C1F10701A06800F0E3
:10775000D7FF002701F030FAEAE701F00BFAA06842
:1077600000F022FF074601F027FA93E797B14FF0A8
:10777000500383F31188BFF36F8FBFF34F8FFEE782
:107780002268013BA363CAB1236933B901F014FA3B
:107790000127CDE701F010FACAE704F1100000F06C
:1077A0004BFE0028F2D04FF0E0234FF08052C3F898
:1077B000042DBFF34F8FBFF36F8FE7E701F000F8A1
:1077C000A060E1E7A8B170B586680D46044600F0F8
:1077D000D5FE864208D029462046FFF769FE10B143
:1077E000E3680133E36070BDE36801200344E360B4
:1077F00070BD4FF0500383F31188BFF36F8FBFF359
:107800004F8FFEE72DE9F84310B30E4617460446A6
:1078100091B101F0E3FAEFF311894FF0500383F3D4
:107820001188BFF36F8FBFF34F8FA56BCDB928467B
:1078300089F31188BDE8F883036C002BE9D04FF081
:10784000500383F31188BFF36F8FBFF34F8FFEE7B1
:107850004FF0500383F31188BFF36F8FBFF34F8F47
:10786000FEE794F84480226C4FFA88F852B1E16840
:10787000A36811449942E16024BF2168E160304669
:1078800014F0B0F8013DB8F1FF3FA56309D008F14D
:1078900001035BB284F84430012089F31188BDE80C
:1078A000F8832369002BF7D004F1100000F0C4FD29
:1078B0000028F1D0002FEFD001203860B8E700BFDA
:1078C00058B110B5044682B001F054F9A06B019094
:1078D00001F072F9019802B010BD4FF0500383F32C
:1078E0001188BFF36F8FBFF34F8FFEE708B1806B36
:1078F00070474FF0500383F31188BFF36F8FBFF3CE
:107900004F8FFEE700000000F0B1214B5A68904213
:1079100025D0DA6890422CD05A6990422BD0DA698F
:1079200090422AD05A6A904229D0DA6A90421ED0F8
:107930005A6B904225D0DA6B904208BF07220FD0D5
:1079400090F846304BB170474FF0500383F31188E5
:10795000BFF36F8FBFF34F8FFEE701F029BB00220B
:107960009FED097B03EBC20383ED007BE8E7052273
:10797000F6E70122F4E70222F2E70322F0E704220D
:10798000EEE70622ECE700BF000000000000000068
:10799000505500202DE9F843044601F0EBF8344A35
:1079A000344D1368013313602B68002B32D0324EF4
:1079B00033683BB3E36A314F3148324902680132E0
:1079C0000260086801229A40024303EB83030A60C5
:1079D00007EB8300211DFEF747FF01F0EDF8336848
:1079E00073B12A68E36AD26A9A4209D24FF0E0235F
:1079F0004FF08052C3F8042DBFF34F8FBFF36F8F4A
:107A0000BDE8F8832A68E36AD26A1C4F9A4298BF9D
:107A10002C60D1E72C601368012B03D0E36A174F69
:107A2000154EC9E7154F3E4607F18C08304614360F
:107A3000FEF70AFFB045F9D1DFF86090DFF860800B
:107A40000D4E4846FEF700FF4046FEF7FDFE0E488D
:107A5000FEF7FAFE0D48FEF7F7FE0D48FEF7F4FEBE
:107A60000C4BC3F800900C4BC3F80080E36AA3E70B
:107A70002856002090550020845600209C55002058
:107A80003456002038560020705600209C560020A6
:107A90008856002094550020985500203C56002020
:107AA00050560020F8B51B4B1B4E1C68336805462A
:107AB000181D0F46FEF700FF40B933681749DB6A0F
:107AC00001229A400B6823EA02030B606B1C17D05B
:107AD000336864195C6007D3114B18683168BDE8DE
:107AE000F8400431FEF7D0BE0E4B186831680431FF
:107AF000FEF7CAFE0C4B1A68A24288BF1C60F8BD94
:107B0000002FE5D031680948BDE8F8400431FEF7A0
:107B1000ABBE00BFB0560020905500203856002064
:107B20009855002094550020645600208856002067
:107B300080B5234D234F244EDFF890804FF0E02A8C
:107B40004FF080592B685BB301F014F8FB68DC68D8
:107B5000201DFEF7B1FE3368013B33602B68013B0B
:107B60002B6001F029F804F1500013F073FE94F833
:107B7000A13063B1012B1ED0022BE3D04FF0500394
:107B800083F31188BFF36F8FBFF34F8FFEE7206B36
:107B900001F00EFA204601F00BFA2B68002BD3D12E
:107BA000D8F80030012BCDD9CAF8049DBFF34F8F10
:107BB000BFF36F8FC6E7204601F0FAF9C2E700BFB6
:107BC0002C5600209C560020285600209C55002052
:107BD0002DE9F04F4A4B1D68013583B01D60002D23
:107BE00045D0484B01931B689D424DD3464EDFF86C
:107BF0002C813368DFF828911C68002C7AD0434F21
:107C000000244FF0010A24E00091FEF755FEDBF856
:107C1000282000990BF1180012B1FEF74DFE0099D3
:107C2000DBF82C003B680AFA00F200EB80001A43F4
:107C300008EB80003A60FEF717FED9F800203068A4
:107C4000DBF82C10D26A0368914228BF0124002B74
:107C500050D03368DB68D3F80CB0DBF804200BF1AC
:107C6000040195420846CFD2019B1A6011E0264BD1
:107C70001A6812680AB34FF0500383F31188BFF3F8
:107C80006F8FBFF34F8FFEE7DFF89080DFF89090A3
:107C90000024D9F800301E49DB6A03EB83039B0004
:107CA00058F803200B68022A28BF0124002B0CBFC0
:107CB0002046012003B0BDE8F08F164A186811680D
:107CC0001960154910600A6801320A601A68126862
:107CD0003AB90C4B01931A464FF0FF331360134629
:107CE00081E71B68074ADB680192DB685B68136009
:107CF000134678E7019A4FF0FF331360C9E700BFDE
:107D0000B0560020645600209455002038560020BC
:107D1000B456002098550020685600209C5500203D
:107D2000905500202DE9F04F454C83B000F022FF24
:107D30002368013B23602368002B67D1414B1B68FC
:107D4000002B63D0DFF818B1DBF80030002B73D0C4
:107D50003D4B3E4DDFF80C813D4F01930126DBF892
:107D60000C30D3F80CA00AF104090AF11800FEF750
:107D7000A3FD4846FEF7A0FDDAF82C002A6806FAB3
:107D800000F300EB80001343494608EB80002B60B2
:107D9000FEF76AFD3B68DAF82C20DB6A9A423DD395
:107DA000019B1E60DBF80030002BD8D1294B1A68EC
:107DB0001268002A3BD01A68274BD268D2685268F2
:107DC0001A60264E356895B1012706E0FFF700FFDF
:107DD00008B1019B1F60013D08D02368002BF5D03E
:107DE0003368013D03F101033360F6D13560019B37
:107DF0001B685BB14FF0E0234FF08052C3F8042DB5
:107E0000BFF34F8FBFF36F8F012000E00020019080
:107E100000F0D2FE019803B0BDE8F08FDBF800302F
:107E2000002B9CD10B4B1A681268002AC3D10A4B55
:107E30004FF0FF321A60C4E7034B0193C1E700BF64
:107E40003056002028560020B45600203856002016
:107E50009055002094550020645600206C56002058
:107E6000705600209C5500202DE9F04184B0DDE9DA
:107E70000B54C5B174B10646A42003900398A428FE
:107E80001AD04FF0500383F31188BFF36F8FBFF305
:107E90004F8FFEE74FF0500383F31188BFF36F8FCE
:107EA000BFF34F8FFEE74FF0500383F31188BFF30A
:107EB0006F8FBFF34F8FFEE702F18042013A05EB6F
:107EC0008202256322F00705039A6564022284F882
:107ED000A120002979D00A7884F83420002A3BD0E8
:107EE0004A7884F83520002A36D08A7884F83620FB
:107EF00092B3CA7884F8372072B30A7984F83820AC
:107F000052B34A7984F8392032B38A7984F83A2016
:107F100012B3CA7984F83B20F2B10A7A84F83C2083
:107F2000D2B14A7A84F83D20B2B18A7A84F83E20F0
:107F300092B1CA7A84F83F2072B10A7B84F840205B
:107F400052B14A7B84F8412032B18A7B84F84220C6
:107F500012B1CA7B84F84320002284F843200A9F90
:107F60000193062F28BF06274FF00008E762A76499
:107F7000201DC4F84C80FEF773FCC7F1070704F11D
:107F80001800FEF76DFCA761C4F89C80414624618F
:107F9000646284F8A0804C2204F1500013F02CFCA1
:107FA0000B4F019B67651A4607F16803D0373146CE
:107FB000A3652846E76500F0B5FD20602046FFF781
:107FC000E9FC204604B0BDE8F08184F83410C6E72F
:107FD000AC1D01202DE9F8439500804628460E4649
:107FE000994600F029FF002800F08C800746A42065
:107FF00000F022FF0446002800F08880043D3D4444
:1080000025F0070500230763456480F8A130002EA2
:1080100000F08280337880F83430002B3BD07378C6
:1080200080F83530002B36D0B37880F8363093B3F3
:10803000F37880F8373073B3337980F8383053B33E
:10804000737980F8393033B3B37980F83A3013B3A9
:10805000F37980F83B30F3B1337A80F83C30D3B118
:10806000737A80F83D30B3B1B37A80F83E3093B183
:10807000F37A80F83F3073B1337B80F8403053B1EE
:10808000737B80F8413033B1B37B80F8423013B159
:10809000F37B80F84330002384F84330089E062E9B
:1080A00028BF06260027E662A664201DE764FEF7C7
:1080B000D7FBC6F1070604F11800FEF7D1FBC4F8A0
:1080C0009C7039464C22A6612461646284F8A070D9
:1080D00004F1500013F090FB114B6365284603F147
:1080E0006805D033E3654A464146A56500F01AFDB0
:1080F000099B206003B11C602046FFF74BFC012068
:10810000BDE8F8834FF0FF30BDE8F883384600F053
:108110004FFF4FF0FF30F3E780F83460BEE700BF59
:10812000AC1D012010B550B94FF0E0234FF0805244
:10813000C3F8042DBFF34F8FBFF36F8F10BD104CEA
:10814000216841B14FF0500383F31188BFF36F8F63
:10815000BFF34F8FFEE7236801332360FFF7A2FCD4
:10816000236843B94FF0500383F31188BFF36F8F37
:10817000BFF34F8FFEE7FFF7D5FD0028D4D010BD29
:108180003056002070B584B002AA002401A96846C8
:10819000CDE90044F8F79AFFDDE90132009DBBB15B
:1081A0006DB1A42103910399A4291AD04FF0500373
:1081B00083F31188BFF36F8FBFF34F8FFEE74FF04C
:1081C000500383F31188BFF36F8FBFF34F8FFEE728
:1081D0004FF0500383F31188BFF36F8FBFF34F8FBE
:1081E000FEE702F18042013A03EB820222F0070629
:1081F0002B630222264B85F8A120281D6B63C5E95D
:1082000012446E6485F8384085F84340EC62039B65
:10821000FEF726FB05F11800FEF722FB0723C5F841
:108220009C402146AB612D616D6285F8A0404C22D7
:1082300005F1500013F0E0FA164B6B6503F168028C
:10824000D0331549AA65EB652246304600F06AFC3A
:1082500028602846FFF79EFB4FF0500383F31188F8
:10826000BFF36F8FBFF34F8F0C4A0D4B0D491B6847
:108270004FF0FF3010600C4A012010600B4A503361
:108280000B60146004B0BDE8704000F005BD00BF95
:1082900049444C45AC1D0120317B00086456002048
:1082A00090550020BC00002084560020B0560020CD
:1082B000024A136801331360704700BF3056002034
:1082C000064B1B6843B94FF0500383F31188BFF38B
:1082D0006F8FBFF34F8FFEE7FFF724BD30560020AE
:1082E000014B1868704700BFB056002008B500F079
:1082F00075FD014B186808BDB0560020054B1B6882
:108300000BB9FFF765BC044A136801330020136002
:10831000704700BF305600206C560020184B1B6879
:108320001BB1184B01221A6070471649164A0B60A0
:108330001368B3FA83F3DBB2C3F11F0303EB8303C8
:10834000124A990002EB8303505840B94FF0500392
:1083500083F31188BFF36F8FBFF34F8FFEE7586829
:108360000831406858600A44904204BF4068586031
:10837000074BC2681A601B68064A50331360704787
:1083800030560020B4560020385600209C5500205E
:1083900090550020BC00002020B370B51F4D0C4646
:1083A00029681831FEF770FA1D4B1E6828680430E2
:1083B000FEF782FA40B92B681A49D86A0B68012285
:1083C000824023EA02030B60631C14D02B68A419BB
:1083D0005C6017D3144B18682968BDE870400431FD
:1083E000FEF752BA4FF0500383F31188BFF36F8F3B
:1083F000BFF34F8FFEE729680C48BDE87040043199
:10840000FEF732BA0A4B186829680431FEF73CFAC5
:10841000084B1A68944238BF1C6070BD905500200C
:10842000B05600203856002098550020885600206D
:10843000945500206456002070B5C368DC6882B093
:10844000002C2CD004F118052846FEF735FA184BFD
:108450001B687BB117482946FEF706FA164BE26AFD
:108460001B68DB6A9A4285BF144B0120002018600C
:1084700002B070BD211D124D01910846FEF71CFA95
:10848000E36A2E680F48019901229A4003EB8303A7
:10849000324300EB83002A60FEF7E6F9DEE74FF097
:1084A000500383F31188BFF36F8FBFF34F8FFEE745
:1084B000305600207056002090550020B456002001
:1084C000385600209C550020034A044B12681B6854
:1084D000C0E90023704700BF68560020B056002056
:1084E00028B3F0B50D4683B0C1B1044600F042FB9D
:1084F0002B681D4A581C116830D0DFF870C0D4E9D1
:108500000060DCF80070BE421AD0884218D8012002
:10851000019000F051FB019803B0F0BD4FF0500303
:1085200083F31188BFF36F8FBFF34F8FFEE74FF0D8
:10853000500383F31188BFF36F8FBFF34F8FFEE7B4
:10854000A1EB000E73450BD95B1ADCF80010126822
:1085500003442B600020C4E90012D9E70020D7E7CC
:1085600000232B600120D3E7B0560020685600207E
:10857000014B01221A607047B4560020014B186865
:10858000704700BF90550020054B1B6833B1054B69
:108590001868B0FA80F04009400070470120704729
:1085A0008456002030560020F0B5044683B0C8B190
:1085B000224DC36A2A68D26A934215D28269002A80
:1085C00004DB2A68D26AC2F1070282611C4E62692A
:1085D00003EB830306EB83039A420ED02B68DB6A1E
:1085E000E362012003B0F0BD2B68806CDB6A984227
:1085F0002CBF0020012003B0F0BD211D08460191D1
:10860000FEF75AF901990F4A30B9E76A1368012059
:10861000B84023EA000313602B681568D86AE0624B
:10862000012404FA00F300EB80002B4306EB8000EA
:108630001360FEF719F92046D4E700BF90550020DB
:108640009C5500203856002020B3F0B5294B1B68FC
:10865000834283B0044608D04FF0500383F311885F
:10866000BFF36F8FBFF34F8FFEE7DB6C4BB1C16A77
:10867000826C013B9142C36400D06BB1002003B017
:10868000F0BD4FF0500383F31188BFF36F8FBFF33A
:108690004F8FFEE700207047011D08460191FEF74D
:1086A0000BF90199A0B11448144AA36C1668E3624F
:1086B0000125C3F10707A76105FA03F403EB830360
:1086C00000EB830034431460FEF7CEF82846D6E76B
:1086D000E36A094803EB8302920082580AB1074A11
:1086E000E3E7064A01259D40136823EA050313606A
:1086F000DBE700BF905500209C5500203856002035
:10870000002843D030B5C36C83B0044653B1806CAD
:10871000E26A814238BF01468A4201D0012B0AD069
:1087200003B030BD4FF0500383F31188BFF36F8F58
:10873000BFF34F8FFEE71F4B1B68A34227D0A369EF
:10874000E162002BA8BFC1F107011B4DA8BFA161C9
:1087500002EB8202616905EB82039942E0D1211D9F
:1087600008460191FEF7A8F80199C8B1E06A134ADA
:1087700001238340146800EB8000234305EB800055
:10878000136003B0BDE83040FEF76EB870474FF09D
:10879000500383F31188BFF36F8FBFF34F8FFEE752
:1087A000064AE06A14680123834024EA0304146043
:1087B000E0E700BF905500209C550020385600206F
:1087C000044B1A681AB11968CA6C0132CA64186875
:1087D000704700BF905500202DE9F041254C82B034
:1087E000154607460E46984600F0C4F9226892F8EE
:1087F000A020022A0DD02368D3F89C2022EA070289
:10880000C3F89C202368012183F8A010B8F1000F61
:1088100019D100F0D1F900F0ADF91DB12368D3F8FA
:108820009C302B60236893F8A030022B19D00020D5
:1088300023680190002283F8A02000F0BDF9019880
:1088400002B0BDE8F0814046FFF72CF94FF0E0237D
:108850004FF08052C3F8042DBFF34F8FBFF36F8FDB
:10886000D7E72268D2F89C3023EA06030120C2F839
:108870009C30DDE79055002020B3F0B51E4683B054
:108880000F461546044600F075F916B1D4F89C3031
:10889000336094F8A0600223F6B284F8A030042D6F
:1088A00057D8DFE805F007181E050300022E3DD05B
:1088B000C4F89C70012E1AD0012600F07DF93046D4
:1088C00003B0F0BD4FF0500383F31188BFF36F8FF7
:1088D000BFF34F8FFEE7D4F89C303B43C4F89C3085
:1088E000E8E7D4F89C300133C4F89C30E2E7211D5E
:1088F0001E4D01910846FDF7DFFFE36A2F681C4813
:10890000019906FA03F203EB83033A4300EB830079
:108910002A60FDF7A9FFA36A53B14FF0500383F318
:108920001188BFF36F8FBFF34F8FFEE70026C4E7B8
:10893000104BE26A1B68DB6A9A42BDD94FF0E02314
:108940004FF08052C3F8042DBFF34F8FBFF36F8FEA
:10895000B3E7D4F89C300133ACD04FF0500383F32D
:108960001188BFF36F8FBFF34F8FFEE7385600209B
:108970009C5500209055002078B32DE9F04182B03D
:108980000F4615461E46044600F028FAEFF31188FC
:108990004FF0500383F31188BFF36F8FBFF34F8FF6
:1089A00016B1D4F89C30336094F8A0600223F6B27C
:1089B00084F8A030042D5DD8DFE805F007181E0507
:1089C0000300022E29D0C4F89C70012E1AD0012079
:1089D00088F3118802B0BDE8F0814FF0500383F3B3
:1089E0001188BFF36F8FBFF34F8FFEE7D4F89C3031
:1089F0003B43C4F89C30E8E7D4F89C300133C4F81A
:108A00009C30E2E7A36A53B14FF0500383F311881F
:108A1000BFF36F8FBFF34F8FFEE70020D8E71C4BEB
:108A20001B680BBB211D08460191FDF745FFE06A5D
:108A3000184B194A0199864000EB800002EB800038
:108A40001A6816431E60FDF70FFF144BE26A1B689D
:108A5000DB6A9A42BBD9089B13B11A460123136003
:108A60000F4B01201860B3E70E4804F11801FDF721
:108A7000FBFEEAE7D4F89C300133A6D04FF0500358
:108A800083F31188BFF36F8FBFF34F8FFEE700BFF3
:108A900030560020385600209C550020905500206C
:108AA000B45600207056002008480068006880F323
:108AB00008884FF0000080F3148862B661B6BFF3F7
:108AC0004F8FBFF36F8F00DF00BF000008ED00E0A5
:108AD000DFF80C00016841F470010160704700008C
:108AE00088ED00E00E4B1B6882B00022013301923A
:108AF00008D04FF0500383F31188BFF36F8FBFF39B
:108B00004F8FFEE74FF0500383F31188BFF36F8F51
:108B1000BFF34F8F019B002BFCD002B0704700BF0A
:108B20002000002010B44FF08073074C40F8043C44
:108B300021F001016FF0020340E9034140E90932ED
:108B40005DF8044B44387047E58A000800000000D7
:108B5000074B19680868B0E8F04F80F30988BFF345
:108B60006F8F4FF0000080F311887047AFF30080E3
:108B7000905500204FF0500383F31188BFF36F8F9F
:108B8000BFF34F8F0B4A13680133012B136000D0E2
:108B900070474FF0E023D3F8043DDBB2002BF7D051
:108BA0004FF0500383F31188BFF36F8FBFF34F8FE4
:108BB000FEE700BF20000020084A136843B94FF0C9
:108BC000500383F31188BFF36F8FBFF34F8FFEE71E
:108BD000013B13600BB983F311887047200000201C
:108BE000EFF30980BFF36F8F154B1A681EF0100F5B
:108BF00008BF20ED108A20E9F04F10602DE9090030
:108C00004FF0500080F31188BFF34F8FBFF36F8F89
:108C1000FFF784FB4FF0000080F3118809BC19684E
:108C20000868B0E8F04F1EF0100F08BFB0EC108AD3
:108C300080F30988BFF36F8F704700BFAFF30080E8
:108C40009055002008B54FF0500383F31188BFF30F
:108C50006F8FBFF34F8FFFF751FB28B14FF0E02329
:108C60004FF08052C3F8042D002383F3118808BD10
:108C70004FF0E02200230649136193610B68054918
:108C8000A1FB03139B090720013B5361106170474F
:108C900000000020D34D62104FF0E023494AD3F882
:108CA000001D914243D0D3F8002D474B9A4235D056
:108CB00070B5464B46481A78464C84B0FF21D2B274
:108CC000029219701B78DBB28DF807309DF80730DF
:108CD0009DF8072003F05003072103701006216060
:108CE00048BF062211D59DF807305B00DBB28DF836
:108CF00007309DF807100906104602F1FF32F2D442
:108D0000032820608DF807301AD04FF0500383F30A
:108D10001188BFF36F8FBFF34F8FFEE74FF0500303
:108D200083F31188BFF36F8FBFF34F8FFEE74FF0D0
:108D3000500383F31188BFF36F8FBFF34F8FFEE7AC
:108D4000029B224A4FF0E0254FF44071DBB22160D4
:108D50001370D5F8203D204C43F47003C5F8203D36
:108D6000D5F8203D43F07043C5F8203D0026FFF7BD
:108D70007FFF2660FFF7ACFED5F8343F43F0404359
:108D8000C5F8343FFFF790FEFFF7C8FA2368039653
:108D9000013308D04FF0500383F31188BFF36F8F76
:108DA000BFF34F8FFEE74FF0500383F31188BFF3FB
:108DB0006F8FBFF34F8F039B002BFCD0002004B0BC
:108DC00070BD00BF71C20F4170C20F4100E400E0EE
:108DD000B8560020BC56002020000020EFF3058389
:108DE0000F2B0ED91149124A5B5C12789A4208D9AE
:108DF0004FF0500383F31188BFF36F8FBFF34F8F92
:108E0000FEE74FF0E0230B4AD3F80C3D126803F461
:108E1000E063934208D94FF0500383F31188BFF306
:108E20006F8FBFF34F8FFEE7704700BFF0E300E0A6
:108E3000B8560020BC5600202DE9F0410546FFF74A
:108E400037FA534A1668002E6ED0524B1F683D42C7
:108E50002ED16DB305F108046D071CBF24F0070483
:108E600008342CB3DFF844C1DCF80050A5421FD30E
:108E70004948036803E01A6822B118461346596846
:108E8000A142F8D3B34213D098460A1B58F808EB16
:108E9000C0F800E0102A29D9191948070FD04FF05F
:108EA000500383F31188BFF36F8FBFF34F8FFEE73B
:108EB000FFF706FA4FF000084046BDE8F0814A602F
:108EC000354A5C60144612689142FBD8606804EB36
:108ED000000E714549D0D1F804E001EB0E0082424A
:108EE0004FD08C420A6018BF216059682B4A106825
:108EF0006D1A854238BF1560294ACCF800503943B5
:108F00000020C3E90001136801331360FFF7D8F9AB
:108F100018F0070FD0D04FF0500383F31188BFF340
:108F20006F8FBFF34F8FFEE71E4B5E0717D11E4EAC
:108F30001946083E26F007061660184A1648154CD2
:108F40000160F31A1360194A4FF0004713600022C2
:108F500042602760C6E90022C1E9006377E7073372
:108F600023F00701104E0B46E3E7496800EB010EC2
:108F700004EB0E018A42C4F804E001D02260B4E799
:108F80002146B242ADD05068126870444860A8E7EC
:108F9000C0560020F4CB002008CC0020FCCB0020E1
:108FA00000CC0020C4560020F4CB0020F8CB0020D9
:108FB000D0B12C4A50F8043C126813420BD050F840
:108FC000081C91B14FF0500383F31188BFF36F8FEA
:108FD000BFF34F8FFEE74FF0500383F31188BFF3C9
:108FE0006F8FBFF34F8FFEE7704710B523EA020380
:108FF00082B040F8043C1C4C0190FFF759F90198ED
:10900000226850F8041C194B0A44083822601A469A
:109010001B689842FBD8546802EB040E704510D0D0
:1090200000EB010C634514D08242036018BF10604E
:109030000F4A13680133136002B0BDE81040FFF718
:109040003FB9214450188342516001D01360EFE7CB
:109050001046084C2468A342E6D0D3E900342144EA
:109060004160E1E7F4CB0020F8CB002008CC0020E1
:1090700004CC0020C05600202DE9F04182B000232E
:10908000019300297ED004460D460B6000286FD066
:1090900000F11008404616460FF062FA074618B372
:1090A00094F8243006F0040603F00303334327D07A
:1090B00001A940460FF042FA01303CD0237803F07A
:1090C000F003102B2AD0019B002B45D01A6812897F
:1090D000E66A1EB101212046B047019B2B600025A6
:1090E000284602B0BDE8F0810FF0C6FA94F90850A6
:1090F00027720FF0CDFA002DF2D16FF00A05EFE7DD
:1091000094F90830002BD3D1226A01A940460FF010
:10911000F3F90130D2D16FF00205E1E701980DF1CA
:10912000030101F017F800B39DF9035015F10F0F7B
:1091300008BF0025D4E70FF09FFA94F908500023E8
:1091400023720FF0A5FA002DCAD194F82430DB0762
:10915000D3D46FF00605C3E70F4B1049104840F217
:10916000912212F09FFA019BB0E7019B1A89AFE7A9
:10917000094B0C490A4840F24A2212F093FA6FF068
:109180000F05ADE7044B084905484FF4127212F081
:1091900089FA6FF00F05A3E784F30108F4F30108DF
:1091A00008F30108D8F30108B8F3010870B50D46BB
:1091B0008AB0114601F04CF8044670B100F10C067B
:1091C0000190324622488DF80C5001A902F070FA45
:1091D0009DF80830184340B210B920460AB070BD5F
:1091E00063682BB11B4B1C491C48A32212F05AFA8E
:1091F00004F1100528460FF0B3F910B304F1140080
:109200000FF0AEF9B0B930460FF0F2F958B1304670
:109210000FF0EAF928460FF05BF92146072003F02A
:1092200053F80024D9E70B4B0D490C48A92212F042
:1092300039FAECE7074B0B490848A62212F032FA3C
:10924000E1E7044B08490548A42212F02BFAD5E7C0
:10925000B1A1000884F3010800F4010808F3010833
:1092600060F401083CF4010824F4010830B5044618
:109270008BB0C8B10190FCF7A7FF019A03460C32EE
:109280000B48049301A902F013FA054610B12846D1
:109290000BB030BD9DF90850002DF8D1204601F0EB
:1092A0001FF828460BB030BD054628460BB030BD30
:1092B00045A4000870B58AB040B30D46E1B116462A
:1092C00082B1044604F10C021548019401A9CDE9CC
:1092D00003568DF8143002F0EBF908B99DF9080037
:1092E0000AB070BD0F4B104910484FF48A7212F04B
:1092F000D9F96FF00F00F3E70A4B0D490B4840F224
:10930000131212F0CFF96FF00F00E9E7054B09498E
:1093100006484FF4897212F0C5F96FF00F00DFE7CD
:10932000E9A6000884F30108BCF4010808F3010869
:109330009CF401087CF4010800B58BB0A8B19446F8
:109340000F4AADF810C00346002908BF114603912B
:109350000C48019303F10C0201A902F0A9F908B924
:109360009DF908000BB05DF804FB074B074908485E
:109370004FF49C7212F096F96FF00F00F2E700BF05
:109380007821020861A5000884F30108DCF40108D3
:1093900008F3010810B58AB098B1027802F0F00223
:1093A000102A03460DD10C460B48019303F10C0221
:1093B00001A9039402F07CF908B99DF908000AB0EC
:1093C00010BD064B0649074840F2B52212F06AF973
:1093D0006FF00F00F3E700BFD9A5000884F3010880
:1093E000F8F4010808F30108F0B593B0002857D04D
:1093F000037803F0F003102B044651D110300F46D0
:1094000016460FF0ADF8002865D094F9242094F8A2
:109410002430002A1DDB324639462046FFF72CFE59
:10942000054698B932073F680FD4002F36D03A89E5
:10943000237803F0F003102B50D102922C480094B3
:1094400004F10C02694602F033F9E7B1284613B083
:10945000F0BD03F07F0384F82430E36A1BB10022DF
:10946000012120469847666826BB0FF005F994F95C
:10947000085026720FF00CF9002D08BF6FF00D0593
:10948000284613B0F0BDF306E7D594F8243063F016
:109490007F036FF0060584F82430D7E70122C7E781
:1094A000144B1549154840F2253212F0FBF86FF0C5
:1094B0000F05CBE701238DF82C300994FCF784FECF
:1094C000099A03460C3209A90D480C936FF00E055A
:1094D00002F0EEF8BAE76FF00A05B7E7054B064968
:1094E000064840F2A72212F0DDF8002FAED1CAE7FD
:1094F000D9A5000884F30108F8F4010808F301086D
:109500007DA700082DE9F04182B000287BD00378C8
:1095100003F0F003102B044675D000230D46019391
:1095200000297AD000F110080B60404616460FF073
:1095300017F8074618B394F8243006F0040603F031
:109540000303334327D001A940460EF0F7FF013053
:109550002FD0237803F0F003102B3BD0019B002B7E
:1095600045D01A681289E66A1EB101212046B0472B
:10957000019B2B600025284602B0BDE8F0810FF06A
:109580007BF894F9085027720FF082F8002DF2D181
:109590006FF00A05EFE794F90830002BD3D1226A67
:1095A00001A940460EF0A8FF0130D2D16FF00205AC
:1095B000E1E70FF061F894F90850002323720FF0EF
:1095C00067F8002DD7D194F82430DB07E0D46FF092
:1095D0000605D0E701980DF1030100F0BBFD78B15D
:1095E0009DF9035015F10F0F08BF0025C3E7104B7D
:1095F0001049114840F2912212F054F8019BB0E753
:10960000019B1A89AFE70A4B0C490B484FF4537280
:1096100012F048F86FF00F05ADE7054B0849064812
:109620004FF4127212F03EF86FF00F05A3E700BF7F
:1096300084F30108F4F3010808F301081CF501089C
:10964000B8F3010810B58AB070B103460C460B4858
:10965000019303F10C0201A9039402F029F808B95F
:109660009DF908000AB010BD054B0649064840F2B6
:10967000B23212F017F86FF00F00F3E799A5000867
:1096800084F3010848F5010808F30108F0B58DB02E
:10969000CDE90112129C002863D01546027802F031
:1096A000F002102A50D190F8241003F0040201F0C7
:1096B000020151EA020720D0C269002C4ED0002DD1
:1096C0004FF001071ED021DB8DF8283000230793CF
:1096D000099301AB0593012303900895ADF8183069
:1096E00062BB0B9200F10C0203A9234801F0E0FFDA
:1096F000064678B130460DB0F0BDC269002ADCD113
:10970000002DE0D1002630460DB0F0BD34B36FF02F
:109710000045D9E79DF91060002EEBD10CB1099BF3
:109720002360002FEED1099B9D42EBD0134B1449CF
:1097300014484FF4866211F0B5FFDBE7FCF744FDF7
:1097400003460B930398CDE70C4B0F490D4840F2AD
:10975000EF3211F0A7FF6FF00506CBE76FF00506BB
:10976000C8E7064B0949074840F2EE3211F09AFF6C
:109770006FF00F06BEE700BF15A6000884F30108CE
:10978000A4F5010808F3010880F5010864F5010853
:1097900038B5044648B10EF06FFF94F90850002325
:1097A00023720EF075FF284638BD0546284638BDA1
:1097B0002DE9F0470446BDF8208016461F460D46A9
:1097C00079B3002C35D06368AB4205D0224B2349D6
:1097D0002348EE2211F066FF04F1100948460EF00E
:1097E000BFFEC8B1062002F00FFD0546A0B1C0E9DA
:1097F000006607B13F68AF602946A5F80C8048466F
:1098000036890EF06FFE0146F0B9E36A0BB33246BB
:109810002046BDE8F04718473046BDE8F04703F062
:109820002DB90D4B0F490E48E52211F03BFF002CDE
:10983000C9D1094B0C490A48E62211F033FF3046E2
:10984000BDE8F04703F01AB92846BDE8F04701F03B
:1098500003B8BDE8F08700BFC8F5010840F601086D
:1098600008F30108FCF5010820F601082DE9F04F86
:1098700083B007460191002800F020817B78012BFE
:1098800006D09E4B9E499F4840F2746211F00AFF39
:10989000BB6A002B00F01A817B68002B00F0068168
:1098A000BA6AD2E90531994280F0DE809389002BB3
:1098B00000F0D18092F81C8097F82430F96903F009
:1098C000020308F0040003430093002940F0B38032
:1098D00090681369DFF824B2DFF840A2DFF8249221
:1098E0000146D1E9006C7868ACEB0305B5F5803F23
:1098F000B0F864102ABF4FF6FF74ACB248F002080B
:109900008C421E4405D9009C002C57D000297AD0E7
:109910000C4623449C4548D34FF6FF739C4240D0ED
:10992000ADB2A5423BD1BB6A9B89012B37D948F028
:109930000208012543462246314606F05BFE90B1FF
:10994000431CDBB2012B06463CD9BA6A019B106866
:1099500016710024BC627C70002B40F08E8018468B
:1099600003B0BDE8F08FBA6A9369916823449361AC
:10997000136923444C681361A34203D0002DB0D176
:10998000064621E09489013CA4B29481002CF5D0D4
:109990000831916010610346002DA2D1F0E7002547
:1099A000C8E7B5F5803FC2D2BAE75B4640F2A36292
:1099B0005146484611F076FE7868ADE748F0020857
:1099C0000C46A6E74FF0FF36009B002B5CD17B686E
:1099D000B3F86420B2F5866F1ED3B3F86630042B5B
:1099E0001AD8002E7AD1BB6A7868D3E905329A4238
:1099F0001AD0009BC3B907F009FD0646301DA4D05C
:109A00004FF0FF30ACE7D2E90523002B0CBF6FF01D
:109A10000606002693423CD3FB6A002BE1D00022CD
:109A2000032138469847DCE707F0F0FC011DBA6ACD
:109A30008CD106468AE7FCF7C7FBBA6AFB69116A54
:109A4000401A9842FFF644AF9369002B0CBF6FF0A9
:109A5000060600267AE740F27962284B2A4929480F
:109A600011F020FEBA6A25E740F27762234B2749BE
:109A7000244811F017FEBA6A18E70C300EF0B0FD5A
:109A8000204603B0BDE8F08FBB6AD3E905329A42A5
:109A90009DD2FB6A1BB1002203213846984797F8F4
:109AA000243043F0100387F824309AE7134B184909
:109AB000144840F2766211F0F5FDF1E60F4B1549BE
:109AC000104840F2736211F0EDFDD7E60B4B1249DE
:109AD0000C4840F2756211F0E5FDDDE6721C7FF482
:109AE00034AF786807F092FC031D06463FF42DAFB3
:109AF000009B002B84D0BA6AA6E700BFC8F5010816
:109B000070F6010808F3010804F70108C4F601081B
:109B1000ACF6010860F6010890F601082CF7010880
:109B20002DE9F84F0F460446002800F0D88023782E
:109B300003F0F003102B06D0A94BAA49AA4840F223
:109B4000A33211F0AFFD6378042B06D0A44BA749D4
:109B5000A5484FF4697211F0A5FD6368002B00F071
:109B6000C680A36A002B00F0CD801B7A6668032BA9
:109B700003F0010803F002095ED0B8F1000F05D030
:109B8000337D5A1F012A57D9082B55D0B9F1000F40
:109B900035D1337D012B00F09D80B8F1000F40F0EE
:109BA00095804A464146304604F00AFD05460028A5
:109BB00065D06B1C4FF0000B53D1D4F81CA044F6B9
:109BC0002063BAF1000FD8BF9A46FCF7FDFAA26AEB
:109BD000D368C01A5045C0F2D980BBF1000F40F0E5
:109BE000A7801568FF2313710C35C4F828B084F8DA
:109BF00001B0002F3FD100252846BDE8F88F718BBA
:109C000011F0100557D00021304604F065F8337D7F
:109C1000012B18D0B8F1000F40F0D9800021304658
:109C200004F07AF800221146304604F0B3F800211F
:109C3000304604F08DF80AE00021304604F04CF87C
:109C4000337D012B67D10021304604F09DF830466A
:109C500004F004FE054600287CD06B1C4FF0010B7D
:109C6000ABD0A36A1A681D71002302F10C05A36230
:109C70006370002FBFD028460EF0B2FCBBE7A36A8A
:109C800018711B68A062607003F10C05B8F1000F39
:109C900006D0E36A002BACD000221146204698473C
:109CA000B9F1000FA5D0E36A002BA2D00022204614
:109CB000022198479DE7337D012B62D0B8F1000F58
:109CC00052D14146304604F027F86AE7494630460B
:109CD00004F006F84946304604F056F861E7404B78
:109CE0004349414840F2A23211F0DCFC1FE73C4BF3
:109CF00040493D4840F2A53211F0D4FCA36A002B44
:109D00007FF433AF364B3C49374840F2A63211F06E
:109D1000C9FCA36A29E70021304603F0E1FF0021D6
:109D2000304604F031F8B9F1000F7FF477AF79E7EE
:109D3000304604F0DFF9A36A1D6800221A710C3561
:109D4000E36A0022A2626270626043B1042120468D
:109D500098479BE7A36A1D6818710C35F0E7B8F1C6
:109D6000000F7FF446AF9BE72946304603F0B8FF6B
:109D70002946304604F008F82946304603F0CCFF67
:109D80000FE72946304603F0FFFF0AE7337D012B3A
:109D900010D0B9F1000F15D101223046174903F058
:109DA000F9FF3046164903F0D3FF2146304603F051
:109DB00093FF21E70A4B13490B4840F2414211F04F
:109DC00071FCE6E71049304603F0A6FFE4E73046B1
:109DD000002103F085FF0021304603F0D5FF1DE789
:109DE000C8F5010868F7010808F3010888F70108B9
:109DF00058F70108ACF7010890F601080D9E00081D
:109E00006D9F0008C0F70108D9A0000838B50446C6
:109E100018B3617801291CD0042926D094F8243085
:109E2000DA0614D5626892B1B2F86410B1F5866FA3
:109E30000DD3B2F86620042A09D8E56A23F010038E
:109E400084F824301DB1002202212046A8470020BA
:109E500038BD2046FFF70AFDE0E7064B06490748F4
:109E60004FF4B57211F01EFCD3E701212046FFF735
:109E700057FED3E7C8F5010860F6010808F30108AA
:109E80002DE9F041054616461C460F46002938D0FC
:109E9000002D3FD0002C4FD16B68BB4206D02C4B1D
:109EA0002C492D4840F2351211F0FCFB05F1100849
:109EB00040460EF055FB044688B1AEB137893146B5
:109EC00040460EF00FFB044600283DD1EB6A3BB143
:109ED00001463A46284698472046BDE8F08136B903
:109EE00000242046BDE8F0811C4E0027E7E73189B9
:109EF000384603F069FB304602F0C0FD2046BDE85D
:109F0000F081134B164914484FF4967211F0CAFBB6
:109F1000002DBFD10E4B13490F4840F22D1211F006
:109F2000C1FB34B10A4B10490B484FF4977211F042
:109F3000B9FB6FF00504CFE7054B0B4906484FF41A
:109F4000977211F0AFFBA7E74FF0FF34C4E700BFF3
:109F5000C8F5010828F8010808F30108F5F9010817
:109F6000E4F7010808F8010848F801082DE9F04174
:109F70000D46044600287DD00EF07EFB94F8243078
:109F80006778257243F00103002684F82430666068
:109F900066700EF07DFBE36A7BB1324604212046F9
:109FA0009847E36A4BB13246314620469847E36A08
:109FB0001BB1324602212046984705F10F03DBB260
:109FC000022B3ED83C4A52F8238004F1100630465A
:109FD0000EF0C6FA00283DD104F1140630460EF00A
:109FE000BFFA002841D1012F0DD0FB1E012B0AD949
:109FF000A36A23B3BDE8F041304B3149314840F208
:10A00000F71211F04FBB94F8243023F004025B07E1
:10A0100084F8242013D4A36A002B44D01E68042F94
:10A0200008BF00250C361D7130460EF0E1FA90B3E2
:10A030000023A3623046BDE8F0410EF0D1BABDE87E
:10A04000F081FDB904F110063046A8460EF088FAFA
:10A050000028C1D03046414604F114060EF042FA01
:10A0600030460EF07DFA0028BDD0414630460EF055
:10A0700039FAB8E7114B144912484FF4DC7211F069
:10A0800011FB79E70D4B11490E487D2211F00AFBB7
:10A090004FF0000899E7094B0D490A4840F2EF12CA
:10A0A00011F000FBC4E7054B0A4906484FF4F37270
:10A0B00011F0F8FAA36AB1E7E8F90108C8F5010858
:10A0C0008CF8010808F3010860F6010860F801083F
:10A0D00070F8010890F6010870B530B34178012995
:10A0E000154604462AD0042918D06368A3B1B3F8F2
:10A0F0006420B2F5866F0FD3B3F86630042B0BD80B
:10A1000094F82430E66A23F0100384F824301EB15A
:10A110002A4602212046B047002070BD0121FFF7EA
:10A12000FFFC6368002BE2D1F6E7074B07490848BC
:10A1300040F2931211F0B6FA002070BDFFF796FBC3
:10A140006368002BD3D1E7E7C8F5010860F6010882
:10A1500008F3010838B504460D4689B10E4B9C4200
:10A160000AD00E4B9C4212D00D4B9C4203BFF123F0
:10A170002B700120002038BDF3232B70012038BD47
:10A18000084B09490948852211F08CFAE6E7F223C9
:10A190002B70012038BD00BFF4F90108F6F9010861
:10A1A000F5F90108C8F50108A8F8010808F3010845
:10A1B00030B50023056803710446686883B008B1B0
:10A1C00003B030BD2B7803F0F003102B16D0202BFA
:10A1D00030D108F02FF922686860506858B11378C0
:10A1E0001649222B04BF0123037408F0DDF823680D
:10A1F0005B68002BE4D1FF232371E1E704F048F80A
:10A200002168686048680028F5D0019003F064FD7B
:10A2100001980B4903F064FD01980A4903F07CFDA5
:10A2200001980949022203F0B5FD0849019803F09D
:10A230008FFDDCE7FA232371C2E700BFB197000866
:10A24000819E0008D9A000080D9E00086D9F00089F
:10A25000F8B5054607200E4601F0D6FF044628B3A0
:10A2600005F0F0030022102B02720570426001D04D
:10A27000202B1DD104F11007062138460EF00CF9F1
:10A280000146E0B904F10C000EF074F90546E8B996
:10A2900004F114000EF06AF9C4E90A56C4E907553E
:10A2A0004FF0FF336570A36184F824502046F8BD59
:10A2B000084B0949094840F2E52211F0F3F921461B
:10A2C0000720002402F000F82046F8BD38460EF0C2
:10A2D000FFF8F4E7C8F50108B4F8010808F301082D
:10A2E00010B5436882B0044633B11A4B1A491B4873
:10A2F0004FF4477211F0D6F904F110000EF030F966
:10A3000098B904F114000EF02BF9D8B904F10C003F
:10A3100001900EF069F901980EF070F921460720BE
:10A3200002B0BDE8104001F0CFBF0A4B0C490B480A
:10A3300040F2233211F0B6F904F114000EF010F9D6
:10A340000028E3D0034B0749044840F2263211F0BD
:10A35000A9F9DBE7C8F50108DCF8010808F30108F2
:10A360000CF9010848F901082DE9F04300F1100546
:10A3700083B0044628460EF0F3F830B32E4FDFF8D2
:10A38000BC80DFF8BC9001AE314628460EF0D6F80E
:10A39000013014D0237803F0F003102B48D1019B37
:10A3A000BB421846F0D04345EED04B45ECD002F00E
:10A3B00065FB314628460EF0C1F80130EAD1284647
:10A3C0000EF086F828460EF0D1F8143420460EF030
:10A3D000C7F850B3184FDFF86480DFF8649001AE1F
:10A3E000314620460EF0AAF8013018D0019DBD423A
:10A3F0002846F5D04545F3D04D45F1D0FFF7B4FFE1
:10A40000686818B103F076FE00236B602846FFF7FA
:10A4100067FF314620460EF091F80130E6D1204624
:10A420000EF056F820460EF0A1F803B0BDE8F08318
:10A43000019800F011FAA7E7F4F90108F6F901080C
:10A44000F5F9010870B50446006845789DB10378B8
:10A4500003F0F003102B36D1022D0CD0032D06D0C3
:10A46000FB232371BDE870400C300EF0C1B890F8AA
:10A4700024305B07F4D500252571FFF775FF2068B0
:10A4800042686AB1037803F0F003102B24D0202B2C
:10A4900004D11046D56107F099FF2068002343607E
:10A4A000C36A002BDED00022114698472068C36A99
:10A4B000002BD7D00022022198472068BDE87040C9
:10A4C0000C300EF095B8204B2049214840F25E42F6
:10A4D00011F0E8F82068BFE7836A3BB11A4B1D49C9
:10A4E0001B4840F2944211F0DDF820680422032357
:10A4F0004270002123728462FFF712FB88B1236847
:10A500005B78042B0ED114480EF09EF820680021D1
:10A510000C300EF049F810480EF090F823685B7884
:10A5200043B970BD084B0D49094840F29A4211F0F9
:10A53000B9F8E8E7BDE87040034B0849044840F229
:10A540009E4211F0AFB800BFC8F5010884F90108B8
:10A5500008F3010898F9010854CC0020B4F9010867
:10A56000036810B50446586830B11B7803F0F00357
:10A57000102B0BD0202B03D06FF00500207110BDE5
:10A58000A289A16807F094FC207110BDA289A1687E
:10A5900002F056FF207110BD10B504460068FFF7A9
:10A5A000F7F848B92368586820B11B7803F0F00326
:10A5B000202B03D06FF00A00207110BDA2689368B1
:10A5C0001BB9116807F058FEF6E7938952F8081B8B
:10A5D00007F0FCFDF0E700BFF8B500220368027148
:10A5E0000646586820B11B7803F0F003102B00D00A
:10A5F000F8BDB4684FF6FF7701E033685868BC4295
:10A60000254628BF3D46A9B202F0DEFF641BF4D107
:10A61000F8BD00BF10B504460068FFF7B9F838B9B7
:10A620002268137803F0F003102B03D06FF00500BD
:10A63000207110BD5378002B3AD15368002B3BD0CA
:10A64000936A0121517033B1214B2249224840F2D3
:10A65000237211F027F86369002B31D020680021A4
:10A660008462FFF703F90028E3D023685B78012BAD
:10A6700006D0174B194918484FF4E56211F012F84B
:10A6800017480DF0E1FF206800210C300DF08CFF21
:10A6900013480DF0D3FF23685B78012BC9D1BDE8C7
:10A6A00010400B4B0D490C4840F22C7210F0FABFD1
:10A6B0006FF004002071BCE76FF00A002071B8E76A
:10A6C000034B0849044840F2247210F0EBFFC5E741
:10A6D000C8F5010898F9010808F30108B4F9010860
:10A6E00054CC0020BCF9010802685368002B31D01B
:10A6F000017C30B481B181681C680C60002101715B
:10A70000127802F0F002102A2FD0202A16D1C26847
:10A710005B8A138030BC704784685D682560017176
:10A72000127802F0F002102A17D0202A06D11A7CE3
:10A7300052070BD5C2689B8A1380EBE730BC0C4BE9
:10A740000C490D4840F27D7210F0ACBFF523037147
:10A7500030BC7047F523037170471A7D012AF5D983
:10A760001A8BC36830BC1A807047DA8AF9E700BFD9
:10A77000C8F50108D0F9010808F3010810B504462E
:10A7800000684368427823B1037803F0F003102B8C
:10A7900002D0F523237110BD237A032B01D0022AA6
:10A7A000F7D0032AF5D0012A02D1FB23237110BD73
:10A7B000DB0734D4836A3BB11B4B1C491C4840F275
:10A7C000BD7210F06FFF2068846204234370002183
:10A7D000FFF7A6F90028DED023685B78042B06D0AB
:10A7E000114B1449124840F2C27210F05BFF12483C
:10A7F0000DF02AFF206800210C300DF0D5FE0E4828
:10A800000DF01CFF23685B78002BC4D0BDE810401E
:10A81000054B0849064840F2C67210F043BFFFF7E7
:10A82000A3FD2068C6E700BFC8F5010898F9010834
:10A8300008F30108B4F9010854CC002000F110031A
:10A84000DBB2102B9DBF4042024B53F82000052085
:10A85000704700BFF8F9010870B110B504460068F0
:10A8600020B102F00BF90023C4E900332146062091
:10A87000BDE8104001F028BD704700BF48B110B5D9
:10A880000446006808B102F0F9F80023C4E9003377
:10A8900010BD034B03490448812210F003BF00BFE1
:10A8A0003CFA0108B0FA010808F3010870B5002568
:10A8B00062F30F0562F31F45B0B1044600680E460F
:10A8C00008B102F0DBF841220021362002F048F9FD
:10A8D0000346206020B1C0E901650020636070BDBF
:10A8E00060604FF0FF3070BD044B05490548992268
:10A8F00010F0D8FE6FF00F0070BD00BF3CFA0108E9
:10A90000CCFA010808F301082DE9F843194F8146F4
:10A910008846002425010DF0AFFE7E594EB101346A
:10A920000DF0B6FE042CF5D14FF0FF342046BDE803
:10A93000F88347F805900DF0ABFE7B195E609B7BBA
:10A9400083B92F4400223A8199F80030BA8103F08C
:10A95000F003102B18BF4FF00108A7F80A8020461B
:10A96000BDE8F883044B0549054840F20E2210F07B
:10A9700099FEE6E714CC0020E4FA010818FB010870
:10A9800008F301082DE9F04F814600680078002A9D
:10A9900000F0F000ACBF15466FF00045102885B000
:10A9A0008B469A4606D0494B49494A4840F29F3265
:10A9B00010F078FED9F804001AF0080F0AF001032D
:10A9C00008BF0822DFF80CA1019318BF0C224FF03A
:10A9D000000830B303900489AC422646A4BFACB251
:10A9E0002E46002322460BEB080102F057FBB5422E
:10A9F00008EB060727DB019B03BB03980389A342EF
:10AA00003AD3B3422CDD214602F0B6F9AD1B002D3E
:10AA1000C9F804002CDDD9F80400B8461C2200282F
:10AA2000D8D1D9F8000003A9FEF7DEFC04460028BF
:10AA300035D1039850B3C9F80400CCE75FB138466C
:10AA400005B0BDE8F08F214B234940F2DD3250467E
:10AA500010F028FECFE70027384605B0BDE8F08F9C
:10AA60000023AD1BC9F8043002F008F8002DD2DC39
:10AA7000002FF0D0B84617E0144B184940F2E332EB
:10AA8000504610F00FFE03980389BAE70F4B1449A4
:10AA900040F2C532504610F005FE0398CBE7B8F1FE
:10AAA000000F08D0019B23B9D9F800004146FEF7FA
:10AAB00071FC4746C3E7FFF7C1FE08B1094B1860B8
:10AAC0000F3418BF01246742B9E700BFE4FA010858
:10AAD00038FB010808F301085CFB010884FB01084E
:10AAE0004C1B0208E81E0120F0B5064685B00F4653
:10AAF0001C461546D2B114B34FF404733846ADF872
:10AB0000003000F02BFE22683368ADF80200102AF6
:10AB100088BF1022019388BF22600023694628461F
:10AB2000CDE9023310F05EFF05B0F0BD084B0949D6
:10AB300009484FF4816210F0B5FD002CDCD1044BC4
:10AB40000649054840F2094210F0ACFDD4E700BFC9
:10AB5000E4FA010894FB010808F30108A4FB0108CA
:10AB60002DE9F04F1646926883B0814688469A4692
:10AB7000002A50D043680193002B7AD01868F368FC
:10AB80000789002B28DD3FB30025CB462B46C14665
:10AB90000CE058F8351002F081FAF36801359D4257
:10ABA00064DAA74262D9019A10682346D6F8088071
:10ABB00008EBC50EA7EB030CDEF804101FFA8CFCA3
:10ABC0008AB2D4186145A4B2E3D9DEF80010624617
:10ABD000C846D94602F062FA32680AB173686BB9A6
:10ABE00032690023B36102B1736118F001030CD024
:10ABF000AAF80070002003B0BDE8F08F0198331D63
:10AC000081890830FFF770FFEAE70198C9F804303E
:10AC1000FFF722FEECE7F368002B1DDC436801938D
:10AC2000C1F3C00292005BB9D9F8000001A9FEF798
:10AC300069FC0028DFD1019B2BB1C9F804309DE7E6
:10AC40001B681F89C8E70D4B0D490E4840F25E4254
:10AC500010F028FD019BF0E7084B0B49094840F232
:10AC6000494210F01FFD6FF00F00C4E7C846D946F7
:10AC7000B2E7C1F3C0029200D6E700BFE4FA0108D0
:10AC8000F4F3010808F30108B4FB0108002800F000
:10AC9000BA802DE9F0478469002C0F46054617DB82
:10ACA000032C10DC614D4FEA041855F8083053B1FD
:10ACB0000DF0E2FC0646042F00F2A980DFE807F061
:10ACC0006D68574F11005A4B09221A60BDE8F08792
:10ACD0000DF0D2FCAC69002C034671DB0DF0D8FC02
:10ACE000DEE745444FF00109AB7BA5F80C90002B43
:10ACF00038D0B5F908806F8930460DF0C9FC4D4B4E
:10AD00001D68002DE2D0012606FA04FAEB6913BB98
:10AD1000696900295CD0A869E8B101F1040C02E07E
:10AD20000133984217D051F833209442F8D1B8F14A
:10AD3000000F03DD3CF83320D20707D41FB13CF8E5
:10AD40003320920702D4B9F1000FE9D0EE6105F18A
:10AD500020000DF045FC2D68002DD7D1B6E7454405
:10AD600000236B813046BDE8F0470DF091BC4544AF
:10AD70006B89002B48D1AB7B4FF0010AA5F80AA0E4
:10AD8000002BEFD0B5F90880B5F80C905746B3E723
:10AD900045442B89013B2B81E4E74544B5F8088005
:10ADA00008F101080FFA88F8B8F1010FA5F808803A
:10ADB000D8DCAB7B002BD5D06F89B5F80C909BE726
:10ADC0000FB9013CAC61BDE8F04718460DF060BC1E
:10ADD000B8F1000F05DDAB681BB11B681AEA030F61
:10ADE000B4D12FB1EB681BB11B681AEA030FADD1C8
:10ADF000B9F1000FAFD02B69002BACD01B681AEA59
:10AE0000030FA8D0A2E7704701236B81AAE745444E
:10AE1000094B0A490A484FF41F6210F043FCAB7B10
:10AE2000002B9FD0B5F90880C6E700BF14CC0020E6
:10AE3000E81E012010CC0020E4FA0108E0FB010824
:10AE400008F3010830B5032883B017D8194D040161
:10AE50002B599BB1102A18D14B78022B15D18B0797
:10AE600013D14B684888019300F078FC01A9024691
:10AE70002859FEF761FA88B903B030BD0E4B09229C
:10AE80004FF0FF301A6003B030BD0C4B0C490D4839
:10AE900040F2E22210F006FC6FF00F00FFF7CEFC4C
:10AEA000034610B94FF0FF30E6E7034A4FF0FF309A
:10AEB0001360E1E714CC0020E81E0120E4FA010849
:10AEC000F0FB010808F301082DE9F0418AB00328DE
:10AED000119D35D8364E070106EB001056F8078055
:10AEE000B8F1000F2CD098F8008008F0F008B8F105
:10AEF000100F3FD09E4601AB059301230693109B94
:10AF000003930023CDE90733144601910292ADF873
:10AF100002300993EDB12B68049371460DF10203E1
:10AF200003AAFFF71DFE00283AD1BDF80220049BBA
:10AF30002B60944228BF144620460AB0BDE8F08139
:10AF40001C4B4FF0FF34092220461A600AB0BDE8BE
:10AF5000F0810DF10203714603AA0495FFF700FE8C
:10AF6000F0B9BDF802309C4228BF1C4620460AB00A
:10AF7000BDE8F081FFF706FD109B0446002BDBD0F7
:10AF8000002DD9D003A901AAF0590023FEF792F9A8
:10AF9000109ABDF804102B4603A8FFF7A5FDCBE7D8
:10AFA000FFF74CFC08B1034B18604FF0FF34C3E7C8
:10AFB00014CC0020E81E01202DE9F043032885B0C1
:10AFC000DDE90CE646D8DFF81C81040158F804C01E
:10AFD000BCF1000F3ED09CF800C00CF0F00CBCF1AE
:10AFE000100F68D0B2F5803F15466CD20F461FFA9D
:10AFF00082F9BEF1000F35D0102E34D19EF8013009
:10B00000022B30D11EF0030F2DD1DEF80430029355
:10B0100000220023BEF80200CDE9002300F09EFBD1
:10B02000ADF80C004A4639466846FFF73FFC064635
:10B03000002831D06846FFF721FC3046FFF7FEFBC1
:10B0400000283DD0234B1860002E39D1284605B08A
:10B05000BDE8F0831F4B09224FF0FF301A6005B0A6
:10B06000BDE8F0838EB11C4B1C491D4840F2526272
:10B0700010F018FB6FF00F00FFF7E0FB0346F8B18C
:10B08000144A4FF0FF301360E1E700220023CDE9BE
:10B09000002302963046C3E7694658F80400FEF7DD
:10B0A000D1FA06466846FFF7E9FB3046FFF7C6FBD4
:10B0B0000028C9D0C6E705B0BDE8F04300F014B8D9
:10B0C0004FF0FF30C3E7034B5A221A604FF0FF30B6
:10B0D000BDE700BFE81E0120E4FA01080CFC0108EE
:10B0E00008F3010814CC002010B5032884B02ED832
:10B0F0001C4C4FEA001C54F80C4044B394F800C0B8
:10B100000CF0F00CBCF1100F1AD113F0100F4FEA35
:10B11000630314BF0320012003F00403034320460C
:10B1200003AC009400240394FEF7B0FA0446FFF742
:10B1300085FB08B10C4B186084B9039804B010BDAE
:10B140000024CDE90044FFF737FF04B010BD064BE3
:10B1500009224FF0FF301A6004B010BD4FF0FF30ED
:10B16000ECE700BF14CC0020E81E012038B50B46E8
:10B17000022B11460AD0032B2AD0012B21D01B4BC6
:10B1800016221A604FF0FF34204638BD882A4FF04F
:10B190000001174A0CBF21202020FEF707F80546C2
:10B1A000EDB100212846FFF7AFFB431C044618BF52
:10B1B000A861E9D12846FEF759F80C4B17221A600E
:10B1C000E2E70B4A00211020FDF7F0FF0546E7E714
:10B1D000074AC9B24020FDF7E9FF0546E0E7034B07
:10B1E00069221A604FF0FF34CEE700BFE81E01204D
:10B1F0008DAC000803282DE9F04121D8AB4E0401A5
:10B2000098463359E3B1B8F1000F00F01F81A84808
:10B210000D4617460DF012FA3359CBB1062D4DD01D
:10B2200040F6FF7295422BD0BDB1A1480DF00CFA4B
:10B230005C23A04A4FF0FF3413602046BDE8F08144
:10B240009C4B09224FF0FF341A602046BDE8F08184
:10B2500097480DF0F9F90923EBE7012F00F0D380AF
:10B26000022FE2D1069A032A60D95B68002B5DD0D9
:10B27000D8F800208E48DA720DF0E6F90024DCE7F9
:10B2800041F20B029742D0DC41F20402974230DDDA
:10B29000A7F58052053A062AC7D801A151F822F035
:10B2A000D5B3000871B300082BB200082BB2000818
:10B2B0002BB20008A3B3000837B30008069A032A8C
:10B2C00034D95A6892B31B7803F0F003102BACD139
:10B2D000137D012B2AD0012F00F0A680022FA4D1CC
:10B2E000D8F800307248C2F894300DF0ADF900245F
:10B2F000A3E7082F00F09580202F96D11A7802F04E
:10B30000F002202A91D1DF21069803280ED95B682C
:10B3100063B1D8F80040002C00F0BB80597A644833
:10B320000A435A720DF090F9002486E760480DF048
:10B330008BF916237DE7069A052AF7D998F80010AD
:10B34000002940F089801A7802F0F002102A00F0FB
:10B350008A80202A00F08F80574B5849584840F681
:10B360007D5210F09FF952480DF06EF9002464E709
:10B37000069A0F2ADAD9D8F808205249D8F80000DE
:10B3800081FB0241D2174FF47A74C2EBA11204FB85
:10B390000022002ACADB46481A620DF055F9002443
:10B3A0004BE7069A032AC1D95A68002ABED01B78F7
:10B3B00003F0F003202B7FF438AFD8F80040137C63
:10B3C0003B48002C5FD043F0010313740DF03CF9AF
:10B3D000002432E7069A0F2AA8D9D8F8082039495C
:10B3E000D8F8000081FB0241D2174FF47A74C2EB07
:10B3F000A11204FB0022002A98DB2D48DA610DF02F
:10B4000023F9002419E7069A032A8FD95B68002BD9
:10B410008CD0D8F8002026489A720DF015F9002437
:10B420000BE7F7213A466FE7D8F80040538B2048E6
:10B4300034B143F0400353830DF006F90024FCE6D9
:10B4400023F0400353830DF0FFF8F6E6194B0E226C
:10B450001A604FF0FF34F0E6404601F0DDF9014696
:10B46000F0B133596FE7586802F06AF810480DF0F0
:10B47000EBF80024E1E6586806F048FF0C480DF0B0
:10B48000E3F80024D9E623F0010313740DF0DCF88F
:10B49000D3E65A7A0648114059720DF0D5F8CCE639
:10B4A00003480DF0D1F81323C3E600BF14CC0020ED
:10B4B00054CC0020E81E0120E4FA01082CFC01080D
:10B4C00008F30108D34D621080B52F4882B00DF00B
:10B4D000B5F82E4B1B6813B12D4A106898472A4DBA
:10B4E0002C4E2D4F10E068B128460DF0ADF82246E5
:10B4F00001A930460DF000F8044628460DF09EF8EC
:10B50000013411D106F090FB06F0B6FB431C044653
:10B51000E9D128460DF098F8002201A930460CF038
:10B52000EBFF28460DF08AF8019C64B12378012BCB
:10B530001ED0022B18D06BB1184919483B46CF22B8
:10B5400010F0B0F8E0E7154915483B46912210F09D
:10B55000A9F8D9E7D4E902136068984780B9214671
:10B56000092000F0B1FECFE7D4E901309847CBE7DE
:10B57000D4E9013098472146082000F0A5FEC3E732
:10B58000606801F07BFAEAE754CC002058CC002038
:10B590005CCC002060CC002058FC010888FC01082D
:10B5A00008F3010870B591F83D3013F0180F064606
:10B5B0000C4621480AD00CF0D3FF48B3092000F014
:10B5C00023FE0546002834D01C4B08E00CF0C8FFD1
:10B5D00088B1092000F018FE054650B3184B1648F4
:10B5E000EB600022C5E901642A7029460CF07AFF5D
:10B5F000D8B9002070BD134B13491448FC2210F039
:10B6000051F8092000F000FE05460028E6D110E0C0
:10B610000C4B0D490D48FC2210F044F8092000F0B5
:10B62000F3FD05460028CFD103E02946092000F0AC
:10B630004BFE4FF0FF3070BD60CC002085830108C9
:10B640000974010858FC0108A8FC010808F3010866
:10B6500070B5064612480D460CF082FF70B1082006
:10B6600000F0D2FD0446C0B10123C4E901650C48D5
:10B67000237021460CF036FF40B970BD094B0A49D2
:10B680000A4840F25D1210F00DF8E8E72146082064
:10B6900000F01AFE4FF0FF3070BD4FF0FF3070BD6C
:10B6A00060CC002058FC0108A8FC010808F3010840
:10B6B00070B5064E0D46044630460CF0BFFF2846D6
:10B6C000A04730460CF0C0FF002070BD54CC0020D5
:10B6D00030B583B005460C4600F058FA154A164BB3
:10B6E0001648156006211C600CF0D6FE68B9144897
:10B6F0000CF094FFA8B90022124900924FF4806325
:10B7000011480CF0A5FF03B030BD104B1049114893
:10B7100040F261220FF0C6FF09480CF07FFF0028BD
:10B72000E9D00A4B0C490B4840F265220FF0BAFFF2
:10B73000E1E700BF58CC00205CCC002060CC0020AA
:10B7400054CC0020C9B4000800FD010858FC0108D1
:10B75000B8FC010808F30108DCFC010840BA80B21B
:10B76000704700BF00BA70472DE9F843414D424E83
:10B770002B68044600EB001006EB0010884600F131
:10B7800010074FEA041913B12A7AA24252D0EB688B
:10B7900013B12A7DA24246D0AB691BB195F8202097
:10B7A000A24239D06B6A1BB195F82C20A2422CD052
:10B7B00009EB040306EB0313DB7B24B1B27A022A04
:10B7C0003ED0012C05D096F81A21022A42D0022C34
:10B7D00005D096F82A22022A41D0032C03D096F8ED
:10B7E0003A23022A40D0032B0DD8244DA14406EB66
:10B7F000091655F8230006F0E9FDF27B0021042329
:10B8000045F82210F373BDE8F883AA6A414638462A
:10B81000984700236B62CBE7EA6941463846984770
:10B820000023AB61BEE72A694146384698470023AA
:10B83000EB60B1E76A683846984700232B60A6E7BB
:10B84000F27B9A42BDD109EB040306EB03130422F9
:10B85000DA73D8E796F81F219A42B8D1F3E796F841
:10B860002F229A42B9D1EEE796F83F239A42BAD1F5
:10B87000E9E700BF74CC0020ACCC002064CC0020F1
:10B880002DE9F04F594B00EB001403EB041487B083
:10B8900003010193E37A012B824607D9544B5549A2
:10B8A000554840F2FA220FF0FDFEE37A534A52F86F
:10B8B0002340002C00F08780019B4C4E03EB0A05CF
:10B8C0002D0105F1100434442046F4F7D1FC123068
:10B8D00081B24FF42072362001F042F981460028EF
:10B8E00068D03544002328890593CDE90333FFF759
:10B8F00035FF0123ADF80C008DF80E3003A94FF48D
:10B9000080730C224846ADF8103001F015FC013C64
:10B910000C264FF6FE7B62782E2A04F101075FD0D9
:10B920003B46002504E05A782E2ACDB245D0034686
:10B93000691C581C002AF6D1A3EB07081C461FFA05
:10B9400088F82B4633445B4531DC2A46314648466D
:10B9500001F0AEFC731C424635449BB23946484662
:10B9600001F050FCADB222786E1CB6B2002AD2D1E2
:10B970003146484601F09CFC4FF00120AB1C9BB2C5
:10B98000042202A90290484601F03CFC019B174AA0
:10B990001A491B48534402EB0313DA7ADB7B01EBB1
:10B9A000820250F823004946352306F00FFC484632
:10B9B00001F064F807B0BDE8F08F1B1B1FFA83F895
:10B9C00004462B46BEE721465046FFF7CDFE019BBD
:10B9D000064A534402EB03139C7207B0BDE8F08F94
:10B9E00000233C4698461D46ACE700BFACCC002087
:10B9F00010FD010840FD010808F30108A4CC002057
:10BA000064CC0020704700BF012800D9704721B1E5
:10BA1000054B0A6843F820207047044A024B12681D
:10BA200043F82020704700BFA4CC002078210208F2
:10BA30002DE9F0474E4CDFF84C814E4F4E4E00251D
:10BA400014F8013C5FFA85FA032B00F28880DFE8E6
:10BA500003F01F023226DFF830910EF031FE99F824
:10BA60000A30022B80B245D099F81A31022B49D006
:10BA700099F82A32022B4DD099F83A33022B51D043
:10BA80003E4B24F8030C504644F8013CFFF7F8FE07
:10BA90000135042D04F58874D2D1BDE8F08754F83F
:10BAA0000B3CF3B9002304F8013C0135042D04F5E7
:10BAB0008874C5D1F1E76378013BDBB26370002B7A
:10BAC000E6D1A3780133DBB2042BA3702FD06370CF
:10BAD00050460135FFF7D4FE042D04F58874AFD12C
:10BAE000DBE7013B44F80B3C002BD1D1002304F8E9
:10BAF000013CDAE7B9F808308342AED099F81A3140
:10BB0000022BB5D1B9F818318342A6D099F82A3260
:10BB1000022BB1D1B9F8283283429ED099F83A333A
:10BB2000022BADD1B9F838338342A9D195E72378F8
:10BB30003BB9134A526822B1A37040F2011323802B
:10BB4000C6E7504600210135FFF70EFE0023042D05
:10BB500004F8013C04F588747FF472AF9DE7434616
:10BB600040F25B42394630460FF09CFD90E700BF43
:10BB7000B7CC002074FD010808F3010802000100A1
:10BB8000A4CC002010FD0108ACCC002008B50CF0BE
:10BB900039FD00F00FF800F0D9FA00F005FC06F0CE
:10BBA0007DF801F023FCFFF72DFFBDE8084005F00C
:10BBB000EDBF00BF124B1349134A23F0030303F5F3
:10BBC000C86070B54FF0010C0860104C104913604C
:10BBD0004FF4C86500220F481D6083F844C6C3F8BF
:10BBE00040161A7123600CF019FD00B970BDBDE854
:10BBF0007040094B09490A4840F21F220FF052BD1C
:10BC000017D1002010D1002004D100200CD1002039
:10BC10004006400608D1002094FD0108C4FD01083B
:10BC200008F30108002800F0988083072DE9F0410F
:10BC3000044640F08D80614E3368A0F10805AB42A8
:10BC400005D85F4F3A6800F10C039A420CD25D4B65
:10BC50005D4940F27F225D480FF024FD0CF00CFDA1
:10BC6000BDE8F0410CF014BD59480CF0E7FC14F8A5
:10BC7000043C002B00F09C8034F8083C326834F817
:10BC8000061CB3F5C86F09D8B1F5C86F06D8A81A55
:10BC900080B2884212D0515A81420FD0494B4D494F
:10BCA00040F2952249480FF0FDFC49480CF0CCFCCD
:10BCB0000CF0E2FCBDE8F0410CF0EABCD7F800C0A3
:10BCC000D118614502D049888142E7D1DFF820814F
:10BCD000002104F8041CD8F80010A94288BFC8F855
:10BCE000005095423AD3654542D23268D1188D4210
:10BCF00014D0087990B9386881420FD0D8F8003054
:10BD000099420B8824F8083C098808BFC8F80050FD
:10BD1000B1F5C86F02D01144A81A488034F8060C57
:10BD200011188D420FD00E796EB91352D8F80060F9
:10BD300034F8083CB54208BFC8F80010B3F5C86F26
:10BD40001CBFD2185080BDE8F04121480CF07CBCEB
:10BD50001C4B214940F273227DE77047194B1F4964
:10BD60001A4840F2DF120FF09DFC3B689D4206D35B
:10BD7000144B1B4915484FF4F0720FF093FC14F864
:10BD8000043C33B10F4B1749104840F2E1120FF059
:10BD900089FC34F8083CB3F5C86FA6D9094B1249A1
:10BDA0000A484FF4F2720FF07DFC34F8083C9CE72F
:10BDB000044B0E494FF4237274E700BF0CD10020EE
:10BDC00010D1002094FD010804FE010808F30108C9
:10BDD00008D1002048FE0108E0FD01087CFE0108B2
:10BDE00094FE0108B0FE0108CCFE010820FE010807
:10BDF00004D100202DE9F843CC1C24F00304A4B2A4
:10BE00000B2C05465ED9B4F5C86F5ED8A1425CD84C
:10BE1000DFF86081D8F80030AB423DD84D4A126857
:10BE2000AA4239D935F8086CA5F10807FF1ABFB244
:10BE3000083EF61BB6B2A64268D371D046480CF055
:10BE4000FDFB35F8082CD8F8003003EB020999F80F
:10BE5000041000293CD1B2F5C86F70D03F49B9F841
:10BE600000000A6808343C44A4B24A4503EB0402CB
:10BE700008BF0A60002110805780117125F8084C16
:10BE80001288B2F5C86F01D01A44548032480CF0C1
:10BE9000DBFB2846BDE8F883314B3249324840F29B
:10BEA000D1220FF0FFFBD8F80030AB4203D8294A6B
:10BEB0001268AA42B6D80CF0DFFB0CF0E9FB28466A
:10BEC000BDE8F8830C24A142A2D90020BDE8F88384
:10BED00004F1140189B2B142D8D808343C44B2F517
:10BEE000C86FA4B21FD019191C480A8000220A7119
:10BEF00006684F8025F8084C0A888E4288BF01608A
:10BF0000B2F5C86F1CBF9B185C80BFE7144B174984
:10BF100015484FF439720FF0C5FB0020BDE8F883D7
:10BF20002846BDE8F8830E4B11490F4840F21632FF
:10BF30000FF0B8FB35F8082CD8F80030D3E7084BE1
:10BF40000B49094840F2F5220FF0ACFBD8F800305D
:10BF500084E700BF10D1002008D1002004D10020C8
:10BF600094FD0108F8FE010808F3010810FF01081C
:10BF700030FF01080CD10020002840D02DE9F84303
:10BF800000F1030828F003081FFA88F8B8F10B0F36
:10BF90002ED9B8F5C86F2FD840452DD84A4E4B4FF3
:10BFA0004B480CF04BFBD6F800C03968ACEB0105F0
:10BFB000ABB2C8F5C86E73451D4613D26FF00709C2
:10BFC00006E0CB5A1A4442451AD273451D4609D29F
:10BFD000CC18A9EB030220790028F2D0CD5A2B46C9
:10BFE0007345F5D33A480CF02FFB0020BDE8F883E9
:10BFF0004FF00C084045D1D90020BDE8F8837047C8
:10C0000008F11400824208F1080829D305EB080959
:10C010001FFA89F9B9F5C86F49D001EB0902002070
:10C02000107121F8093001235580A4F80090237184
:10C0300031F80930B3F5C86F02D00B44A3F8029071
:10C040006445244D26D022480CF0FEFA2B68A0440B
:10C05000434517D3A30706D104F10800BDE8F883D0
:10C0600001232371ECE71C4B1C491D4840F2BB32F5
:10C070000FF018FB184B1B49194840F2BD320FF066
:10C0800011FBE9E7144B1849154840F2B9320FF09B
:10C0900009FBDFE72868234603E01B880B441A7975
:10C0A0001AB19842F9D13060CDE73360CBE70A4B43
:10C0B0000E490B4840F287320FF0F4FA39682388B2
:10C0C000D6F800C0A9E700BF04D100200CD10020A1
:10C0D00008D1002010D1002094FD010874FF010850
:10C0E00008F30108A4FF010844FF010830FF01081C
:10C0F00038B501FB00F4A3B29C420AD11846FFF701
:10C100003BFF054618B1224600210FF075FB28467B
:10C1100038BD0025284638BD30B4D0E90135448803
:10C12000002129607CB10333B0F800C023F0030381
:10C130000A4600E003460132A242196003EB0C00FC
:10C140001946F7D12B6030BC704700BFF0B5DFF85F
:10C1500054E0124B124D0EF138070424002603332D
:10C160005EF8042B2E6023F003036CB10021B2F8BB
:10C1700000C00A4600E003460132A242196003EB08
:10C180000C001946F7D12B60774505D0DEF800206A
:10C19000D2E901355488E2E7F0BD00BF140901205F
:10C1A000CC0901203401020838B50446B0B10CF0C6
:10C1B00063FAA3681C680546CCB122681A60A3071D
:10C1C00004D128460CF064FA204638BD0A4B0B49CE
:10C1D0000B484FF48C720FF065FAF2E7064B0949F1
:10C1E00007484FF49E720FF05DFA204638BD0CF000
:10C1F0004FFA204638BD00BFC8FF01080C000208F6
:10C2000008F30108F8FF01080D2838B519D8144BB8
:10C2100053F820400CF030FAA3681C680546D4B1EE
:10C2200022681A60A30704D128460CF031FA204690
:10C2300038BD0C4B0C490D484FF48C720FF032FA9C
:10C24000F2E7084B0A49094840F2571200240FF060
:10C2500029FA204638BD0CF01BFA204638BD00BF35
:10C2600034010208C8FF01080C00020808F30108A5
:10C2700030000208C0B170B50C4661B1A307054695
:10C280000AD10CF0F9F9AB681A6822601C60BDE8AD
:10C2900070400CF0FDB970BD074B084908484FF4D9
:10C2A000B6720FF0FFF9ECE7034B0649044840F281
:10C2B00095120FF0F7B900BFC8FF0108500002083F
:10C2C00008F30108F8FF01080D2812D870B50C46D4
:10C2D00071B10F4B53F820508B0711D10CF0CCF9F2
:10C2E000AB681A6822601C60BDE870400CF0D0B9E1
:10C2F00070BD084B084909484FF4D5720FF0D2B908
:10C30000044B074905484FF4B6720FF0CBF9E5E747
:10C3100034010208C8FF01087000020808F3010890
:10C32000500002086FF00B00704700BF70B5054663
:10C3300082B016460C4641B36B6822689A4202D11D
:10C34000002002B070BD336001A93046019202F0B6
:10C3500093FB01A9304606F07BF895F83D20236851
:10C360006B6002F00501052906D0EB690BB1284688
:10C370009847012002B070BD002BF6D01307F4D50A
:10C38000291D28460AF068FEEFE7044B04490548DA
:10C3900040F2CB120FF086F9CEE700BF6C01020825
:10C3A000A001020808F30108704700BF2DE9F04121
:10C3B000344D002914BF0F462F46002A14BF904663
:10C3C000A846002B18BF1D463B6886B00646002BCA
:10C3D00038D0002340201C46D8F80020B1688A429B
:10C3E00004D00091B2600446CDF810D02A68F168FC
:10C3F0008A4222D044F02004F26001AA0191A4B242
:10C40000059273BB0DF10808424639463046FFF7E6
:10C410008DFF30B31C4BCDF80C8044F090051C68A8
:10C42000ADB264B1236803AA2946304698476468D0
:10C43000002CF7D106B0BDE8F081C3B18CB906B0CD
:10C44000BDE8F08102AA3946FFF770FF28B102ABC0
:10C450000393502001231024BEE70446012340200B
:10C46000BAE7094B44F08005ADB21C68D9E70DF17D
:10C470000808424639463046FFF758FF0028DDD00D
:10C48000C8E700BF78210208D00901202DE9F84F44
:10C490000B9D0646002800F08280002D00F0888069
:10C4A0000A9C4462474F0C9C0461474C3F7880F8DB
:10C4B0004070002B08BF2346002A08BF22460029EF
:10C4C00008BF2146414F47610024C0E90144C0E94B
:10C4D0000744C460848680F83D408462C462FFF7EC
:10C4E00065FF3046A8478246002855D196F840207F
:10C4F000DFF8F490DFF8E4B0D9F80040FF2A04BF79
:10C5000086F840A0002274B3DFF8E080304F0025A9
:10C5100007E094F8403096F84020934214D0246805
:10C52000FCB1A64205F1010513D0FF2DF1DD5B46FC
:10C5300040F28D12274938460FF0B4F894F8403095
:10C5400096F840209342EAD10132D2B286F84020D8
:10C55000D2E75B4640F28B12414638460FF0A2F814
:10C56000E3E7D9F80040FE2A14D0531CDBB21A4A84
:10C570003460144914680B70C9F800603CB123683A
:10C5800000220121304698476468002CF7D13046DC
:10C59000BDE8F88F0023EAE72046BDE8F88F0F4B8F
:10C5A0000F490B4840F227120FF07CF83046EFE7B6
:10C5B0000A4B0C4906484FF494720FF073F8284662
:10C5C000E6E700BFDC0901207821020825C3000846
:10C5D00008F3010804020208D00901206C010208D6
:10C5E000B0010208CC010208D8090120F0010208BC
:10C5F000014B1860704700BFD409012038B330B533
:10C6000090F83D30DA0785B005461ED4C26943F084
:10C61000010380F83D3002B19047144A14680123A9
:10C620008DF804303CB1236801AA082128469847B8
:10C630006468002CF7D195F83D3003F00502052A17
:10C6400003D16A680AB11B0708D405B030BD084B96
:10C65000084909484FF454720FF024B8291D2846A0
:10C6600005B0BDE830400AF0F7BC00BFD00901209A
:10C670006C0102083402020808F3010850B330B517
:10C6800090F83D30DA0785B0054601D405B030BDDD
:10C6900014490C6800228DF804204CB1236801AACB
:10C6A0000821284698476468002CF7D195F83D305A
:10C6B00023F001021B0785F83D2007D4EB69002B0E
:10C6C000E4D0284605B0BDE83040184728460AF0B7
:10C6D00055F9F3E7044B0549054840F29B320EF04B
:10C6E000E1BF00BFD00901206C010208500202081E
:10C6F00008F3010800B1C161704700BF002836D0BF
:10C7000030B590F83D305A0785B0054601D505B0E3
:10C7100030BD43F0040380F83D3007F04BFA284663
:10C7200005F02EFF95F83D3003F00502052A14D0E0
:10C730002B6A0BB128469847104A146801238DF8DC
:10C740000430002CE3D0236801AA0421284698472E
:10C750006468002CF7D105B030BD6A68002AE7D0C4
:10C760001B07E5D5291D28460AF076FCE0E7044BB7
:10C77000044905484FF478720EF094BFD0090120A7
:10C780006C0102087002020808F30108E8B130B534
:10C7900090F83D305A0785B0054614D5026A23F05B
:10C7A000040380F83D3002B190470B4A146800231F
:10C7B0008DF804303CB1236801AA0421284698472B
:10C7C0006468002CF7D105B030BD044B044905481E
:10C7D00040F206420EF066BFD00901206C0102084B
:10C7E0009402020808F3010800B10162704700BF1B
:10C7F00068B1084B1A6812B907E012682AB192F8BA
:10C8000040300133DBB28342F7D110467047024615
:10C8100010467047D8090120E0B110B50446023037
:10C820000DF096FE0C4BC2B2186810B910E000680B
:10C8300070B190F840309342F9D190F83E302178B1
:10C840009942F4D190F83F3061789942EFD110BD10
:10C85000002010BD00207047D809012038B50D46D2
:10C86000044630B175B10B4B25601A6862601C60DC
:10C8700038BD094B09490A4840F2C9620EF012FF5F
:10C88000002DF0D1044B0749054840F2CA620EF072
:10C8900009FFE8E7D00901206C010208B80202088C
:10C8A00008F30108D402020808B50BF0E5FE094BB5
:10C8B00000221A700BF0ECFE074B186810B908E064
:10C8C000C06830B1436F002BFAD0BDE8084002F0D9
:10C8D0002DB908BDDD090120E009012010B50330A4
:10C8E00020F0030C1846002361F30F03BDF80CE0A1
:10C8F000029C61F31F43614471450BD804B1644449
:10C900000021C0E901430160012302210273417348
:10C91000C38110BD002010BD10B5F0B1B1F5803F4E
:10C920000BD2C1B103898AB213449BB29A4204D894
:10C9300090F90CC0BCF1000F01DB012010BD446870
:10C9400000F1100C611A6145F7D3B0F80AC04160DC
:10C95000624442810381002010BD044B0449054814
:10C9600040F2DF120EF09EFE012010BDE802020828
:10C970004C1B020808F3010810B598B1B1F5803FCF
:10C980000ED259B143898AB2934214D344680C44FD
:10C99000018944609B1A8A1A43810281002010BDDC
:10C9A000012010BD084B0949094840F24B220EF006
:10C9B00079FE012010BD044B0649054840F255227E
:10C9C0000EF070FE012010BDE80202084C1B0208A8
:10C9D00008F301082C030208002910B515DB20B369
:10C9E00009B303898AB213449BB29A422AD890F9B8
:10C9F0000C40002C4468A4EB01011FDB448941601A
:10CA0000224442810381002010BD4942E0B14389A4
:10CA10008AB29A4221D844680C44018944609B1A26
:10CA20008A1A43810281002010BD104B1049114821
:10CA300040F2DF120EF036FE012010BD00F11004AE
:10CA4000A142DBD2012010BD084B0949094840F240
:10CA50004B220EF027FE012010BD044B064905486D
:10CA600040F255220EF01EFE012010BDE802020821
:10CA70004C1B020808F301082C0302082DE9F047BB
:10CA80000546002856D0DFF8C890DFF8D0A0DFF8C0
:10CA9000C880002608E02B69002B3DD02846984727
:10CAA0000136F6B2FCB125460BF0E6FDAB7B07463E
:10CAB000E3B1013BDCB2AC7338460BF0E9FD94B94D
:10CAC0006A7B2C682B7B9207E5D403F00F03022BC3
:10CAD0001DD0012B29D093B928460136FFF7A2F8C3
:10CAE000F6B2002CDFD13046BDE8F0874B4640F26D
:10CAF000F122514640460EF0D5FDAB7BD9E71249F5
:10CB00004B4640F20F3240460EF0CCFDC8E72946B6
:10CB10000D20FFF7D9FBC3E74B460C4940F2FF223B
:10CB200040460EF0BFFD2B69B8E729460C20FFF701
:10CB3000CBFBB5E7064B074907484FF437720EF0B9
:10CB4000B1FD2E46CFE700BF880302086403020848
:10CB5000E80202084C1B020808F301084C03020813
:10CB60002DE9F843002561F30F05B2F5C17F0F46AB
:10CB700061F31F451FFA80F948D0164610D822F0FD
:10CB80004003012B9CB231D0464B4749474840F205
:10CB900027120EF087FD4FF000084046BDE8F883ED
:10CBA000B2F5207FF0D109F10303033727F0030723
:10CBB00023F003033B449BB20446BB4203F1100045
:10CBC00080B2E8D38742E6D8FFF7D6F9804600283E
:10CBD000E3D0374A0319C0E902521333002123F08E
:10CBE0000303C0E900134046BDE8F8830C20FFF7BB
:10CBF0000BFB80460028D0D0002306734373C4810A
:10CC0000C0E9003385604046BDE8F8830026294C22
:10CC1000B046354606E08FB23060002FBDD00646E4
:10CC20004FF000090D20FFF7EFFA09F1030323F09D
:10CC30000303C3F514739BB2BB42814428BF3B4638
:10CC400009F11309F91A29F0030268B1C0E9005289
:10CC500007814381C460B8F1000FDCD1F91A8FB2AB
:10CC60008046002FDBD198E7134D0BF005FD2C78A3
:10CC70000123E4B22B700BF00BFD34B1B8F1000FBF
:10CC800089D04046FFF7FAFE85E70C482146FEF7BB
:10CC9000DFFC0028F2D00BF0EFFC2C700BF0F8FC5E
:10CCA000ECE700BFE80202089C03020808F3010851
:10CCB0008000010082000100DD090120A9C80008F0
:10CCC00070B50D46044600283BD02289AA421FD9E0
:10CCD00063899D420DD9A91A89B20A442281246828
:10CCE000EB1A9DB2002C34D06389AB4201D2228969
:10CCF000F3E7227B002665F30F06120765F31F4654
:10CD000007D02068A66008B1FFF7B8FE00232360B3
:10CD100070BD9D42F5D0637B9B07F2D463681B1BFB
:10CD2000E918204689B2FFF765F804460028E8D1E3
:10CD30000C4B0D490D4840F2BD120EF0B3FC64815E
:10CD4000FFDE084B0A4909484FF4CC720EF0AAFCEA
:10CD5000BBE7044B0749054840F2AF120EF0A2FCB6
:10CD60006389FFDEE8020208E803020808F301080D
:10CD7000B8030208D003020870B50346C9B1D8B1A0
:10CD80000C46002607E01D681E608CB2FFF776FE99
:10CD900084B18DB12B465A89A2421846A4EB0201F8
:10CDA000F1D9586819892044121B091B58605A810F
:10CDB00019811D46284670BD0025284670BD00BF5C
:10CDC00038B10023006801339BB20028FAD118461D
:10CDD000704703461846704758B110B504460BF02B
:10CDE0004BFCA37B0133A3730BF052FCA37B0BB171
:10CDF00010BD7047BDE81040034B0449044840F2A1
:10CE000042320EF04FBC00BFE802020804040208E0
:10CE100008F3010870B540B30D4631B304680CB98E
:10CE20002CE014460389B5F808C0226863440381E6
:10CE30002046002AF5D1638922899A4210D0104BEE
:10CE40001049114840F262320EF02CFC236833B1D5
:10CE50000B4B0E490C4840F263320EF023FC238941
:10CE60002A8925601344238170BDBDE87040044BBE
:10CE70000749054840F259320EF014BC0446DAE77F
:10CE8000E80202085004020808F3010880040208BE
:10CE90001804020870B50D4600282FD0002940D094
:10CEA000036804463BB1228929890A4422811C4631
:10CEB0001B68002BF7D1638922899A4210D01D4B41
:10CEC0001D491E4840F262320EF0ECFB236833B17C
:10CED000184B1B49194840F263320EF0E3FB2389DB
:10CEE0002A892560134423810BF0C6FBAB7B0133F9
:10CEF000AB730BF0CDFBAB7B53B170BD0D4B114948
:10CF00000E4840F259320EF0CDFB002DECD170BD31
:10CF1000BDE87040074B0C49084840F242320EF021
:10CF2000C1BBBDE87040034B0649044840F259328A
:10CF30000EF0B8BBE80202085004020808F301082A
:10CF40008004020818040208040402082DE9F84FBE
:10CF5000002800F08B800E46002900F087800289AF
:10CF60000B899A428046C0F08180002544894B8914
:10CF7000DFF80CA1DFF820B1DFF80C912F46E41B9D
:10CF80005B1B9C42D8F80400716828BF1C462944EA
:10CF9000384422460EF026FDB8F80A3027449F4256
:10CFA000254440D873899D4234D89D42B8F80A3050
:10CFB00024BF366800259F420FD0B6B173893289ED
:10CFC000934238D0B8F80A40B8F80820A242D6D127
:10CFD000D8F80020002AD2D010E0D8F80080B8F1AC
:10CFE000000F37D00027002EE8D1B8F80820B8F895
:10CFF0000A309A420BD1D8F8003043B1204B214976
:10D00000214840F2EE320EF04DFB6FF0050630463F
:10D01000BDE8F88F53461D4940F2DA3248460EF01B
:10D0200041FB7389C1E7534640F2D932594648461D
:10D030000EF038FBB6E73268002AC3D0104B114916
:10D04000114840F2E9326FF005060EF02BFB304636
:10D05000BDE8F88F002EDAD0094B0D490A484FF48D
:10D0600079720EF01FFB6FF00F06D0E7044B0949F1
:10D07000054840F2C9320EF015FB6FF00F06C6E707
:10D08000E80202080405020808F30108D8040208AF
:10D09000F404020890040208C00402082DE9F041DB
:10D0A000054670B30E46002934D01746904672B13B
:10D0B0004FF00008B5F80AC006EB080053B19C45D4
:10D0C000A3EB0C0206D82D6893B2002DF2D1404696
:10D0D000BDE8F081ACEB0304A4B2BC4228BF3C46DF
:10D0E00069683F1B224619444444BFB20EF07AFCE3
:10D0F0001FFA84F82D68002FE9D00023002DD9D124
:10D10000E5E7094B09490A4840F20A420EF0CAFA1B
:10D11000A846DCE7044B0749054840F20B420EF0F5
:10D12000C1FAB046D3E700BFE802020830050208A2
:10D1300008F30108500502082DE9F84F002849D0EE
:10D140000F4600293CD003899342904604462DD3D4
:10D150004AB3DFF898B0DFF8A8A015460026628928
:10D160006068AA4228BF2A469146B9190EF03AFCD7
:10D17000B5EB090524684E4409D0002CEFD15B467D
:10D1800040F2BD42514618480EF08CFAE7E7B04530
:10D1900009D0164B164914484FF499620EF082FAE2
:10D1A0002846BDE8F88F0020BDE8F88F0F4B1149E5
:10D1B0000D4840F2B5420EF075FA4FF0FF30F3E73C
:10D1C0000A4B0D49084840F2B4420EF06BFA6FF07A
:10D1D0000F00E9E7054B0949034840F2B3420EF05E
:10D1E00061FA6FF00F00DFE708F30108E8020208B8
:10D1F000E0050208A80502088C050208740502086B
:10D20000C805020890B32DE9F0410D46044602E03E
:10D21000246883B234B367899F42A3EB0700F7D930
:10D22000218903EB020841451CDBF91A8A4207DC1D
:10D230006068294618440EF0D5FB0020BDE8F08157
:10D2400060688EB23246184429460EF0CBFBA8EB3C
:10D25000070082B2002AF0D02068A919BDE8F04189
:10D26000FFF76ABF4FF0FF30BDE8F0814FF0FF30AD
:10D27000704700BF38B515460A462989FFF770FC8C
:10D28000044618B12946FFF761FE08B9204638BDAB
:10D29000044B0549054840F224520EF003FA20469B
:10D2A00038BD00BFE8020208F805020808F30108CB
:10D2B00018B90AE0006899B230B143898B42A1EBFA
:10D2C0000303F7D943685A547047704710B50446B2
:10D2D00008B3237D042B05D0072B0ED0032B01D0E0
:10D2E000002010BD204603F0A9FD50B90523237589
:10D2F000204604F08BF8002010BD204603F09EFD70
:10D3000038B1431CEDD1638B43F0080300206383E5
:10D3100010BD0923EBE7044B044905484FF4CE72D6
:10D320000EF0C0F9D5E700BF0C0602083C06020863
:10D3300008F3010870B50646806F18B1FFF79EFB31
:10D340000023B367746FBCB160682568214660B183
:10D35000FFF794FB21460320FEF7B6FF55B12C469C
:10D360002146606825680028F2D10320FEF7ACFF53
:10D37000002DF4D100237367F46E4FF6FF733386EC
:10D38000ACB160682568214660B1FFF777FB2146A4
:10D390000320FEF799FF55B12C46214660682568A9
:10D3A0000028F2D10320FEF78FFF002DF4D1346F57
:10D3B000ACB160682568214660B1FFF75FFB21468C
:10D3C0000320FEF781FF55B12C4621466068256891
:10D3D0000028F2D10320FEF777FF002DF4D10023BF
:10D3E000C6E91B33A6F8683070BD00BF08B50DF064
:10D3F00067F9034B6FEA80406FEA9040188008BDE0
:10D400002800002010B5037D012B044605D02146DD
:10D410000120BDE81040FEF757BF0649064B0748FC
:10D42000D4220EF03FF921460120BDE81040FEF75E
:10D430004BBF00BF480602080C06020808F30108AB
:10D44000F8B5364B002914BF8C469C4600285BD0AB
:10D45000037D002B4ED12AB3314D05F1100E55F846
:10D46000043B1B6813B90EE0DB6863B1D98A9142B3
:10D47000FAD1196821B1DCF800400CB1A142F3D116
:10D480006FF00700F8BDAE45E9D1DCF8003003B11C
:10D490000360244BC2821A68C260186004F032FB39
:10D4A0000020F8BD204E214F32884FF480454FF6C2
:10D4B000FF7E013292B21A4C724508BF4FF44042CF
:10D4C00054F8043B1B6813B90CE0DB6853B1D98AEC
:10D4D0009142FAD1013DADB2002DEAD132806FF018
:10D4E0000100F8BDBC42EBD13280002ACDD16FF0F3
:10D4F0000100F8BD0E4B0F490F4840F2AB220EF071
:10D50000D1F86FF00500F8BD094B0C490A4840F20C
:10D51000A9220EF0C7F86FF00F00F8BD78210208BD
:10D52000CC0B0208E809012028000020DC0B0208CF
:10D530000C0602087406020808F301085C060208DB
:10D5400019B191F840100131C9B20172704700BFA2
:10D5500038B50446C0B1238DE16AB4F832C0626ABE
:10D56000581ABCF5866F104494BFA0EB0C05A0F5CB
:10D570008665002D01DB638538BD531A002B0BDD5A
:10D5800000231846638538BD0B4B0C490C4840F20C
:10D59000A6320EF087F8DEE78D1AB5F5803F03D28C
:10D5A000ABB20020638538BD034B0649044840F206
:10D5B000B6320EF077F8F3E70C0602089C06020874
:10D5C00008F30108C0060208002844D070B5037DA6
:10D5D000012B0D46044630D0238D591989B2B1F57F
:10D5E000066F26D94FF406631946656AE06AB4F8F7
:10D5F00032C02185BCF5866F94BF00EB0C0200F5AC
:10D6000086622B449A1A002A0DDB1B1AB3F5067F9B
:10D6100061850DD3638B43F0020320466383BDE82D
:10D62000704003F0F3BE2B1A002B0EDD0023638540
:10D6300070BD8B42D6D80B46D7E70E4B0E490F482C
:10D6400040F2D2320EF02EF8C6E7451BB5F5803F0A
:10D6500008D2658570BD074B0949084840F2CF32B2
:10D660000EF020B8034B0749044840F2B6320EF0E2
:10D6700019F8EEE70C060208F406020808F30108A0
:10D68000DC060208C00602082DE9F04FA94DDFF8BC
:10D69000D8B22A689BF80030A74F0132013387B017
:10D6A0002A608BF80030A54B1C68002C00F091809C
:10D6B00000230593237D002B00F00C81012B00F04B
:10D6C00014810A2B00F01C819BF80030A27F9A4243
:10D6D00000F02381227DA377022A94F8423000F0E3
:10D6E00022810B2B40F2CB8002204FF0010A062A48
:10D6F00000F0E58094F8098018F0080820D0042A8A
:10D7000040F0E481236A2A68D4F894108C4ED21A2F
:10D7100001F5242303F6B843A6FB0363B2EB531FC2
:10D7200000F2C78194F89B308648854E00FB0311B8
:10D73000A6FB0131B2EB511F00F208824FF0000846
:10D74000666F56B12B68226A9A1AB4F9403003EB1F
:10D750004303B2EB430F80F09081237D032B00F055
:10D760000981092B40F033812B68226A9B1AF02B28
:10D7700040F20681D4F890602046FFF7DBFD059B60
:10D78000002B00F033816D4B1B68A34200F0208218
:10D79000059AE368D360B8F1000F40F03981237D2A
:10D7A000012BD4E9038A00F0458121460120664C13
:10D7B000FEF78AFD002323703EB16FF00C01504646
:10D7C000B0472378002B7FF46EAF4446002C7FF4E3
:10D7D00071AFDFF89881D8F800406CB3DFF858A13A
:10D7E000DFF88C91594F0026237D0A2B00F0298108
:10D7F000534640F2A152564938460DF053FF2B686C
:10D80000226A9B1AF02B40F22281237D012B16D82D
:10D81000E6B1D8F80030A34200F0EA81D4F80CB0A9
:10D82000C6F80CB0237D012B22D0214601205C4696
:10D83000FEF74AFD002CD7D107B0BDE8F08F0A2BC8
:10D84000E6D02046FFF776FD002EE2D1D8F8003072
:10D85000A34206D03F49534640F2B35238460DF03A
:10D8600021FF237DD4F80CB0C8F800B0012BDCD127
:10D870005346D422494638460DF014FFD5E794F8B4
:10D8800099A0BAF1000F00F0E880236F33B132495C
:10D890002E483B4640F2D4420DF004FFE36E002BCD
:10D8A00000F09E8194F89A300B2B40F21381227D78
:10D8B000062A4FF002004FF0010A7FF41BAF638B82
:10D8C000DB067FF53BAF2B68226A9B1A282B88BFAB
:10D8D000824633E73B461D48204940F2BE420DF0E8
:10D8E000E1FE237D012B7FF4ECAE3B461C4917483B
:10D8F00040F2BF420DF0D6FE237D0A2B7FF4E4AE4A
:10D900003B464FF49862174910480DF0CBFE9BF848
:10D910000030A27F9A427FF4DDAE0594E468002CCB
:10D920007FF4C8AE55E7052BA9D94FF000084FF09A
:10D93000010A05E7F00901200C060208E0090120B0
:10D94000D34D6210F8240100E409012008F3010816
:10D9500068080208C0080208A40702081C07020899
:10D960004807020874070208F5090120F809012098
:10D97000480602082B68226A9B1A282B3FF6FAAE4B
:10D98000BAF1000F7FF4F6AE237F627FE6680133C1
:10D99000DBB29A42237714D8DFF89C82D4F88C202B
:10D9A0000023237788F80030002A00F08680206961
:10D9B0002146904798F80030002B7FF474AE002881
:10D9C0007BD005943446002C7FF474AE01E7BAF1A5
:10D9D000000FD9D0012BD4F890607FF6D0AE0A2B7F
:10D9E0007FF4CAAE059B002B7FF4CDAE894B1B683C
:10D9F000A34206D0884989483B4640F271520DF057
:10DA000051FE844AE3681360B8F1000F3FF4C7AEDB
:10DA1000238B626A216D0293E38A0193231D009395
:10DA20002046234603F010FC237D012BD4E9038A12
:10DA30007FF4BBAE7A4979483B46D4220DF032FEE2
:10DA4000B3E62B68226A9B1AF02B3FF6E1AE26461E
:10DA5000E468002C7FF4C8AEEEE6B4F9303047F647
:10DA6000FE7099B2814202D801310BB22386B4F91B
:10DA70004010994243DD012039E67068A1463146E5
:10DA8000346860B1FEF7FAFF31460320FEF71CFC54
:10DA900054B126463146706834680028F2D103201C
:10DAA000FEF712FC002CF4D100234C46C9F8743068
:10DAB00053E682464FF0010842E62046059434467C
:10DAC00003F0A4FC002C7FF4F5AD82E6072A3FF4B6
:10DAD00019AE33E694F89930524A1A4494F89830C3
:10DAE00012F8012C934213D20133DBB2934284F833
:10DAF00098300DD2227D01204FF0000AF7E5204634
:10DB000003F0DCFA90B3236F6BB3227D0120EEE5C6
:10DB1000B4F860603EB9204603F0E6FE48B1227DCD
:10DB2000B2460120E3E53146204603F0AFF8002875
:10DB300066D094F89930062B4FF0000A98BF013355
:10DB400084F898A098BF84F89930DEE7204603F067
:10DB500089FE00287FF4F2AD94F89B3001338046B3
:10DB600084F89B30ECE5E36E002BCED0237D022BB6
:10DB700014D094F842302C4AB4F93C100C2B28BF36
:10DB80000C23D25CB4F93E3003EBE103934047F63B
:10DB9000FF729342A8BF1346A4F84030638EB4F8D6
:10DBA0004810A4F848305B009AB2B4F860308B4259
:10DBB00028BF0B465B08934238BF1346A4F84A308F
:10DBC00000232386A4F86A30204603F0FFFD9CE77B
:10DBD000164912483B4640F26D520DF063FDD7E501
:10DBE00013490E483B4640F2D5420DF05BFD59E625
:10DBF0001049534640F2AF5238460DF053FD0DE642
:10DC0000204603F003FC002893D18246227D0120A8
:10DC10006DE500BFE00901203C08020808F3010897
:10DC200048060208DC0B0208BC0B020810080208B8
:10DC3000D807020898080208E4090120C0B138B5E5
:10DC4000044621466068256860B1FEF717FF21464B
:10DC50000320FEF739FB55B12C4621466068256844
:10DC60000028F2D10320FEF72FFB002DF4D138BDA0
:10DC7000704700BF58B110B50446406808B1FEF7C0
:10DC8000FDFE21460320BDE81040FEF71DBB704796
:10DC900038B5054688B10320FEF7B6FA044650B100
:10DCA00068682968AA68EB68606060682160A260A3
:10DCB000E360FFF791F8204638BD044B044905485E
:10DCC00040F282620DF0EEFCE5E700BF0C060208B0
:10DCD000E808020808F3010800B10161704700BFBD
:10DCE00040B138B5037D012B0D46044603D0C4F87E
:10DCF000845038BD7047054B0549064840F2DF7235
:10DD00000DF0D0FCC4F8845038BD00BF0C060208EA
:10DD10000409020808F3010840B138B5037D012B5E
:10DD20000D46044603D0C4F8805038BD7047054BFB
:10DD30000549064840F2F3720DF0B4FCC4F8805077
:10DD400038BD00BF0C0602082C09020808F30108C0
:10DD500040B138B5037D012B0D46044603D0C4F80D
:10DD6000905038BD7047054B0549064840F60D02F6
:10DD70000DF098FCC4F8905038BD00BF0C060208A6
:10DD80005409020808F3010818B1037D012B08BFEC
:10DD900081617047A8B170B5037D012B0E46154611
:10DDA000044603D06577C4F88C6070BD084B094900
:10DDB000094840F63E020DF075FC6577C4F88C60AA
:10DDC00070BD034B0549044840F63D020DF06ABCA6
:10DDD0000C0602089409020808F301087C090208ED
:10DDE00038B1037D012B03D90A2B01D0FFF7A2BA6A
:10DDF0007047034B0349044840F651020DF052BCF2
:10DE00000C060208B409020808F3010838B50546F3
:10DE10000C46002951D0002D58D02B68A3423CD08D
:10DE20002BB1DA68A24240D01346002BF9D1237DF2
:10DE30000022E2600BBB638BDA074FD4E36E33B191
:10DE40002D4B2E492E4840F693020DF02BFC236FEC
:10DE500033B1294B2B492A4840F694020DF022FC9D
:10DE6000636F33B1244B2849254840F696020DF0E4
:10DE700019FC00232375E38238BD0A2BDED0012B69
:10DE8000F7D02046FFF756FA237D0A2BD6D0012B78
:10DE9000D1D100232375E38238BDE3682B60237D55
:10DEA0000022E260002BE8D1C5E7E268DA60237D5A
:10DEB0000022E260002BE0D1BDE70F4B1349104870
:10DEC00040F683020DF0EEFB002DA6D10A4B10495F
:10DED0000B4840F684020DF0E5FB9EE743F0020399
:10DEE0006383204603F092FA237D012BA6D1002301
:10DEF0002375E38238BD00BF0C0602080C0A020835
:10DF000008F30108240A0208400A0208D00902089E
:10DF1000EC090208002800F0CD802DE9F04F037DC8
:10DF2000012B87B00E46054600F0AB800A2B00F0AF
:10DF3000B380D5F850A0D5F824B0D5F89080D5F8A6
:10DF400010907BB9EA8A0592002A6FD0604A136864
:10DF5000AB4200F09380002B6CD0DA68AA4267D005
:10DF60001346F8E7EB8A5B4805932946FFF74EFF17
:10DF7000594B01221A702C6FACB16068276821469A
:10DF800060B1FEF77BFD21460320FEF79DF957B1F6
:10DF90003C462146606827680028F2D10320FEF73E
:10DFA00093F9002FF4D1EC6EACB16068276821467C
:10DFB00060B1FEF763FD21460320FEF785F957B1F6
:10DFC0003C462146606827680028F2D10320FEF70E
:10DFD0007BF9002FF4D16C6FACB1606827682146E3
:10DFE00060B1FEF74BFD21460320FEF76DF957B1F6
:10DFF0003C462146606827680028F2D10320FEF7DE
:10E0000063F9002FF4D1D6B92B7D012B26D02946F8
:10E010000120FEF759F9B8F1000F2CD06FF00C0178
:10E020004846434607B0BDE8F04F18471E46A2E7F2
:10E03000EA68DA600027EF603E4605979BE7059B9C
:10E0400001932B8B02932B1D00935A462B4651466E
:10E05000284603F0F9F82B7D012BD8D11F49204B1E
:10E060002048D4220DF01EFB29460120FEF72CF992
:10E07000B8F1000FD2D107B0BDE8F08FEB681360A4
:10E08000D8E7174B184917484FF410720DF00AFBE8
:10E090002B7D0A2B7FF44DAF14482946FFF7B6FEBF
:10E0A0002B7D012B0DD02946012007B0BDE8F04F94
:10E0B000FEF70AB90A4B0E490A4840F23D220DF01C
:10E0C000F1BA074B05490748D4220DF0EBFAEAE70D
:10E0D000E8090120E0090120E409012048060208BE
:10E0E0000C06020808F30108740A0208F809012066
:10E0F000580A02080121FFF70DBF00BFF8B5054619
:10E100000120FEF781F8034620B39C220021184627
:10E110000DF072FB554A56491268034655485D7525
:10E12000047899624FF4866053491A62FF25534A76
:10E13000A3F86400196352485249C3F89420DD7271
:10E140004FF006129C779864C3F88410C3F83E2001
:10E150001846F8BD4C4E34685CB12046E468438BE9
:10E160001907F9D523F008034383FFF7AFF8002C14
:10E17000F3D1464B186890B13C4B016A1C68C368E8
:10E18000611A4BB11A6AA21A914298BF1846DB680D
:10E1900098BF1146002BF5D10121FFF7BBFE0120EE
:10E1A000FEF732F803460028AFD1316889B12F4A13
:10E1B00014680A7D092A05D10A6AA21A90429CBFF6
:10E1C0000B461046C9680029F3D113B11846FFF772
:10E1D000A1FE0120FEF718F80346002895D131680A
:10E1E00089B1224A14680A7D082A05D10A6AA21A4E
:10E1F000824224BF0B461046C9680029F3D113B1EF
:10E200001846FFF787FE0120FDF7FEFF03460028B2
:10E210007FF47BAF2A0627D4EDB129463268013955
:10E22000C9B2C2B111480026076805E0146A3E1B56
:10E2300001461346D2684AB1507D8142F6D8F9D1E1
:10E24000146AA7EB040EB645F4D3F0E71BB1012125
:10E250001846FFF75FFE0120FDF7D6FF03460028B2
:10E260007FF453AF1846F8BD7F21D7E7F0090120AE
:10E2700060086008F5090120FFFF180200DD6D004D
:10E280000100300439E60008E0090120F809012006
:10E2900038B50120FDF7B8FF034628B39C220021C2
:10E2A00018460DF0A9FA534A534912780968534C9D
:10E2B000034653489862FF204025D8729A774FF062
:10E2C0000610504AC3F83E0019624F484F49C3F840
:10E2D00094205D754FF486621C639864C3F88410C3
:10E2E000A3F86420184638BD494D2C685CB120461F
:10E2F000E468438B1A07F9D523F008034383FEF73C
:10E30000E5FF002CF3D1434B186890B13A4B016AFA
:10E310001C68C368611A4BB11A6AA21A914298BF6D
:10E320001846DB6898BF1146002BF5D10121FFF795
:10E33000F1FD0120FDF768FF03460028AED12968F2
:10E3400089B12D4A14680A7D092A05D10A6AA21AE0
:10E3500090429CBF0B461046C9680029F3D113B107
:10E360001846FFF7D7FD0120FDF74EFF03460028B2
:10E3700094D1296889B1204A14680A7D082A05D1F8
:10E380000A6AA21A90429CBF0B461046C96800292F
:10E39000F3D113B11846FFF7BDFD0120FDF734FF9F
:10E3A000034600287FF47AAF2A68D2B11249844626
:10E3B0000D683F2006E0146AA5EB040C08461346DE
:10E3C000D2684AB1517D8842F5D8F9D1146AA5EBDB
:10E3D000040EE645F4D3EFE71BB101211846FFF721
:10E3E00099FD0120FDF710FF034600287FF456AF8A
:10E3F000184638BDF5090120F0090120FFFF180279
:10E400006008600800DD6D000100300439E6000896
:10E41000E0090120F809012030B50D4685B0044619
:10E42000002875D0237D1DB1042B0DD0072B0BD0F8
:10E43000012B75D0022B4CD0002B5BD0204605B0B1
:10E44000BDE83040FEF742BFA26F02B3638BDB062C
:10E4500022D5208BE18A626ACDE90110231D216D4E
:10E4600000932046234602F0EFFE237D012B04D9C2
:10E470000A2B02D02046FEF75DFF454A1368A342EF
:10E4800012D09BB1DA68A24272D01346F9E7228D0E
:10E49000B2F5066FCCD0D9E73E4B3F493F484FF429
:10E4A000B2720DF0FFF8D4E7E36813603C4B3D4ACD
:10E4B0001B6800200121A342E06011705BD0237D26
:10E4C000012B10D021460120FDF7FEFE002005B0F3
:10E4D00030BD21462E48FFF799FC237D314A0121AA
:10E4E0008B421170EED12B4B2F492C48D4220DF0CA
:10E4F000D9F8E7E7E38A002BE4D02C4A1368A3425B
:10E500003CD0002B31D0DA68A2422CD01346F8E779
:10E51000204B274921484FF4AF720DF0C3F881E733
:10E520002449002001F10C0551F8043F1B682BB170
:10E53000DA6F944212D0DB68002BF9D18D42F3D10F
:10E540001D482146FFF762FC237D012B19D021468F
:10E550000220FDF7B9FE002005B030BDD867DB68AA
:10E56000002BE5D1EAE7E268DA600023E360A9E77F
:10E57000E268DA609AE701F00FFFA7E7E36813604B
:10E58000F3E7044B0D490548DF220DF08BF8DEE779
:10E59000E00901200C060208C80A020808F3010875
:10E5A000240A0120E409012048060208E8090120A4
:10E5B000A80A0208CC0B0208EC090120E40A0208B0
:10E5C00038B540B3037D012B044606D0154639B952
:10E5D000D2B1042B10D8022B10D86FF00A0038BD2E
:10E5E000438B43F01003438382B9806F60B1FEF721
:10E5F00045FAA567284638BD072BEED120460021F5
:10E60000BDE83840FFF708BF002038BDBDE83840FE
:10E610000121FFF701BF054B0549064840F20722DB
:10E620000DF040F86FF00F0038BD00BF0C06020877
:10E63000000B020808F3010870B5002964D01546E4
:10E640000C467AB30B7D1689012B30D0228DB3187E
:10E650009BB2B3F5066F01D89A4226D94FF40662F1
:10E660001346666AE06AB4F832C02385BCF5866F4B
:10E6700094BF00EB0C0100F586613244511A002969
:10E680001DDB121AB2F5067F638506D3638B43F058
:10E6900002032046638302F0B9FE2846FEF7EEF936
:10E6A000002070BDABB1104670BD1A46D9E71B4BB8
:10E6B0001B491C4840F2D2320CF0F4FFC6E7331A73
:10E6C000002B13DD002363852846FEF7D7F90020D1
:10E6D000E7E70B7D012B03D04B8B43F010034B83FB
:10E6E00020460121BDE87040FFF796BE861BB6F5B7
:10E6F000803F01D26685D0E7084B0B49094840F2BC
:10E70000B6320CF0CFFFF5E7044B084905484FF44B
:10E71000D3620CF0C7FF6FF00F0070BD0C0602084B
:10E72000F406020808F30108C00602081C0B0208E0
:10E73000F8B578B3856FD0F884606F7B002304460A
:10E74000836756B100692A462146B04758B10D305B
:10E750001DD0A5676FF00400F8BD2989FEF734FFCE
:10E760002846FEF78BF9BB060FD5238DD4F88450CD
:10E77000B3F5066F1CBF0133238535B10023206933
:10E780001A462146A8470D3001D00020F8BD6FF091
:10E790000C00F8BD044B0549054840F209620CF035
:10E7A00081FF6FF00F00F8BD0C060208380B02085D
:10E7B00008F301082DE9F8431C4DDFF878802B7829
:10E7C0001B4E01332B700027D8F80040BCB12A78CB
:10E7D000A37F934215D0638BA277D9071AD41A0767
:10E7E00011D4A36FD4F80C9033B120463770FFF7E3
:10E7F0009FFF3378002BE7D14C46002CE7D1BDE8D2
:10E80000F883E468E2E723F0080363832046FEF719
:10E810005DFDE6E743F002036383204602F0F6FD68
:10E82000638B23F003039BB26383D8E7F5090120D0
:10E83000E4090120E009012008B5FFF7BBFF064A03
:10E8400013780133DBB21370DB0700D408BDBDE8D9
:10E850000840FEF719BF00BFF409012030B585B0AC
:10E86000002800F0AB80037D012B04466FD0428B63
:10E87000042B42F01002428334D1A26F002A3CD014
:10E88000208BE18A626ACDE90110231D216D00937E
:10E890002046234602F0D8FC237D012B04D90A2B05
:10E8A00002D02046FEF746FD494A13689C423BD001
:10E8B0002BB1DA6894423AD01346002BF9D1454B7C
:10E8C000454A1B68002501219C42E560117061D01A
:10E8D000237D012B21D001202146FDF7F5FC0020EE
:10E8E00005B030BD072BC8D0022B0CD013B3204687
:10E8F00005B0BDE83040FEF7E9BC228DB2F5066FE9
:10E90000BED1022BF2D121463148FFF77FFA237D99
:10E91000314A01218B421170DDD1304B30493148F1
:10E92000D4220CF0BFFED6E7E3681360C7E7E268C5
:10E93000DA60C4E7E38A002BCDD02B4A13689C42EF
:10E9400032D073B3DA68944229D01346F9E72749E5
:10E95000002001F10C0551F8043F1B682BB1DA6F60
:10E96000944212D0DB68002BF9D18D42F3D12048BC
:10E970002146FFF74BFA237D012B18D021460220B8
:10E98000FDF7A2FC002005B030BDD867DB68002B86
:10E99000E5D1EAE701F000FD284605B030BDE268A8
:10E9A000DA600023E36096E7E3681360F9E70B4B56
:10E9B00010490C48DF220CF075FEDFE7074B0E49CB
:10E9C00008484FF4F4720CF06DFE6FF00F0087E70B
:10E9D000E0090120240A0120E40901200C060208B4
:10E9E0004806020808F30108E8090120CC0B0208D8
:10E9F000EC090120E40A0208600B020808B530B1F6
:10EA0000074B084A186812681044186008BD064B86
:10EA10000649074840F6AF020CF044FEF0E700BF9D
:10EA200024000020F00901200C060208780B0208DF
:10EA300008F3010838B505460C4672B144B1A38EFF
:10EA400033B1282B06D9283B9BB29D4228BF1D46D7
:10EA5000284638BD0025284638BD044B04490548E2
:10EA600040F6C5020CF01EFEE8E700BF0C060208E7
:10EA7000940B020808F30108002843D0F8B5036896
:10EA8000054603B9F8BD264A14680E46ACB12168A4
:10EA90008B424FF6A96705D0E46874B12B682168F2
:10EAA0008B42F9D19BB2BB4220464FF00101F3D01B
:10EAB000E468FFF72FFA002CF0D11A4B1C6844B120
:10EAC0004FF6A96720682B6898421CD0E468002C98
:10EAD000F8D1002ED6D03368002BD3D0124B1A6851
:10EAE000002ACFD02B681168994205D0D268002A3D
:10EAF000C8D011689942F9D133681360D268002AEE
:10EB0000F0D1F8BD704780B2B8424FF00101204605
:10EB1000DCD0E468FFF7FEF9002CD3D1D9E700BFC1
:10EB2000E0090120E8090120EC09012070B5446FDB
:10EB3000C4B1064660682568214660B1FDF79EFFB6
:10EB400021460320FDF7C0FB55B12C4621466068E5
:10EB500025680028F2D10320FDF7B6FB002DF4D183
:10EB60000023736770BD00BF2DE9F0410446002803
:10EB700000F08D80544B188800283FD0534B544AE6
:10EB80001D68544BDFF85C81B2F800E01E6800217C
:10EB9000A8F800105FFA8EF7E5B101F1140CB44447
:10EBA0004B1C9BB2DA1B013A8842D2B240F28280FF
:10EBB0008E4525D8AA5C012A26D0022A28D0DAB1AF
:10EBC0009E4554D933441B7D012B79D90B4499B20E
:10EBD000002DE2D101F1130232444B1C88429BB25A
:10EBE00068D912F801CFBCF1010F5BD0BCF1020F64
:10EBF00055D0BCF1000FE5D1A8F80030BDE8F08198
:10EC00009CF80020012AD8D10CF1010C1946C7E765
:10EC10008A1C9E4592B226D933441B7D042B4CD1CD
:10EC2000531C834249DA01F1030C1FFA8CFC002DBE
:10EC30003AD096451FD8D21BD2B20431AB5CE64520
:10EC400089B24FEA03231ED8ACEB070C5FFA8CFCA9
:10EC500015F80C2013435A1EB2F5067F28BF4FF457
:10EC60000673638698E7DB1BDBB2EB5CD6E7DB1B46
:10EC7000DBB2EB5CA8E732440431137DE64589B290
:10EC80004FEA0323E0D9B4449CF81420E2E7124B86
:10EC90001249134840F27D720CF004FD6AE78A1CA9
:10ECA00092B2B9E7194698E732440431137D89B22C
:10ECB0001B02E8E7A8F80010A0E7A8F800209DE7ED
:10ECC0000231A8F8001099E7380A0120340A01201F
:10ECD000300A01202C0A0120E40B0208180C02085B
:10ECE00008F30108280A01202DE9F0410C460546E9
:10ECF000002845D0EB689889FCF730FDC30738D46D
:10ED0000234EE168238937682A8948683A440344D6
:10ED1000D31A002B21DB8889FCF720FD10F0010FAE
:10ED2000204605D12768FEF7A5FF97B13C46E8E7E6
:10ED3000EB680120B3F80C80FCF710FDEB68276846
:10ED400048EA0008A3F80C802046FEF793FF002F46
:10ED5000ECD13C462C60BDE8F081121A002AF9DDA6
:10ED6000C11B89B268682981FDF7AAFF2C60BDE844
:10ED7000F08120460024FEF761FF2C60BDE8F081A1
:10ED8000044B0549054840F21F420CF08BFCB1E7EB
:10ED9000200A0120E40B0208340C020808F30108E1
:10EDA0002DE9F04F83B0019200293CD0DFF8C880F4
:10EDB000DFF8B8B0DFF8C4A0DFF8B89006460C461C
:10EDC000E3685868FCF7CEFCE36827890546988914
:10EDD000FCF7C4FCD8F8003010F00300A5EB0305E5
:10EDE00018BF01203D440544002D2DDCD4E90070FE
:10EDF000FDF7E6FFB6F86630984205461AD81A497C
:10EE00002289B1F800C05B1B20466244A6F8663038
:10EE10000A80FEF72FFFB6F866303C463BB1002F64
:10EE2000CED1019BA3B1002003B0BDE8F08F002F2D
:10EE3000C6D1F8E75B4640F25742514648460CF0CF
:10EE400031FCB6F86630DAE7204603B0BDE8F08F53
:10EE5000064B0749074840F261420CF023FC019839
:10EE600003B0BDE8F08F00BF140A0120E40B0208D4
:10EE7000840C020808F30108FC0901205C0C02085C
:10EE80002DE9F84F0446002800F0E181237D032B93
:10EE900040F2F780B04BB14E1B78DB0670D4B04F18
:10EEA0003B8813B1227D062A11D93268636AD11AD0
:10EEB000002906DB218DC3F101035B1A1344002BEB
:10EEC00003DD638B43F002036383BDE8F88F616A5F
:10EED0003268A1EB0208B8F1010F06D4C2F10100BB
:10EEE000C31A0B44002B40F3BF81531A002BC0F20E
:10EEF000B681208D02F1010CACEB01031B1A002B33
:10EF000039DC914200F05084656F002D00F0598388
:10EF1000E86843689A424FF0000802F1FF3E19D0BA
:10EF2000B8F1000F00F02E81D8F80C104968AEEB54
:10EF30000101002904DBACEB0301002940F34A8303
:10EF40002968A846002900F029810D46E868436831
:10EF50009A42E5D183482B8902899A420BD9FEF760
:10EF600097FE40B1B8F1000F00F0F583C8F800003B
:10EF70002946FFF7B9FE2046BDE8F84F02F0F0B988
:10EF8000636D3268B4F860E0D4F858C0991A00296B
:10EF90007FDB754D93422B6800F0CD809C4500F0DF
:10EFA000D380D4F84480A3EB080000287146E146E2
:10EFB00040F38680226D9A1A002A00F38D80628BBE
:10EFC00057070AD5B4F84A10A4F8481022F00402F2
:10EFD00092B200216283A4F86A10B4F93C10636411
:10EFE000E38F03EBE103A4F84030237D0021032BE2
:10EFF000A4F8421013D9B4F84830B4F84A10994232
:10F0000080B200F2C981B4F86A20104480B2824212
:10F0100000F2BE82834240F2BD82A4F86A00D4E9C5
:10F020001B212046FFF7BCFEE16E2067024620460A
:10F03000FFF7B6FE226FE066B2FA82F35B095B422D
:10F04000238600232377002800F0A381474B1988EB
:10F05000B4F864300B44A4F86430638B19053ED5D2
:10F06000002A00F0AF81D368E76C5868FCF77AFBA0
:10F07000381A002833DC638B394F23F40063638331
:10F080002EE03B4B3B493C4840F27C420CF00AFBF3
:10F0900000E73A4B344D1B68D9892B68B4F86200FD
:10F0A000D4F84480A4F860108842A3EB080038BF6D
:10F0B000A4F862100028C4E9152399463FF77AAFF7
:10F0C000274F388820B94944E644714500F08A81C9
:10F0D000002384F8433003E0204602F041F9204F3A
:10F0E000616B00293FF4DCAE2B68A26BD21A002AB8
:10F0F000BFF6D6AE224BB4F93C201D88C2F3CF0038
:10F1000089B22B1A5B1A9BB21A4412B213F4004F45
:10F11000A28702D0401B01448BB2B4F93E10A1EB90
:10F12000A1010B449BB203EBE202E3870023A4F8A6
:10F1300040206363B4E6ACEB03010029BFF62EAFB9
:10F140000E490968C989A9E70C490968C9898E452A
:10F15000BFF427AFA2E700BF000A0120200A012068
:10F160003A0A0120040A0120FC090120140A0120A6
:10F17000E40B0208C00C020808F301082C0A012065
:10F18000F0090120D11A0029BFF6DAAEAC48FEF72B
:10F190007FFD00283FF4EFAE6067E9E6D31A002B4D
:10F1A0007FF7E9AE8089FCF7D9FAC1073FF5E3AEF6
:10F1B000A348FEF76DFD286000283FF4DCAEEB6845
:10F1C0002A89596833680A44D21A002A05DD5B1A75
:10F1D00099B268682981FDF773FD32683B88134452
:10F1E000626A9B1A228D9B1A002B7FF7C4AE2B6894
:10F1F000DB689889FCF7B2FAC2072B6800F1C2827B
:10F20000218D32685868891A626A114489B219815D
:10F21000FDF756FD2B681D89DB689889FCF79EFA7F
:10F2200010F0030018BF01203168228D2B189BB20B
:10F2300019443B80636A134499423FF49CAE814B6E
:10F24000814982484FF4DF620CF02CFA93E67D4B43
:10F250007F497E4840F27B420CF024FA16E6638B2D
:10F2600043F00203638386E6DFF8D491D9F80450B3
:10F27000002D00F085814FF6FE73984500F2D8808E
:10F28000D9F804301A891FFA88F84245C0F0C580C1
:10F29000B9F80830A3EB0803A9F808306B89A2EB92
:10F2A0000802434592B20AD2002169812A812D6861
:10F2B000A8EB03031FFA83F86B894345F5D3414656
:10F2C0002846FDF759FBD9F80C20636A3360536078
:10F2D000238D002B3FF44FAE13469889B9F80850A0
:10F2E000FCF73CFA10F0030018BF0120228D2B1808
:10F2F0009BB29A423B80C0F09781636F002B00F075
:10F30000B680D9F80C309889FCF728FAC20700F1CA
:10F31000AB80656F55B90AE2D5F800802846FEF744
:10F32000A9FC4546B8F1000F00F00182E8683A8870
:10F33000D6F800E02B89D0F804C002EB0E0163443C
:10F34000CB1A002BC0F2BB818089FCF707FAC307F8
:10F35000E2D5D9F80C309889FCF700FA8007DBD4A5
:10F36000D9F80C300120B3F80C80FCF7F7F9D9F884
:10F370000C3048EA0000988180B2B9F80880FCF7A8
:10F38000EDF910F0030018BF01208044A7F80080B9
:10F39000C2E7A4F8680059E612F4006F628E14BF49
:10F3A0000121022112FB01F292B2824294BF99180C
:10F3B00019188AB2934240F2F6804FF6FF73A4F810
:10F3C00048302CE648B1C368E76C5868FCF7CAF9C6
:10F3D000381A00283FF783AE638B1E4F23F4006377
:10F3E00063837DE6B4F930100029FFF671AE9845CD
:10F3F0007FF46EAE94F84310FF2900F05081013184
:10F40000C9B2032984F8431000F2498100F0538106
:10F41000616B00297FF469AE48E50A4B0E490B4841
:10F4200040F297520CF03EF9D9F804301A892FE7D0
:10F43000044B0A49054840F295520CF033F91FE796
:10F44000040A0120E40B02080C0D020808F301086D
:10F45000A40C02083A0A0120FC0C0208EC0C020879
:10F4600003686367FEF706FC606F0028F8D13A88EE
:10F4700031681144238D61629342C0F0CB809B1AA6
:10F4800023852046FEF764F8D9F804301A8922B1A2
:10F49000B24A13600023C9F80430D9F80C309889B7
:10F4A000FCF75CF9C20704D5AD4A137843F020039A
:10F4B0001370656F002D7BD0DFF8AC92DFF8C0824F
:10F4C000A84F33E0EB68B5F808A09889FCF746F937
:10F4D00010F00300238D18BF012050441B1A238510
:10F4E0002046FEF735F869680B893BB19B4B1868DD
:10F4F00000285BD0FDF78EFC00236B60EB689889D9
:10F50000FCF72CF9C30709D5954A217D1378042906
:10F5100043F02003137004BF072323752B68636730
:10F520002846FEF7A7FB656F002D41D0EA68616AA7
:10F5300053688B423CD133609089B5F808A0FCF742
:10F540000DF9636AB5F808B010F0030018BF012088
:10F550009A445044EB6860629889B4F828A0FCF79C
:10F56000FDF810F0030018BF012058448245A9D2CD
:10F570004B4640F22B62414638460CF093F8A1E727
:10F58000794B7A49774840F294520CF08BF872E646
:10F590004FF6FF70628E1A4492B2C01A9342A4F8DA
:10F5A0006A003FF60AAFA4F8482038E51960A3E7DF
:10F5B000638BD8070AD523F0010343F0020363836A
:10F5C00083E46B48FEF764FB6067D4E443F0010317
:10F5D00063837AE46648FEF75BFB074600283FF446
:10F5E000CAACD8F80C3032685968B8F808300B4407
:10F5F0009B1A002B07DD521A91B2D8F80400A8F824
:10F600000810FDF75DFBC8F8007029463846FFF783
:10F610006BFBB0E4544B5749524840F207620CF080
:10F6200041F8238D3A882AE7D9F80C309889FCF7FD
:10F6300095F8C507D9F80C307DD49889238DA9F8A1
:10F640000830FCF78BF8B9F80810800744BF01F1C7
:10F65000FF3189B2D9F8040048BFA9F80810FDF7B6
:10F660002FFBD9F80C30B9F808509889FCF776F8D8
:10F6700010F0030018BF01203268616A2B189BB29A
:10F680003B801344228D0A4493423FF436AE364BFE
:10F690003949344840F2CB520CF004F82DE6B4F866
:10F6A0004820638E13449BB24FF6FF719A4288BF85
:10F6B0000B46A4F84830204601F08CFD10E5A1EB84
:10F6C0000C03002B01DC6567D4E6D9F80C30ACEBF9
:10F6D0000E0CA9F808C09889FCF740F8810704D5FA
:10F6E000B9F80830013BA9F80830B9F80810D9F882
:10F6F0000400FDF7E5FAD9F80C30B9F808809889CC
:10F70000FCF72CF810F0030018BF012008EB0002F2
:10F71000EB6892B23A805968336813448B42D2D076
:10F72000114B16490F4840F2FC520BF0BBFF3A88D0
:10F7300031681144C7E79D892846FCF70FF800F0AF
:10F740003E00FCF70BF825F47C55D9F80C30284323
:10F75000988180B272E760670AE400BF180A01204E
:10F760001C0A012008F30108E40B0208DC0C020863
:10F77000040A0120800D02080C0D0208440D020845
:10F78000A00D0208DB68B3F80C804046FBF7E6FFEB
:10F7900000F03E00FBF7E2FF2B6828F47C58DA68A3
:10F7A00040EA080090812BE5DFF80890D9F80C308A
:10F7B00093E500BF040A01202DE9F04F044687B00D
:10F7C000002800F0D68063896D4E62683260132B8A
:10F7D00005D8204607B0BDE8F04FFDF74FB9694F97
:10F7E0003968786908F014F805460028F1D17B697A
:10F7F00003F0F003E02BECD033689889FBF7AEFF01
:10F80000800A00F0FC011329E3D923898B428AB2D4
:10F81000DFD36089DFF8A091DFF8A081A2F11403A3
:10F820009BB29042C8F80050A9F8003080F09A814D
:10F830002368002B00F0748314212046FDF79CF808
:10F840006589514BB9F800A01D8029462046FDF777
:10F8500093F82068AAEB050943891FFA89F94B45FB
:10F86000B7D34368C8F800304946FDF785F82389C7
:10F8700062892B44A3EB0A039BB22381002A40F048
:10F880005683226812899A4205D0404B404941482C
:10F89000E0220BF007FF35682888FBF75FFF288020
:10F8A00035686888FBF75AFF688035686868FBF739
:10F8B00059FF394B686035681860A868FBF752FF3C
:10F8C000364BA86035681860E889FBF747FF336856
:10F8D000E8819889FBF742FF314A00F03F03800737
:10F8E0001370228940F044812E4B05931A802E4BD1
:10F8F0001D68002D00F0E580DFF890A0DFF8C0B0B3
:10F90000DFF890904FF0000817E00A2B21D0012B70
:10F9100028D02A7A32B17B6893F840300133DBB2C9
:10F920009A4204D13368298B1A8891424AD0EB68F5
:10F93000A846002B00F0C5801D462B7D002BE4D18E
:10F940005346FB22594648460BF0ACFE2B7D0A2B52
:10F95000DDD153461549FC2248460BF0A3FE2B7D12
:10F96000012BD6D112495346FD2248460BF09AFE90
:10F97000CFE7064B0F49074883220BF093FE22E79F
:10F980002C0A0120ECD00020300A0120E40B0208F0
:10F99000FC0D020808F30108200A0120FC090120DF
:10F9A000000A01203A0A0120E0090120440E020861
:10F9B000700E0208C80D0208380A0120340A01201E
:10F9C0001C0E02085B88EA8A9A42B0D16A683B69D9
:10F9D0009A42ACD12A687B699A42A8D1EB68AB42C3
:10F9E00000F04E84B8F1000F09D06E4AC8F80C3010
:10F9F0001368EB601560EB68AB4200F04F846A4B14
:10FA00006A4FDFF8C081DFF8C091DFF8C0B11A7823
:10FA10007C6000233B60C8F8003089F80030ABF808
:10FA2000003023893B813368FB60130703D5637B78
:10FA300043F001036373AB6F73B12846FEF778FEA2
:10FA40000D3000F07C82AB6F23B1059B1B88002B2F
:10FA500040F07582544B1A78554C5107256040F19F
:10FA60005181297D022900F03683524B6A6A1B6856
:10FA70009A4200F02E849B1A04D42A8D9B1A002BE4
:10FA800040F3248399F800301A0740F17882D5F8C2
:10FA900090301BB128696FF00D0198474148294605
:10FAA000FEF7B4F92846FDF7ADFC7868002525601F
:10FAB000C8F8005010B1FCF7E1FF7D6007B0BDE869
:10FAC000F08F3D4B1D68002D5BD0DFF80481DFF81F
:10FAD00004B1DFF8049102E0ED68002D51D02B7DD8
:10FAE0000A2B434605D040F21F12594648460BF0F8
:10FAF000D9FD2A7A32B17B6893F840300133DBB20A
:10FB00009A42E9D132682B8B11888B42E4D152881A
:10FB1000E88A9042E0D169683A699142DCD129686B
:10FB20007A699142D8D1204A127851073FF551AEF7
:10FB3000970740F1C7831F4A696A1268511A04D4B3
:10FB40002E8D891B002940F3D383059B1B88002B36
:10FB50003FF43FAE6B8B43F0020328466B8301F00A
:10FB600055FC36E6154A20461380FCF705FF92E661
:10FB7000531C134905919BB29A420B807FF6B7AE96
:10FB800027E6DFF85890D9F80080B8F1000F00F0B0
:10FB9000378378683168D7F814C045460022A246FA
:10FBA00024E000BFE0090120000A0120040A01202E
:10FBB000240A0120200A0120F8090120300A01202E
:10FBC0003A0A0120180A01201C0A0120140A012007
:10FBD000E40B0208F00E020808F30108EC0901200A
:10FBE000EB682A46002B00F0B0811D462C7A2CB120
:10FBF00090F840300133DBB29C42F1D1B5F816E009
:10FC00004B889E45ECD1D5F800E0E64502D0BEF128
:10FC1000000FE5D154462AB1E868D060C9F8005019
:10FC2000C5F80C80A84A127850073FF5D2AD12F003
:10FC3000100840F0738290077FF5CBAD687DFEF72A
:10FC40005DFA8146002800F0DD82D7E904239F4F4A
:10FC50003168C0E900323B680A784978013342EAEA
:10FC60000122E98A4362C3620323C18202830375CE
:10FC7000FEF7C4FE3B68C9F85000013BC9E91530E6
:10FC80002B69C9F84400C9F85C00C9F87C50C9F870
:10FC900010306B7A8E4A03F00C0389F809302B7A06
:10FCA00089F808301368C9F80C30C2F8009001F0E8
:10FCB00029FF884B012248461A70FEF755FF32682B
:10FCC000B9F83250D289434662F30F0362F31F43FF
:10FCD00009F10402C9F860301046059207F05CFB98
:10FCE000059A01462846FEF7A5FE1221A9F8320022
:10FCF000484601F037F9002840F08F82484601F06D
:10FD000085FB66E5930704D52B7D023B012B00F2B2
:10FD1000DD816B8BD80602D46F4B1B682B620023EE
:10FD2000A5F89A302846FEF71FFF2B7D023B072BD4
:10FD30003FF6A8AEDFE803F03413048F7404A85B29
:10FD40002846FFF79DF899F8003099067FF59AAE9E
:10FD50006B8B43F002036B8307232B7592E65A4BA0
:10FD60001B78DA0640F138825C4B19686B6CDB4318
:10FD7000CB4204D42B6DCB1A002B40F35482059A4E
:10FD800033681088514A12680244188802905B88D0
:10FD90000193534B00932846043301F055FA71E662
:10FDA000494B1A7802F01203122B00F03581D1066C
:10FDB0007FF568AE059A33681188444A188812683E
:10FDC0000A444649096802905B880193444B0093BA
:10FDD0002846043301F038FA95F84230052B3FF6F7
:10FDE00051AE00232B86284601F00EFD4AE6284638
:10FDF000FFF746F8344B1B78D9067FF543AE374BF7
:10FE00002A6D1B689A427FF43DAEEB6E002B7FF4A7
:10FE100039AE99F8003043F0100389F8003031E62C
:10FE20002846FFF72DF899F800309E067FF52AAE98
:10FE30006B8B43F002036B832846FDF7D1FF244B05
:10FE40001B68AB425DD0002B5ED0DA68AA4200F09E
:10FE50002E821346F7E72846FFF712F899F800308C
:10FE600013F0200F184B1B7800F08D81DA0604D5B3
:10FE70001A4B2A6D1B689A4234D06B8B43F00203F5
:10FE80006B8308232B75FDE52846FEF7F9FF0E4B23
:10FE90001B78D8067FF5F6AD104B2A6D1B689A4289
:10FEA0007FF4F0ADEB6E002B7FF4ECAD2846FDF750
:10FEB00097FF074B1B68AB4223D02BB3DA68AA42EB
:10FEC00000F0F5811346F8E7000A0120200A01201E
:10FED000E0090120E4090120F0090120FC090120CA
:10FEE000FCD00020EB6E002BC7D16B8B43F00203DC
:10FEF0006B832846FDF774FFAB4B1B68AB4240F0A9
:10FF0000D981A94AEB681360A84BA94A19681D60FA
:10FF10000A232B75E9600123137001F0F3FDB1E5AD
:10FF2000A44BA549A548C2220BF0BCFB84E4A14B1D
:10FF3000A349A248DF220BF0B5FB2389A1E46B8D16
:10FF4000002B00F0E7809F4CAFE554468889FBF713
:10FF500005FC10F004007FF43CAC059A336811886E
:10FF6000994A1D8812680A449849096802955B8875
:10FF70000193974B0093043301F066F929E4BBF831
:10FF800000206AB1D5F880603EB128692946B047A3
:10FF90000D303FF48AAD99F800300022ABF8002014
:10FFA000DE0600F1A980D8F80020002A00F0C88001
:10FFB000AB6F43B14FF4F3727E4B86497F480BF031
:10FFC00071FBD8F800206B8B13F0100340F0D48045
:10FFD000D5F88460002E00F00D8128692946B047CD
:10FFE00010F10D0F3FF461AD10B1D8F80030AB67E0
:10FFF00099F80030980607D5AA6F002A00F0A6806D
:020000040801F1
:10000000517B41F0200151730022D906226073D444
:10001000284601F0FBF948E56C496B6C096801332F
:100020008B427FF4C4AE6B64674B31681B686E8E85
:100030005A1C6A62EA62CA89013B6B65002362F35B
:100040000F0362F31F432B662A1D04232B751046F2
:10005000059207F0A1F9059A01463046FEF7EAFC41
:1000600041F21C1342009A42164638BF1E46B6EBB8
:10007000800F68864FEA800140F269818BB2A5F853
:100080004830B5F86630002B00F05981B5F866307D
:100090002E6F013BA5F86630002E00F04B813368CF
:1000A0002B673046FDF7E6FD2B6F002B00F03F81FC
:1000B000002385F842302B86D5F8883033B1286983
:1000C0000022294698470D303FF4EFAC6B8B43F08C
:1000D00002036B83D6E43D4B2A6D1B689A427FF482
:1000E000D1AC99F8003043F0080389F800306B8BED
:1000F00023F001036B83C5E46B8BDA063FF5CEACCE
:10010000D5F89030002B3FF4C9AC28696FF00E0190
:100110009847C3E4284601F023F914E7059A0988B3
:100120001088294A12680291284909680193284BCE
:10013000009302440433284601F086F8FFF749BBD8
:1001400013F020027FF458AF226061E72A8DD5F8C2
:100150008460B2F5066F1CBF01322A85002E3FF481
:1001600053AF002328691A462946B0470D303FF4A3
:100170009CAC99F8003047E71046FCF77FFC284616
:10018000FDF7B8FF91E4DB067FF57CAC0F4B2A6DE1
:100190001B689A427FF476ACEB6E002B7FF472AC56
:1001A00006232B756EE400BFE0090120F809012049
:1001B000E4090120E40B0208E00D020808F301083D
:1001C000F00D0208240A0120200A0120FC09012068
:1001D000FCD000208C0F020898077FF553AC624BCF
:1001E0001A686B6A013B93427FF44CAC284600F0DE
:1001F000ABFF47E4334630462946FEF71DFAEFE6EB
:100200003168A3E6AB69002B3FF4E3AA28694FF0FD
:10021000FF3249469847FFF7DCBA41464846FDF7AA
:1002200079FEFFF7D6BAEB6F04222A75002BA6D011
:100230009B69002B6FD02869002229469847002827
:1002400065D12846FEF71CFEBBF8003013B1013B18
:10025000ABF80030698E41F21C134A009A421646F0
:1002600038BF1E46B6EB810F4FEA81003CD983B2FE
:10027000A5F8483099F800309E067FF503AC67E595
:100280003A4B3B493B4840F20D120BF00BFAB8F1E8
:10029000000F3FF4B0ABEB68FFF7A7BB334B364919
:1002A000344840F215120BF0FDF9FFF7A8BBEA68DD
:1002B000DA6029E6002B3FF427AEDA68AA42F6D0CE
:1002C0001346F7E7D6077FF540AC2C4B1B682B6233
:1002D0003BE400297FF405AF244B294925484FF41E
:1002E0004E720BF0DFF9FCE69A4288BF93B2BFE78B
:1002F000CDE90103059B1B881A44224B1968224B48
:1003000000932846043300F09FFFFFF762BA0D30D8
:100310003FF4CBAB33E7154B1C4916484FF46A72D8
:100320000BF0C0F9EB6F9B69002B84D127E74FF0EE
:10033000FF33C0E6EE6E76B13368EB66B1E60B4B89
:1003400013490C484FF45B720BF0ACF99EE69A42ED
:1003500088BF93B293E6054B0E4906484FF45D7291
:100360000BF0A0F9E8E700BF200A0120E40B020827
:10037000980E020808F30108C40E0208F0090120D3
:10038000200F0208FC090120FCD000206C0F02089D
:10039000400F0208580F0208024A137843F0100376
:1003A000137070471C0A01202DE9F84F0A9F9DF831
:1003B0002CA09DF830B0002661F30F060C46814654
:1003C0001546984661F31F46002F33D0AC420ED23B
:1003D0001AF0020F08D004F21B2121F00301A942F8
:1003E00028BF294689B203E07B8B5B0618D52146DE
:1003F00048464FF42072FCF7B3FB054668B103682A
:1004000033B1104B1049114840F20B120BF04AF96E
:100410006B891B1BA8F80030AE602846BDE8F88F3A
:10042000BBF1000FD7D0FB6E002BD4D13B6F002B5C
:10043000D1D1DCE7034B06490448E9220BF032F93D
:10044000C4E700BFA80F0208FC0F020808F3010868
:10045000DC0F02082DE9F0470E469DF820A09046DB
:100460009946074600284AD0002E50D00320FBF7BB
:10047000CBFE4FEA8A0505F004050446002854D057
:1004800080F80AA0328946600023AA4203601FFA5E
:1004900085FA2CD3A2EB0A02304622811421FCF704
:1004A0003BFA0646002839D16368F88AD3F804A0DD
:1004B000C4F80CA0FBF752F9AAF80000388BE768E3
:1004C000FBF74CF978804846E768FBF74BF9AD023B
:1004D00005F5A045786045EA0800E568FBF73EF9B8
:1004E000E368A8819E74DE742046BDE8F087B022E0
:1004F000104B114911480BF0D5F83289CAE70D4B62
:100500000F490E48A3220BF0CDF8002EAED1094BB7
:100510000C490A48A4220BF0C5F8A7E7204600249E
:10052000FDF7A8FB2046BDE8F0873046FCF7A6FAA9
:10053000DAE700BFA80F02085410020808F3010808
:1005400010100208301002082DE9F0470D4617463A
:10055000044600283ED005F1140189B24FF4207200
:100560002220D4F82490E58AB4F818A0B4F82A80A0
:10057000FCF7F6FA064610B34389132B22D9284616
:100580007568FBF7EBF828805046FBF7E7F86F60DB
:1005900068804846FBF7E6F8A86045F21000FBF7D4
:1005A000DDF8A8814046FBF7D9F80023628D2B7453
:1005B0006B74AB74EB74636AE8811344E362304696
:1005C000BDE8F087074B0849084840F223720BF05A
:1005D00069F8D4E7034B0649044840F242720BF035
:1005E00061F8B8E7A80F02089410020808F30108A0
:1005F0006C1002082DE9F04F91B000240791099387
:10060000ADF83E40002800F01383B0F86230914608
:10061000428E5B08934228BF13469B46002B08BFBF
:100620009346079B8046002B00F0EF82037D072B4B
:1006300007D0023B022B04D96FF00A0011B0BDE8CD
:10064000F08FB9F1000F00F0CA80B8F864304B4564
:10065000C0F0CE82B8F86660082E00F2C982D8F8E1
:100660007030002E00F0B180002B40F0BA80D8F836
:100670006CA0BAF1000F00F0958253461A461B6831
:10068000002BFBD1947A0C929A46A400138904F0B3
:1006900004041A199345C0F21D82ABEB0404E41A5A
:1006A000A3B20A93B8F868300B93ADF83E30002B34
:1006B00040F0B080B9F1000F00F0B4810A9A002A2E
:1006C00040F04281099B0B9C03F00107FBB20893A9
:1006D0000023CDF834A005939A4642E0BDF83E30A1
:1006E000002B40F0A981012229463620FCF738FA78
:1006F000002800F0B981079A069022444260002148
:100700004FF420723620FCF72BFA069B0746002890
:1007100000F0EA811946FCF77DFB3846FCF750FBF8
:10072000304486B2092E4AD8D8F85C3000223946C7
:10073000234400924046FFF78DFE0746002800F054
:100740009381059B002B00F07581BAF1000F00F03A
:100750007B81CAF800702544ACB2A14540F27C828E
:10076000BA46A9EB0405ADB25D45089B28BF5D46BE
:10077000ADB2002BB2D0099BCDE90083059BB3FA43
:1007800083F35B0902935A460DF13E032946362056
:10079000FFF70AFE0746002800F066814389AB4256
:1007A000C0F05A81079B78682A4619190BF01AF98C
:1007B0003846FCF705FB304486B2092EB4D93846DA
:1007C000DDF834A0FCF75AF950E1002B00F0AA80C4
:1007D000B64BB749B7484FF4AC720AF063FFB8F8AC
:1007E0006660D8F86CA0BAF1000F7FF446AFB8F895
:1007F0006830002B40F0A080B9F1000F00F0248297
:100800000023CDE90A331C460C939A46099B03F05A
:1008100001075BE70A9A934200F2F9800A9A0B9B60
:100820004A45174628BF4F469F4228BF1F46BFB2C2
:10083000DB1BD21B9BB292B2ADF83E300A92002B6A
:1008400000F0E080B94540F0D6800C9B002F00F00E
:10085000EA8000250C9C0A95D4F804B0BBF1000F87
:100860002AD0BBF808300595DBF800103D462B4434
:100870002746ABF80830079C49B18B46BBF80830D7
:10088000DBF800102B44ABF808300029F5D1BBF899
:100890000A30DBF80400214618442A460BF0A2F87F
:1008A000BBF80A30DBF800102B44ABF80A30002903
:1008B000E3D13C462F46059D23893B442381BDF867
:1008C0003E30A8F86830002D00F037816068294676
:1008D000FCF7A0FA2A89238913442381C4F800A0D5
:1008E000D8F85C30A8F866604B44C8F85C30B8F8BB
:1008F0006430A3EB0903A8F8643026B1D8F870304F
:10090000002B00F00D810C9B002B00F05581D86866
:1009100000283FF493AE099B13F0020400F0F68028
:1009200000208BE6D8F86C30002B7FF451AFB8F87C
:100930006830002B3FF464AF5C4B5F495D4840F288
:100940004A220AF0AFFE57E70C9B1B89002B00F0F0
:10095000DB800B9BA9EB03039342A8BF13460593CF
:100960009CB2099BD90703F0010700F105810C9B9C
:100970005D682B462D68002DFBD11A7B12F0C00F4D
:1009800006D15A895B681344079A9A4200F039816C
:10099000012221460020FCF7E3F80546002800F07C
:1009A0002081079B0B9A13444360FCF709FA00234C
:1009B000304486B20A930B9B1C44A4B2A14588BF65
:1009C000AA463FF683AE0C9C1F460B9B002B7FF480
:1009D00043AFBDF83E30A8F86830002D00F0EE803F
:1009E000002C7FF473AF314B344932484FF43872E6
:1009F0000AF058FE6AE72D4B31492E484FF4007239
:100A00000AF050FEB9457FF620AF0B9756E6274B0C
:100A10002C4928484FF4FC720AF044FEBDF83E30E1
:100A20000B93FBE64B460C9C0C93BDF83E30A8F8AC
:100A3000683053E705908EE61C4B23491D4840F271
:100A400071220AF02FFE4EE62049184B194840F259
:100A5000AB220AF027FE7CE61D49144B154840F2F4
:100A600066220AF01FFE9DE6DDF834A0B8F81A30C1
:100A700043F08003A8F81A30BAF1000F02D05046B4
:100A8000FBF7FCFF059B13B11846FDF7D7F8B8F844
:100A900066302BB1D8F8703013B9D8F86C304BB33E
:100AA0004FF0FF3011B0BDE8F08F00BFA80F020873
:100AB0004C11020808F301080412020898120208F7
:100AC000B811020898110208741202088412020870
:100AD00034120208644B654965484FF4F3720AF01A
:100AE000E1FD0C9B1B89D8E51846DDF834A0FBF727
:100AF000C5FFBBE75C4B5F495D4840F227320AF017
:100B0000D1FD4FF0FF3099E50A93DBE58589082098
:100B1000FAF724FE0C9BDB682843988120468DE57C
:100B2000D8F86C30002B7FF4EEAE4F4B5149504853
:100B300040F212320AF0B6FDE5E60A9B002B3FF4C4
:100B4000CDAE616800293DD00A68002A7AD00A9D9E
:100B500000E002460B8910682B440B8111460028E7
:100B6000F7D10A9913890B44138153890B4453819C
:100B700023890B442381B1E6CDE90083012302934D
:100B800021460DF13E030020FFF70EFC054640B361
:100B9000079B0B99BDF81420406859180AF022FFF2
:100BA000284602E7304B3449314840F255120AF0EA
:100BB00079FDB8F8666014E618463FE50A9B53B124
:100BC000002CBED12D49284B294840F2E6220AF0DC
:100BD00069FD6168B8E7002C7FF480AEC8F86CA0AE
:100BE0007EE6B8F81A3043F08003A8F81A304EE7D2
:100BF000B8F81A3043F080034FF0FF30A8F81A30ED
:100C00001CE50B9B5BB90A94D5E6174B1C491848A9
:100C100040F2AD120AF046FD6FF00F000EE5124BE8
:100C20001849134840F231220AF03CFD0A94C2E60A
:100C30000D4B15490E484FF4CF720AF033FD6FF09B
:100C40000F00FBE40A468CE7BDF83E30A8F8683098
:100C5000CA46CDF83090C1E7DDE90C4A0C975546FD
:100C60000B9FDDF814A0B0E6A80F0208801102085F
:100C700008F301080813020810110208D012020834
:100C8000DC100208D8110208C41002082DE9F04F48
:100C90000C4683B00546002800F0A880EE6E76B3BF
:100CA000002C00F0B480B6F80890A14540F29A807C
:100CB0006B8EA34228D396F80AA0A9EB04084FEA4A
:100CC0008A0B1FFA88F80BF0040B08EB0B0189B2B2
:100CD0004FF420723620FBF743FF074678B1706867
:100CE0003289038979689B1A23449BB2594442464E
:100CF000FCF7D4F940451DD03846FBF7BFFE4FF056
:100D0000FF3003B0BDE8F08F464B4749474840F2FB
:100D10005B320AF0C7FCB6F80890B9F1000FCAD1EF
:100D2000404B434941484FF457720AF0BBFCB6F8B8
:100D30000890C0E7F3689889FAF710FD10F0080BE7
:100D40005FFA80F85AD108F03F08012318F0010F2C
:100D500018BF9B46F368586818BF08F0FE08FAF7FA
:100D600001FDCDF800A023185A4639462846FFF762
:100D700071FB82460028BFD07068FCF721F87268CA
:100D8000B5F866301189A4EB0904A4B21B1A2144FA
:100D9000104689B2A5F86630FBF792FF33891C44F0
:100DA000F368348140469C89FAF7D8FCF368044321
:100DB00070689C81FCF704F8B5F866300344DAF8F3
:100DC0000400A5F86630FBF7FBFFB5F86630184461
:100DD0003368A5F86600CAF80030C6F800A0DAF853
:100DE000000088B1002003B0BDE8F08F0D4B114921
:100DF0000E4840F24B320AF055FC4FE708F0370836
:100E000009234FF0080BA1E7A5F8680079E7054B27
:100E10000949064840F253320AF044FC6FF00500DD
:100E20006FE700BFA80F02087013020808F301085B
:100E300080130208281302084C130208F0B5054677
:100E400083B0002858D0EC6E4CB126462468002CA4
:100E5000FBD1F3689889FAF781FC420754D000214E
:100E60004FF420723620FBF77BFE0146002866D047
:100E70000022EB6D009228460122FFF7EBFA0446B0
:100E800000285CD0C3689B072ED1238903BBEB6E7F
:100E900043B31A461B68002BFBD11460EA6D6B8BC1
:100EA000606843F02003013200266B83EA65A5F8F1
:100EB0006860FBF785FFB5F86630C418A0B2A5F8E6
:100EC000660018B1286F00282DD0304603B0F0BD61
:100ED0001E4B1F491F4840F243420AF0E3FBEB6EF2
:100EE000002BD6D1EC66D9E7184B1B49194840F2C4
:100EF00042420AF0D7FBC8E7144B1849154840F2A4
:100F0000EB320AF0CFFB9EE7F36801209F89FAF7E6
:100F100025FC6B8BF2683843908143F02003204618
:100F20006B8303B0F0BDED6E002DCFD1074B0C49A4
:100F3000084840F265420AF0B5FB2846C6E76B8BCD
:100F400043F080034FF0FF306B83BFE7A80F020828
:100F5000C413020808F30108AC1302089013020836
:100F6000F01302082DE9F04111F0030782B00D469D
:100F700004465ED0002C65D015F002084FF42072B4
:100F800049D004213620FBF7EBFD0646002849D066
:100F90004389032B72D8414B4149424840F23942C0
:100FA0000AF080FB4FF00108CDF800803146E36D78
:100FB0002A462046FFF74EFA0646002832D0C3687C
:100FC0009A0753D13389002B44D1E36E002B4BD0C9
:100FD0001A461B68002BFBD116600023A4F868306A
:100FE00017B1E36D0133E365EB0703D5638B43F082
:100FF000200363837068FBF7E3FEB4F8663018449F
:1010000080B2A4F8660018B1206F002839D0002003
:1010100002B0BDE8F08141463620FBF7A1FD06464F
:101020000028C1D1638B43F080034FF0FF3063830E
:10103000EEE71A4B1C491B4840F211420AF032FB02
:10104000002C99D1154B1949164840F213420AF069
:1010500029FB91E7114B1649124840F243420AF02E
:1010600021FBE36E002BB3D1E666B6E70B4B1149CB
:101070000C4840F242420AF015FBA3E74FF001088A
:1010800092E7E46E002CC3D1044B0B49054840F2B3
:1010900065420AF007FB2046BAE700BFA80F020826
:1010A0009014020808F301081814020870140208CA
:1010B000C4130208AC130208F0130208F8B5054681
:1010C000002832D0296F39B10C6864B10A465368E0
:1010D0009B7B012B224602D06FF00500F8BD2368F0
:1010E00013B11C46F3E70C4663689B7B012BF3D1DD
:1010F0006B8BEA6E2260002643F400636B83E36827
:10110000C5E91B165868FAF72DFBE36824890746E2
:101110009889FAF723FB10F0030318BF0123274433
:101120003B44EB646E633046F8BD044B044905480C
:1011300040F263620AF0B6FAC4E700BFA80F0208E3
:10114000CC14020808F30108F8B50746002832D08D
:101150003E6F56B373689B7B012B26D1FB6E3268C2
:101160003A6707F16C051BB90FE02D682B6863B176
:10117000DB685868FAF7F6FAF36804465868FAF735
:10118000F1FA241A002CF0DB2B6833602E603368F0
:1011900073B197F84230FF2B18BF01334FF00000B6
:1011A00018BF87F842307863F8BD6FF00500F8BDCE
:1011B000A7F86830EDE7044B0449054840F2C162E6
:1011C0000AF070FAC4E700BFA80F0208F014020882
:1011D00008F3010810B5044638B3236F13B1638BCD
:1011E0005B0700D510BD2046FFF7AEFF0028F9D100
:1011F000B4F86010B4F84830628E994228BF19469E
:1012000050004B08B0EB510F618BA4F84A300244F8
:1012100084BF83B2A4F84A30134441F00402002191
:10122000A4F848306283218610BD044B0449054868
:1012300040F2F9620AF036FACFE700BFA80F0208C1
:101240000815020808F301082DE9F04F85B006469D
:10125000DDF838A0BDF83C40BDF840B00D469046E2
:101260001F46002B59D0BAF1000F60D02846FAF77C
:1012700079FA4FF42072814614212220FBF770FC8A
:101280000546002846D04389132B36D920466C6882
:10129000FAF764FA20805846FAF760FAC4F8049026
:1012A00060804046FAF75EFAA06045F21400FAF753
:1012B00055FAA08146F20800FAF750FA0023E081BF
:1012C00023746374A374E374002E38D0307AE0B9C9
:1012D000504606F061F850B1F37AB67A02900624CF
:1012E0000096524639462846019406F081F9284670
:1012F00005B0BDE8F04FFBF7C1BB144B14491548CE
:1013000040F223720AF0CEF9C0E7FBF771FA002829
:10131000E2D1ECE705B0BDE8F08F0C4B0E490D486B
:1013200040F2C4720AF0BEF9BAF1000F9ED1074B29
:101330000A49084840F2C5720AF0B4F996E75046E7
:1013400006F02AF80028D2D0FF23C7E7A80F02082A
:101350009410020808F30108281502084415020831
:1013600070B5044686B000283BD0206DFAF7FAF934
:10137000002102462046FFF7E7F80546002838D04E
:10138000207A221D40BB1046059206F005F8059A0A
:10139000B0B10621A37A0093CDE901102146E37A8A
:1013A000284606F025F906462846FBF767FB66B98E
:1013B000638B23F003039BB23046638306B070BD9A
:1013C0002846FBF75BFB6FF00306638B304643F068
:1013D0000303638306B070BD0592FBF709FA059A13
:1013E000D6E7074B0749084840F2EA720AF05AF973
:1013F000BBE7638B6FF0010643F00303DCE700BF3C
:10140000A80F02086015020808F301082DE9F04F43
:10141000044685B0002800F0B281237D012B00F046
:101420006981AE4B1B68A34200F07081E56EB4F891
:101430004860B4F8607025B3207A04F104090028EC
:1014400040F0A581484605F0A7FF8046B8F1000F9F
:1014500000F0AF81236813B9D8F804302360EB683B
:10146000BE42586828BF3E46FAF77CF92B89626C69
:101470009B1A1844B0420FD9B4F86030B34200F060
:101480004F81628B910700F1458122F080026283D7
:10149000002005B0BDE8F08F236F002284F899206A
:1014A000002B00F04D811F461B68002B00F0AF8021
:1014B0001F461B68002BF6D1A9E0EB681020B3F89B
:1014C0000CA0FAF74BF94AEA0000D5F80CA0AAF8EC
:1014D0000C006B689B7B012B54D1606AFAF742F9D0
:1014E000CAF80800608DD5F80CA0FAF737F9628DBC
:1014F000636AAAF80E001344E362AB7AD5F80CA035
:10150000DB0700F1C2800AF1140BB4F93030002B74
:10151000BCBF00232386636B002B00F0AB806868A0
:1015200043684189C0F804A0AAEB03039BB2C91A1F
:10153000418101890022CB1A03818AF810208AF8A0
:101540001120AB7A13F0010F14BF182314239A440F
:10155000D34507D06249634B634840F21C620AF0EE
:10156000A1F86868CDF80880A37A00930623019358
:10157000E37A4A46214606F03BF8002840F0148101
:10158000D5F80CA0237D2A68E266022B03D0638B7A
:1015900023F003036383DAF80400FAF7E3F8EB6857
:1015A000B5F808B082469889FAF7D8F810F0030326
:1015B000226DDA4418BF01235344D21A002AB8BF5F
:1015C0002365EB68B5F808A09889FAF7C7F810F01A
:1015D000030018BF012010EB0A0F44D0236F002234
:1015E0002A60002B43D0EB685868FAF7BBF8FB6819
:1015F00082465868FAF7B6F8AAEB00000028C0F255
:10160000A1803D602F46E56E002D00F0C480EB68A0
:101610005868FAF7A7F8636CC01A2B891844B042CF
:1016200000F2BB80EB689889FAF798F8420712D469
:10163000236F4BB1638B13F0440F1A4604D1E16E54
:10164000002938D0086888B3237D022B7FF435AF9A
:10165000D5F80CA03DE7234B2449234840F23652ED
:101660000AF020F8E4E72846FCF704FBCBE72567FF
:101670002F46C8E71E4B1B686363DAF80400FAF7CD
:1016800071F8D5F80CA0A06349E74A4641464FF4EB
:101690000670FDF7CFF940F00170FAF763F80AF130
:1016A000180BCAF81400D5F80CA02EE7B1F808C042
:1016B000608E8445C8D2B4F864000028C4D0B4F861
:1016C00066000828C0D813F0A00FBDD100297FF410
:1016D000DCAE0022A4F868201A46D6E6240A0120CF
:1016E000D8150208A80F020808F30108C01502085F
:1016F000F0090120304B3149314840F2E34209F012
:10170000D1FF304B1B68A3427FF490AE002005B0A0
:10171000BDE8F08F204605B0BDE8F04FFFF720BED2
:10172000236F002B7FF4ADAE94F89930002B7FF43B
:10173000A8AE4FF48072A4F8982084F89A30A0E6FE
:101740001F4664E7236F04F1700B2BB913E0DBF83D
:1017500000B0DBF8003073B1DB685868FAF702F8C4
:10176000EB6882465868F9F7FDFFAAEB00000028F5
:10177000EDDBDBF800302B60CBF8005043E70E4B7D
:1017800011490F4840F2E14209F08CFF45E6FBF7B2
:101790002FF880465AE6638B9BE7638BE16E1A460F
:1017A00000297FF472AE94E7638B43F08003638378
:1017B0006FE66FF003006CE6A80F020898150208A8
:1017C00008F30108240A01208015020810B5044618
:1017D00058B194F84230FF2B1CBF013384F84230DB
:1017E0002046BDE81040FFF711BE044B04490548F0
:1017F0004FF4D36209F056FFEBE700BFA80F0208D1
:10180000EC15020808F3010810B5044618B1FFF7FB
:1018100055FC98B110BD0F4B0F49104840F2AD6216
:1018200009F040FF2046FFF749FC0028F2D1094BA0
:101830000B490A484FF4D36209F034FF94F8423060
:10184000FF2B1CBF013384F842302046BDE8104016
:10185000FFF7DCBDA80F02081016020808F3010804
:10186000EC15020830B5044687B060B3206D01382E
:10187000F9F778FF002102462046FEF765FE05468F
:1018800048B3207A221DC8B91046059205F084FDA0
:10189000059A80B10621A37A0093CDE90110214673
:1018A000E37A284605F0A4FE04462846FBF7E6F84E
:1018B000204607B030BD6FF00304F6E70592FAF753
:1018C00097FF059AE5E7054B0549064840F62402CF
:1018D00009F0E8FECAE74FF0FF34E9E7A80F020875
:1018E0002C16020808F301082DE9F041044686B0E1
:1018F00000286DD0E56E002D45D094F89A30FF2B6E
:101900001CBF013384F89A30EB689889F9F726FFF9
:10191000C3073CD52989002939D1EB6820465A688C
:10192000FEF712FE0646002844D0D6F804801120A7
:10193000B8F90C70F9F712FF27F47C573843A8F870
:101940000C00EB685868F9F70DFF236D01301B1A86
:10195000002B00DA2065207A221D002833D11046A2
:10196000059205F019FD059A50B30621A37A00935C
:10197000CDE901102146E37A304605F039FE0546EF
:101980003046FBF77BF8284606B0BDE8F081EB68EF
:1019900001215A682046FEF7D7FD064650B1686817
:1019A0002A89038971689B1A9BB214310122FBF7C3
:1019B00075FBC6E74FF0FF35284606B0BDE8F0815D
:1019C0006FF00305DCE70592FAF712FF059ACBE703
:1019D000034B0449044840F64F0209F063FE89E7CF
:1019E000A80F02084816020808F3010870B504465B
:1019F0000A200E461546FAF707FC90B10D494460DF
:101A0000002303600B68C0E902651BB907E01946B3
:101A10001B681BB15A68A21A002AF8DA0360086032
:101A200070BDBDE87040044B04490548BE2209F072
:101A300039BE00BF400A01206C160208A016020839
:101A400008F3010838B5436804469847F4F7BCFB2F
:101A5000094B25681B6809492B441A1A002A22469B
:101A600004DA2844BDE83840FFF7C0BF1846BDE897
:101A70003840FFF7BBBF00BF3C0A0120451A0108F0
:101A800010B5FCF7D9FE174B1B68DBB1F4F79CFBD4
:101A900004460A20FA34FAF7B7FBD0B11249134BC7
:101AA00083600B68446000220260C2601BB907E0DB
:101AB00019461B681BB15A68A21A002AF8DA03609B
:101AC000086010BD0A4B1B68002BDFD1094A136068
:101AD00010BDBDE81040084B08490948BE2209F076
:101AE000E1BD00BFE0090120400A0120811A010880
:101AF000F8090120440A01206C160208A016020809
:101B000008F30108194B1A6802B17047184A1268A5
:101B1000F2B110B501221A60F4F756FB04460A2010
:101B2000FA34FAF771FBC0B11249134B83600B68AA
:101B3000446000220260C2601BB907E019461B68BE
:101B40001BB15A68A21A002AF8DA0360086010BDB7
:101B50000A4A1268002ADCD1D7E7BDE81040084BDA
:101B600008490948BE2209F09DBD00BF440A012072
:101B7000E0090120400A0120811A0108F80901202A
:101B80006C160208A016020808F301082DE9F843B4
:101B90001E4C1F4FDFF88C801E4E04F1300554F8A8
:101BA000089FB9F1804F22D2F4F70EFB03460A20BA
:101BB0009944FAF729FB10B31749184A0B68C0F883
:101BC00004904FF0000CC0E90224C0F800C01BB91B
:101BD00008E019461B6823B15A68A9EB0202002AE3
:101BE000F7DA03600860AC42D9D1BDE8F8833B4620
:101BF00040F229124146304609F054FDD4E7084925
:101C00003B46BE22304609F04DFDECE718170208AE
